:020000040800F2
:10000000000001207DCF0508FDCF050831A20408BE
:1000100095A20408FDCF0508FDCF050800000000EB
:10002000000000000000000000000000FDCF0508F7
:10003000FDCF050800000000FDCF0508A15F040802
:10004000FDCF0508FDCF0508FDCF0508FDCF05084C
:10005000FDCF0508FDCF0508D1AD0408FDAE0408AD
:10006000C1AE040885AE040849AE040839B10508DC
:1000700029B1050819B1050809B10508F5B0050849
:10008000E1B00508CDB00508FDCF0508FDCF050896
:10009000FDCF0508FDCF0508FDCF05080DAE04080E
:1000A0002D750508B57505081D750508DD7505086C
:1000B000A57505089575050885750508C9B805086D
:1000C000EDB80508FDCF0508FDCF0508FDCF0508F3
:1000D000FDCF050831690408E9660408A164040835
:1000E00095AD0408FDCF0508FDCF05080D75050881
:1000F0003D750508FDCF050865750508B9B005080B
:10010000FDCF0508FDCF050875750508FDCF05086D
:1001100059620408FDCF0508FDCF0508E1F4000889
:10012000A5B0050891B005087DB0050869B00508BF
:1001300055B00508000000000000000000000000AD
:1001400000000000000000000000000065F9000849
:1001500041B005082DB0050819B005081160040864
:10016000FDCF0508FDCF0508FDCF0508FDCF05082B
:10017000FDCF0508FDCF05080000000000000000CD
:10018000FDCF0508FDCF0508FDCF0508FDCF05080B
:10019000FDCF0508FDCF050800000000FDCF0508D4
:1001A000000000000000000000000000FDCF050876
:1001B000FDCF0508FDCF050800000000000000008D
:1001C000000000000000000000000000000000002F
:1001D000000000000000000000000000FDCF050846
:0801E000D4CA05000100000073
:1001E8000E020100020000001C4D01207C4D012080
:1001F800000000006809000823200100100000002A
:100208006C4C0120804D01200000000019260208D6
:100218000D10010058000000084C0120904D0120ED
:10022800000000007DF203080400080080000000C0
:10023800484B0120E84D01200000000000000000AC
:10024800FB01010001000000E04A0120684E012086
:1002580000000000E9470508FC0101000900000052
:10026800AC4901206C4E012000000000F947050848
:10027800F701010006000000A0490120784E012086
:10028800000000006A090008F901010004000000EC
:100298009C490120804E01200000000065380408B8
:1002A8000A8001002800000074490120844E0120C2
:1002B8000000000005250208160215003F00000096
:1002C800542A0120AC4E012000000000CD4805084A
:1002D8003400010010000000A0480120EC4E01206D
:1002E80000000000B9BF0208110201000800000068
:1002F80078480120FC4E0120000000007009000829
:10030800121201000400000070480120044F01206F
:1003180000000000780900081820010032000000E1
:100328003C480120084F0120000000003D49050815
:10033800061001001C000000382A01203C4F012053
:100348000000000019480508FD0101002100000017
:1003580030470120584F012000000000B73704083B
:100368001220010011000000AC4401207C4F012044
:10037800000000007C090008000201000B000000DA
:10038800E8410120904F012000000000513F05087E
:10039800FF110100060000008C4101209C4F012044
:1003A80000000000013F05080812040014000000C6
:1003B80098410120A44F012000000000593F050882
:1003C8001302010004000000342A0120B84F012064
:1003D800000000008E090008FA0101000300000077
:1003E80048410120BC4F012000000000353F0508AE
:1003F8000202010003000000303B0120C04F012031
:1004080000000000000000000C02010004000000D1
:100418000C3B0120C44F0120000000001D3F0508CF
:10042800FE01010014000000D4350120C84F01204E
:1004380000000000793E05080B3001001A0000009A
:10044800006A0120A46C0120000000009409000843
:100458001F30010024000000C8690120C06C012081
:1004680000000000B00900080502010004000000B7
:10047800AC6A0120E46C012000000000D4090008E7
:10048800030101000A00000068690120E86C0120EE
:100498000000000095270108010201000B00000080
:1004A800B8770120FC7A012000000000413F0508D0
:1004B8001B02010010000000A4770120087B012026
:1004C80000000000C53F05081B1001000C000000DB
:1004D800E0700120187B01200000000049BB0108E2
:1004E80021020100F0000000586F0120247B012048
:1004F800000000002D9D01082312010010000000DB
:10050800D8740120147C012000000000D8090008DC
:10051800371001002E00000020770120247C0120E4
:1005280000000000E809000816100100060000009D
:10053800D0740120547C012000000000160A000835
:100548002F10010022000000D87A01205C7C0120D5
:10055800000000001C0A00081E000100090000003D
:100568000C740120807C0120000000003E0A000875
:100578000510010006000000B07401208C7C0120E9
:1005880000000000480A0008F5810100680000002A
:10059800E86E0120947C01200000000099B0010859
:1005A800FD070100760000002E6E0120FC7C012072
:1005B8000000000019870108261001000E00000045
:1005C800847D0120747D01200000000089850108D8
:1005D800F62101000C0000006C890120D48A01205A
:1005E80000000000500A00081C0202001C00000065
:1005F80010890120248B012000000000554A0508BD
:1006080028200100180000002C890120408B0120BF
:1006180000000000B53702081400010004000000C3
:1006280008890120588B0120000000005C0A00089E
:10063800012001000C000000F08101205C8B0120EA
:1006480000000000600A00080EF003009E01000090
:10065800087F0120688B0120000000007DAE0208A1
:1006680013000100040000001C860120088D0120F1
:10067800000000006C0A00080101010004000000ED
:10068800547E01200C8D01200000000000000000B5
:1006980000010100040000004C7E0120108D0120A3
:1006A80000000000700A00080201010003000000B9
:1006B800487E0120148D01200000000039C1030884
:1006C800220201001C01000068830120188D01200E
:1006D80000000000854805080C200600CC0000003A
:1006E800CC800120348E012000000000F9C00308EE
:1006F80019000100050000002C9C01203C9C0120F1
:1007080000000000740A00081A0001000E00000032
:10071800189B0120449C0120000000007A0A000870
:10072800203201000A000000089A0120549C012090
:100738000000000059AE020815001000700000000B
:10074800C8980120609C0120000000000000000003
:100758002A00080060000000D8970120D09C0120E2
:100768000000000031AE02082C0004001000000058
:10077800409D0120309D01200000000011AC0208BE
:100788002B00120024000000749D0120509D0120C0
:1007980000000000E5AB02082920140078000000E2
:1007A800B8950120989D012000000000000000007D
:1007B8000300010001000000249F01204CA2012039
:1007C8000000000000000000031201003D000000CE
:1007D8000CA2012050A2012000000000880A000895
:1007E80025201E002C010000749F012090A20120EA
:1007F80000000000000000001010010002000000CE
:10080800709E0120BCA3012000000000C60A000859
:10081800F821010006000000149F0120C0A3012058
:1008280000000000C80A0008020001000C000000D7
:1008380080A7012028A80120000000000000000077
:100848002902010040000000B8A6012034A80120B8
:1008580000000000CE0A00080A020100140000008F
:100868002CA6012094A801200000000059C4030808
:100878002802040004000000C4AC0120C0B101201B
:1008880000000000C13F0508270204000400000022
:10089800C0AC0120C4B1012000000000B53F05082C
:1008A8001F0208001000000008AA0120C8B101209A
:1008B80000000000AD3E05081A0201003C000000DF
:1008C800CCA90120D8B1012000000000C9490508C1
:1008D8003810010001000000C0A8012014B2012056
:1008E800000000000E0B00082700010004000000B3
:1008F8009CB20120A0B2012000000000100B0008EB
:100908000702010002000000FCBB012014BC01200A
:1009180000000000140B00081D0202000600000081
:10092800CCBB012018BC0120000000000000000022
:100938000602040010000000D4BB012020BC0120E6
:1009480000000000B1490508100201000100000084
:1009580060DB01205CDB012000000000160B0008B2
:1009680000003D01000000003839000001010101CC
:10097800FFFFFFFF000000010000054D4637530050
:100988000000000200000000013E0000AE014A0124
:100998005E012C0164010100000001000A019A01B6
:1009A800001E0A0000020000000000000001000014
:1009B8000005000001020300000000000000000024
:1009C8000000000000000000008007000000000098
:1009D800000000000000000000000000000000000F
:1009E80020003200C800D00796001400320028000A
:1009F8004C0440060005500014000F000800640075
:100A08000100010005000A000000F4019600C40975
:100A180000001900000000000000000000000000B5
:100A280000000000000000000000000000000000BE
:100A380000000000000000050100000000000000A8
:100A4800200002010000000000000000010000007A
:100A58000202000003000023E8036400040A000106
:100A680014001E0008044430B300000000002801F0
:100A780000007E05EA05B4053200E803D00700004F
:100A8800000000000000000000000000000000005E
:100A9800000000000000000000000000000000004E
:100AA800000000000000000000000000000000003E
:100AB8000000000000000000000000000100000528
:100AC8000101F40114000000000000000000000013
:100AD800000000000000000000000000000000000E
:100AE80000000000000000000000000000000000FE
:100AF80000000000000000000000000000000000EE
:0F0B0800000000000000000020030000003C007F
:100B170000C20100000008000A06000200000040B1
:100B27000100000009026400030100C0320904004B
:100B3700000103000000092111010001223600070E
:100B470005830308000A080B0102020201000904D9
:100B57000100010202010005240010010524010023
:100B67000204240202052406010207058203080085
:100B7700FF09040200020A00000007050102400005
:100B87000007058102400000952C0108952B0108FC
:100B9700055A0108000000002121010861560108DB
:100BA7004D210108000000000000000000000000C7
:100BB7000121010811210108F1200108E1200108A4
:100BC7001A03000000000000000000000000000001
:100BD70000000000000000000000000004030904FA
:100BE70000600240106002400000000000000000AA
:100BF700000B0000000000000000000000000000E3
:100C07000060024028600240010000000000000070
:100C1700060C0000000000000000000000000000BB
:100C27000060024040600240020000000000000037
:100C3700100D000000000000000000000000000090
:100C470000600240586002400300000000000000FE
:100C5700160E000000000000000000000000000069
:100C670000600240706002400400000000000000C5
:100C7700200F00000000000000000000000000003E
:100C8700006002408860024005000000000000008C
:100C97002610000000000000000000000000000017
:100CA70000600240A0600240060000000000000053
:100CB70030110000000000000000000000000000EC
:100CC70000600240B860024007000000000000001A
:100CD700362F0000000000000000000000000000A8
:100CE70000640240106402400000000000000000A1
:100CF70000380000000000000000000000000000B5
:100D07000064024028640240010000000000000067
:100D1700063900000000000000000000000000008D
:100D2700006402404064024002000000000000002E
:100D3700103A000000000000000000000000000062
:100D470000640240586402400300000000000000F5
:100D5700163B00000000000000000000000000003B
:100D670000640240706402400400000000000000BC
:100D7700203C000000000000000000000000000010
:100D87000064024088640240050000000000000083
:100D970026440000000000000000000000000000E2
:100DA70000640240A064024006000000000000004A
:100DB70030450000000000000000000000000000B7
:100DC70000640240B8640240070000000000000011
:100DD7003646000000000000000000000000000090
:100DE700120100020000004083042A57000201029A
:100DF7000301000012010002020000408304405773
:100E0700000201020301000012010002EF0201408B
:100E17008304563200020102030110007D00000026
:100E2700A59D00082D8D00084DCF0008CDCF0008E7
:100E370051D00008D1D1000841200108A98B000832
:100E4700A18B0008010000000000803F0A06000295
:100E5700000000400100000009072000010104C054
:100E67003209040000020806500507058102400008
:100E7700000705010240000009022000010104C02B
:100E870032090400000208065005070581024000E8
:100E9700000705010240000009022000010104C00B
:100EA7003209040000020806500507058102000206
:100EB70000070501020002000A06000200000040C8
:100EC7000100000009022200010100E032090400CC
:100ED7000001030102000921110100012236000768
:100EE70005830308000A000009022200010100E04F
:100EF7003209040000010301020009211101000168
:100F070022360007058303080007000009022200B4
:100F1700010100E032090400000103010200092178
:100F2700110100012236000705830308000A0000AB
:100F37000A06000200000040010000000907430004
:100F4700020104C032090400000102020100052465
:100F570000100105240100010424020205240600F3
:100F6700010705820308001009040100020A0000B6
:100F7700000705010240000007058102400000004C
:100F870009024300020100C0320904000001020205
:100F970001000524001001052401000104240202B8
:100FA7000524060001070582030800100904010053
:100FB700020A00000007050102000200070581027E
:100FC7000002000009024300020100C032090400C8
:100FD700000102020100052400100105240100019F
:100FE70004240202052406000107058203080010F5
:100FF70009040100020A0000000705010240000081
:10100700070581024000000000FF0000000000000B
:101017000000AA550701000001AA550501000008B4
:1010270038130608FF1FFF1F05010905A101A100CD
:1010370005010930093109320933093509340936FF
:1010470009371581257F750895088102050919015A
:10105700290815002501950875018102C0C0000007
:101067000921110100012236002D202D2D202D2DC3
:101077002D2D202D2D2D2D0000000000000000003B
:101087000000000000000000AA550B010000AA554F
:1010970005010000AA550902000000AA5503009F98
:1010A70001000000C0120000010000000000010064
:1010B700E0017EFFFFFFFFFFFF000000FFFFFFFFD4
:1010C70008000000BC7D012000000000947D012085
:1010D70000000000B89B0608349B060800000000CB
:1010E700ADC10308A0860100040000000000000055
:1010F70000000000000000000000000000000000E9
:1011070000000000000000000000000000000000D8
:1011170000000000B89B0608C09B060800000000FE
:101127007D480408E80300000400000000000000F8
:1011370000000000000000000000000000000000A8
:101147000000000000000000000000000000000098
:1011570000000000C89B0608000000000000000017
:10116700B50F00007D000000FF0000000000000038
:101177000000000000000000000000000000000068
:101187000000000000000000000000000000000058
:10119700000000007C1807080000000000000000A5
:1011A700ED0500007D000000FF00000000000000CA
:1011B7000000000000000000000000000000000028
:1011C7000000000000000000000000000000000018
:1011D7000000000034AC060800000000000000001A
:1011E7002D1100007D000000FF000000000000003E
:1011F70000000000000000000000000000000000E8
:1012070000000000000000000000000000000000D7
:1012170000000000D09B060800000000000000004E
:10122700A13F0408E80300000300000000000000DD
:1012370000000000000000000000000000000000A7
:101247000000000000000000000000000000000097
:1012570000000000D49B060800000000000000000A
:10126700953303081027000003000000000000006A
:101277000000000000000000000000000000000067
:101287000000000000000000000000000000000057
:10129700000000008414070800000000DDA7020812
:1012A700E5A204085F7600000500000000000000CA
:1012B7000000000000000000000000000000000027
:1012C7000000000000000000000000000000000017
:1012D70000000000201807080000000000000000C0
:1012E7008DB704081027000001000000000000006F
:1012F70000000000000000000000000000000000E7
:1013070000000000000000000000000000000000D6
:1013170000000000E09B060800000000000000003D
:10132700C5360408E80300000500000000000000BF
:1013370000000000000000000000000000000000A6
:101347000000000000000000000000000000000096
:1013570000000000EC9B06080000000000000000F1
:10136700ADC60308204E0000030000000000000087
:101377000000000000000000000000000000000066
:101387000000000000000000000000000000000056
:1013970000000000FC9B06080000000000000000A1
:1013A70095C40308204E0000030000000000000061
:1013B7000000000000000000000000000000000026
:1013C7000000000000000000000000000000000016
:1013D700000000000C9C0608000000000000000050
:1013E700E1440408400D0300030000000000000072
:1013F70000000000000000000000000000000000E6
:1014070000000000000000000000000000000000D5
:10141700000000001C9C06080000000000000000FF
:1014270081000408102700000100000000000000F0
:1014370000000000000000000000000000000000A5
:101447000000000000000000000000000000000095
:1014570000000000609B060800000000000000007C
:101467001DC701081027000003000000000000004E
:101477000000000000000000000000000000000065
:101487000000000000000000000000000000000055
:1014970000000000249C0608000000000000000077
:1014A700517A0208A0860100010000000000000038
:1014B7000000000000000000000000000000000025
:1014C7000000000000000000000000000000000015
:1014D700000000002C9C060800000000000000002F
:1014E700213E040850C30000010000000000000076
:1014F70000000000000000000000000000000000E5
:1015070000000000000000000000000000000000D4
:1015170000000000349C06080000000000000000E6
:10152700113A0408A8610000010000000000000053
:1015370000000000000000000000000000000000A4
:101547000000000000000000000000000000000094
:1015570000000000409C060800000000000000009A
:1015670075500208A086010001000000000000007D
:101577000000000000000000000000000000000064
:101587000000000000000000000000000000000054
:10159700000000004C9C060800000000000000004E
:1015A7000D700408A00F00000100000000000000FB
:1015B7000000000000000000000000000000000024
:1015C7000000000000000000000000000000000014
:1015D70000000000589C0608000000000000000002
:1015E70009010208102700000100000000000000A8
:1015F70000000000000000000000000000000000E4
:1016070000000000000000000000000000000000D3
:1016170000000000649C06080000000000000000B5
:1016270035F901081A410000010000000000000020
:1016370000000000000000000000000000000000A3
:101647000000000000000000000000000000000093
:1016570000000000689C0608000000000000000071
:10166700CD2701081027000001000000000000003E
:101677000000000000000000000000000000000063
:101687000000000000000000000000000000000053
:1016970000000000489B0608000000000000000052
:1016A700E159020850C300000100000000000000DB
:1016B7000000000000000000000000000000000023
:1016C7000000000000000000000000000000000013
:1016D70000000000749C06080000000000000000E5
:1016E700E12F0108400D030000000000000000008A
:1016F70000000000000000000000000000000000E3
:1017070000000000000000000000000000000000D2
:10171700000000007C9C060800000000000000009C
:101727003DC20308400D0300000000000000000058
:1017370000000000000000000000000000000000A2
:101747000000000000000000000000000000000092
:1017570000000000849C0608000000000000000054
:10176700D50C020850C30000030000000000000071
:101777000000000000000000000000000000000062
:101787000000000000000000000000000000000052
:1017970000000000909C0608000000000000000008
:1017A700F9D4030840420F000000000000000000C9
:1017B7000000000000000000000000000000000022
:1017C7000000000000000000000000000000000012
:1017D700000000009C9C06080000000000000000BC
:1017E700BDC9030850C3000000000000000000004E
:1017F70000000000000000000000000000000000E2
:1018070000000000000000000000000000000000D1
:101817000000000001FF010001000000651B020835
:101827000000000000000000681B06080000000020
:10183700000000000000000010350608000000004E
:101847000000000000000000C83506080000000086
:1018570000000000000000007435060800000000CA
:1018670000000000A92C0208C1820120010100002C
:10187700893D020800000000000000009C360608B1
:10188700B1400208000000000000000054360608BE
:101897002D202D2D202D2D2D2D202D2D2D0000001F
:1018A7000000000000000000000000000000000031
:1018B700FFFFFFFF013102080000000000000000E9
:1018C700A034060801000000FA0000000100000033
:1018D70001000000010000000001010100000000FC
:1018E700E88101200000F40101000000E6810120E9
:1018F7000000F40101000000E48101200000F40170
:1019070001000000E28101200000F4010100000055
:10191700E08101200000F40101000000DE810120C8
:101927000000F40101000000DC8101200000F40147
:1019370001000000512302081523020800000000DF
:1019470020210608CC81012005320100DA8101201F
:101957006400F40101000000D88101206400C4097B
:1019670001000000CA810120E803D0070100000040
:10197700C8810120E803D00701000000C6810120CB
:10198700E803D00701000000C48101201E00B80B46
:1019970001000000D281012005000F0001000000B6
:1019A700D481012003000A0001000000C281012048
:1019B7001E00F40101000000D68101200200000092
:1019C700AC210608C081012014006400010000005A
:1019D700CE8101203200E80301000000BE81012012
:1019E7000000C80001000000C980012000C80100F4
:1019F700C880012000500100C7800120005A010063
:101A0700C580012002000000B821060874A306085B
:101A17007CA30608C24C01200100C4090000000095
:101A2700C04C01200100C40900000000BE4C012089
:101A37000100C40900000000BC4C01200100C409DA
:101A470000000000B84C01200100C409000000009C
:101A5700BA4C01200100C40900000000B64C012067
:101A67000100C40900000000B44C01200100C409B2
:101A770000000000737E012000C80100727E012073
:101A870000C80100707E01200000FFFF0A0000006F
:101A97006E7E01200100C800010000006C7E01205D
:101AA70032003075320000006A7E01207EFF14008C
:101AB70005000000687E012005002C0105000000DC
:101AC700667E0120055A0500637E012000FF0100A4
:101AD700657E012002000000FC0E0120617E0120CE
:101AE7000300000084150608627E012000FF010044
:101AF700647E012002000000FC0E0120607E0120B0
:101B07000300000084150608A522020835220208F2
:101B170000000000C421060800820120EE02CA0866
:101B270001000000FE81012000C8010064000000E0
:101B3700FD81012000C8010064000000FC81012034
:101B470002000000D02206085A7E01200000803ED5
:101B570005000000587E012080C1803E050000007E
:101B6700527E01200083007D05000000507E012089
:101B770080C1803E050000004B7E012000FF010070
:101B8700447E01206400F40101000000427E012030
:101B970004000000DC220608417E0120020000004C
:101BA700F0220608F97E01200D000000FC2206083D
:101BB700F67E012000640100F47E01203200102728
:101BC7000A000000F27E01200D000000FC2206083A
:101BD700F17E01200D000000FC220608F07E0120A6
:101BE7000200000034230608000000000000000087
:101BF7000000000040230608068201203E00000086
:101C070078230608048201200100FF7F01000000FD
:101C1700038201200200000074240608FB7E0120D5
:101C27000300000084240608FA7E01200300000058
:101C370084240608B6800120000A0100B480012030
:101C47000000E80301000000B28001200000E80363
:101C570001000000B08001200000E803010000003F
:101C6700AE8001200000E80301000000A6800120EB
:101C77000000E80301000000AC8001200000E80339
:101C870001000000AA8001200000E8030100000015
:101C9700A880012000140100C48001200200000078
:101CA70094240608C28001200000F401010000000E
:101CB700C08001200000F40101000000BE80012067
:101CC7000000F40101000000BC8001200000F401C5
:101CD70001000000BA8001200000A00F01000000F1
:101CE700B88001200000A00F01000000AB81012097
:101CF70019640100AA81012002000000A02406083F
:101D0700A8810120E803D0070A000000A68101206E
:101D1700006401000A0000009B81012000640100AB
:101D27009A81012000640100A28101200064010062
:101D37000A000000A1810120006401000A000000E0
:101D4700A0810120006401000A000000A581012094
:101D570000FF01000A000000A481012000FF01002C
:101D67000A000000A381012000FF01000A00000013
:101D77009F81012001FF01000A0000009E810120D0
:101D870001FF01000A0000009D81012001FF010001
:101D97000A000000047F01200000F4010100000098
:101DA700027F01200000A00F01000000007F01203A
:101DB7000000A00F01000000FE7E01200000A00F20
:101DC70001000000FC7E01200000A00F01000000C0
:101DD7000983012000C80100088301200064010075
:101DE70007830120006401000683012000640100CD
:101DF700058301200064010004830120FF0801001E
:101E070003830120016401009D210208612102086A
:101E170000000000AC2406080C83012001320100F9
:101E27000B830120010000001C2506080A830120FE
:101E37000400000024250608028301200064010035
:101E4700008301201400E80301000000FE82012046
:101E5700E80330750A000000FD82012000C8010078
:101E6700FC82012000C80100FB82012000C801009C
:101E7700FA820120003201000E830120004B01008D
:101E87000D8301200400000038250608F98201208F
:101E9700006401000A0000001C8301200000D00735
:101EA700010000001783012000C8010016830120EC
:101EB70000C801001583012000C801001A83012012
:101EC7000000D007010000001483012000C80100B2
:101ED7001383012000C801001283012000C80100FC
:101EE700188301200000D0070100000011830120A2
:101EF70000C801001083012000C801000F830120E2
:101F070000C80100551F02083D1F0208000000001D
:101F17004C250608ED7E0120005A0100EC7E0120C9
:101F270000C80100EA7E0120E803D0070100000095
:101F37000000000000000000E92C0208E825060860
:101F47004D4154454B463732324D494E490000000A
:101F57005F7E0120000301005E7E01200003010077
:101F6700791E02082D1E0208000000003C26060804
:101F7700ED1D0208A51D020800000000D82606086E
:101F8700C51E0208E53002080000000058270608B1
:101F97005C7E0120010301002D24020801240208B0
:101FA70000000000B02A0608291D0208DD1C0208EF
:101FB70000000000202B0608651F02089146020852
:101FC70000000000BC2B06087D35020859240208D2
:101FD70000000000642C0608B51F0208000000007E
:101FE70000000000F02C06089120020839200208A2
:101FF70000000000542D060825210208E9200208E8
:1020070000000000FC2D0608558B0208D9210208A4
:1020170000000000882E0608BD810120010601008E
:10202700FD1F0208C91F020800000000842F0608D0
:102037008B8A02088532020800000000F42F060888
:102047009D8B02084D33020800000000443106084A
:10205700BC810120010301000D1F0208DD1E0208DB
:102067000000000018320608F98B02080000000083
:10207700000000007C320608751D0208CD300208FA
:1020870000000000FC32060800000000000000000D
:1020970000000000883306080D220208C533020835
:1020A70000000000F83306080000000000000000F0
:1020B7000000000010360608586A01209CFF2C011A
:1020C7000000000018850120E0150C170000000033
:1020D7005382012002000000483606083C7E01209A
:1020E70088136F17010000003E7E012088136F17C9
:1020F70000000000064D0120000000000000000065
:10210700044D01200000000000000000024D0120E6
:102117000000000000000000004D0120000000004A
:1021270000000000FE4C012000000000000000003D
:10213700FC4C012000000000000000009405012075
:102147000000000000000000C47D01200300000023
:1021570038370608347E012088136F170100000006
:10216700A26A012088136F17000000001D1C0208D7
:1021770000000000000000004837060854820120D4
:10218700010000009C370608A46A01200100000036
:10219700A83706089A6A012002000000B03706082F
:1021A700000000000000000000000000BC37060827
:1021B700051C02080000000000000000583806084F
:1021C700000000000000000000000000AC38060816
:1021D7000000000000000000000000001C39060895
:1021E700407E012002000000543906089E6A012043
:1021F700E0150C170000000080900120D49001200A
:10220700D60101FFFFFFFFFF0000803F0000000035
:1022170000000000000000000000000000000000B7
:1022270000000000000000000000000000000000A7
:102237000000803F000000000000000000000000D8
:102247000000803F000000000000000000000000C8
:102257000000803F000000000000000000000000B8
:10226700010000000000FA430000FA430000803F2D
:10227700FFFFFFFFFF0000000000000084A801200F
:10228700080000000000000074A8012008000000FA
:10229700C5890008A98900086589000800000000B1
:1022A70059890008458900083189000800000000A5
:1022B7000000000000000000000000002189000865
:1022C7000000000011890008658E0008B98A00081F
:1022D700818A0008958A0008398A0008258A00083B
:1022E700118A0008419200080D89000889880008B2
:1022F70081F7000815F70308000000000000000040
:1023070000000000685E0C0002010000A00F000042
:10231700B80B00000102FFFF01000000FFFF0000F3
:1023270078140708000008020503040000000000F5
:1023370080140708010008020504040000000000DB
:1023470030C106080200FE01011003000000000072
:10235700E8A60608030014020003000000000000BE
:102367008814070804001F0202000800000000008C
:102377009014070805001F02020108000000000072
:10238700FFFFFFFFE12B0108412B01085D57010803
:1023970000000000000000003155010869550108E0
:1023A7000000000000000000000000008520010878
:1023B700752001086520010855200108F553050817
:1023C70021540508E55305080D40050895530508F0
:1023D70041530508FD3F05082C190120E94A050866
:1023E700154005081140050809400508514E050824
:1023F7000540050801400508288C06081F00000055
:102407001C0000001F0000001E0000001F0000004D
:102417001E0000001F0000001F0000001E0000003B
:102427001F0000001E0000001F0000000068214C74
:10243700FFFF0100F4010000C895060800800202B2
:102447001F00000053544D202020202050726F643D
:10245700757420202020202020202020302E30318D
:102467000000000004010000000700000000000059
:102477000000000000020000100000000000000043
:102487000000000007000000B0010000020000008B
:1024970009000000010000008C1901200000000065
:1024A7000000000000000000000000000000000025
:1024B7000000000000000000000000000000000015
:1024C7000000000000000000000000000000000005
:1024D70000000000000000000000000000000000F5
:1024E70000000000000000000000000000000000E5
:0C24F700000000000000000000000000D9
:102503000100000001000000202300200000000063
:0425130020000000A4
:082800000000000000000000D0
:10800000026C03463AB11A6CD20608D50022012050
:1080100083F83C207047426480F83C20F3E71A6CF8
:1080200049494A4811401A6841F00201F0B4196404
:108030004168474D21F44031416041685C6821430B
:1080400041605168186921F48071D3F808C0DF6875
:10805000516054689E6A44EA0024AE4254605468F9
:1080600024F040745460506840EA0C0050609068FE
:1080700020F400609060916841EA0701916054D05B
:108080009068DC6A20F07060906091680E439660A2
:10809000906820F040509060916821439160906812
:1080A0009C6920F002009060916841EA440191606F
:1080B00093F82010002941D05468596A44F40064B0
:1080C000481E5460516821F460415160516841EA92
:1080D00040315160D06A0025DC6920F470005E698F
:1080E000611ED0622846D46A44EA0154D46294687E
:1080F00024F400749460946893F8301044EA4124A6
:108100009460946824F480649460916841EA8621C4
:1081100091605D641A6C22F0030242F001021A645D
:10812000002283F83C20F0BC7047916821F0706118
:108130009160916821F040519160B0E7516821F45D
:1081400000615160C6E700BFFDEEFFFF0023014064
:108150000100000F2DE9F04F022389468A462DEDDC
:10816000108B99B0DFEDCABA14930346169004330E
:10817000159217934FEADA06169DDDF85CC04FEAB8
:10818000CA0305EB46111396F0004FF0000B01EB0C
:10819000061437010390A6EB86020194049706EBC0
:1081A000460E04EBC202041D381D06EB86072C4464
:1081B000C6EBC60802972844029D02EB46174FEA19
:1081C000C808ED0001EBC60602954FEA0E150595AD
:1081D0004FEACE050695139D4FEA451E019D95ED8C
:1081E000007AD34492ED005AD7ED004AD945D1ED3B
:1081F000006A50ED013A35EE241AD6ED002A1CED46
:10820000016A73EE875A54ED017A33EEC73A36EEBF
:10821000264A77EEA21A36EE666A77EEE27A74EEB6
:10822000256A71EE812A77EE633A37EEC57A36EE2B
:10823000A22A77EEE47A76EEE26A0CED012A37EEB6
:10824000247A77EE857AD1ED018AC1ED006A74EE69
:10825000655A96ED015AB0EE460A94ED004AA7EE33
:108260002B6AD2ED010AE7EEAB3A74EE456AD7ED20
:10827000012AA7EE6B0A9CED007AD5ED014A34EE97
:10828000054A37EE689A90ED005A36EEE02A76EE0F
:10829000E26A30EEA28A32EE222A76EEA06AF0EE90
:1082A000492A75EE640A37EE287A75EE249AE2EED2
:1082B0006B2A74EEC54AF0EE608AB0EE40AAE6EE94
:1082C000AB4AE6EEAB8AA6EEEBAAF0EE496AB0EE58
:1082D000629A37EE695AE2EE2B6AB0EE432A74EEE8
:1082E00008AAA7EEEB9AA7EEAB2A77EE297A35EE2D
:1082F000617A75EEC89A35EE415A75EEC45A37EE7A
:10830000AABA77EEEA7A37EE011A8CED00BA36EEA9
:10831000287AC1ED017A39EE844A76EEC27A1944A0
:1083200075EE885A9C4435EE215A00ED014A70EEF4
:108330008A0A70EE244AC5ED005A36EE686A80ED6E
:10834000001A72EEA33A85ED015A33EE093A04EDB4
:10835000017A72EE266A87ED006A1D44C6ED000AB6
:108360001844C2ED004AC4ED007A1C44C7ED016A0E
:108370001F44C6ED013A1E4482ED013A1A443FF60D
:108380002EAF139A072A40F2C681039A0EF1080E07
:10839000169F08F108000832029E059D4FF0000864
:1083A00094463A46083608357244069C0499D346EA
:1083B000109207EB0C0208340C310F92BA190E928E
:1083C0007A190D923A190C923A180B927A1809926E
:1083D00007F10C020A9201220892149ADDF824C0D7
:1083E0009044159A0A9F02EBC8020B9EA8EB880ED8
:1083F0000C9D02EBC80192ED00BA0D9C01EBC80286
:10840000D1ED00AA0E9802EBC80192ED00AA01EB93
:10841000C802D1ED009A02EBC80192ED009A01EB7F
:10842000C802D1ED008A0F9902EB0E1E92ED008A70
:10843000109A0EEBC80ADEED017A1192CDED047AA6
:108440000AEBC802DAED017A02EBC80A1291CDED0F
:10845000057AD2ED017A0AEBC802DDF820E0CDED15
:10846000017ADAED017A02EBC80ACDED067AD2ED97
:10847000017A0AEBC802CDED027ADAED017ACDED90
:10848000077AD2ED017ADDE91121CDED037A01E021
:10849000F304353F17ED017ADE44D2ED007A94ED16
:1084A000005AF145D5ED006A37EE274AD0ED004A73
:1084B00077EE677A1CED016A96ED007A91ED001A6D
:1084C00076EE055A36EE872A97ED00DA71EE24EA49
:1084D00076EE453A74EE252A31EE641A35EE466A98
:1084E0003EEE825A74EE655A31EE664A72EE854A65
:1084F00031EE471AB0EE67CA47ED014A34EE077A0B
:10850000D1ED014A31EE261AD0ED016A72EEC52A8C
:1085100095ED014AA7EE6BCA74EEE60A96ED010AE4
:10852000E7EE2B7A92ED017A94ED015A74EEA64AA9
:108530003DEE473ADCED006A70EEC4CA70EEC00A48
:10854000B0EE43EA7CEE80CA74EE001A70EE840A44
:10855000ACEEEBEA36EEC54A3DEE077AB0EE63DAF2
:1085600036EE850AACEEAB3AF0EE4EDAA1EE2BDA3F
:10857000A1EE2B6AE1EE6BDA75EE666AB0EE441A94
:10858000F0EE4CCA37EE405AA0EEAB1AE0EEEBCA62
:10859000E0EEAB6A37EE007A74EEA10A35EEE1FA4E
:1085A00075EEE45A75EE6EFA37EE600A71EEA55A72
:1085B000DDED061A35EE425A7FEE244A3FEE822A5E
:1085C00022EEE1FA61EE80FADDED051A3EEE855A03
:1085D0003EEE066A73EEAD3A21EE82EA73EE4DDAB4
:1085E0003DEE033A24EEE1DADDED071A34EE2C4AD3
:1085F0007CEE266A61EE85CA25EEE1CADDED041A3D
:1086000077EE81EA77EEC17AE9EEA2FADDED032A90
:10861000A9EE80FA9DED030AAAEEA4EADDED014A77
:10862000AAEE82DA9DED012AE8EEA5CADDED025A36
:10863000A8EE85CA9DED025A21EEAD1A62EE832A9C
:108640006EEEE11A27EEC00A64EEA34A26EEC22AB5
:1086500065EE865A24EE455AABEE2E1AEBEE2D1A35
:10866000E8EE272AA8EE030AEAEE264AAAEE232A13
:10867000E9EE045AA9EE065A37EE207A87ED007A21
:108680001F44C2ED00FA82ED01FA1A440CED01EA32
:108690008CED00DA9C44C4ED00CA84ED01CA1C4490
:1086A00081ED001AC1ED011A1944C6ED002A86EDCC
:1086B000010A1E44C0ED005A80ED015A1844C5ED70
:1086C000004A85ED012A1D443FF6E4AE1099089A50
:1086D0000831013210910F99089208310F910E99CB
:1086E00008310E910D9908310D910C9908310C91BA
:1086F0000B9908310B910A9908310A9109990831AF
:108700000991139991427FF468AE149B8A46DB006D
:108710009BB214932EE519B0BDEC108BBDE8F08F21
:10872000124B30B41D686B6A28B943EA014300203C
:10873000AB6230BC7047AC6A013803EB14440BD019
:10874000002303F14002013305EB8202DBB25268E1
:10875000834204EB1244F4D3403044EA014405EB75
:1087600080004460002030BC704700BFF019012039
:10877000037870B42BB30246C0F10105531912F807
:10878000014FDBB2002CF9D101335B000E4C032208
:108790000B8084F8043484F80524017879B102232D
:1087A00000265A1CE518023354FA82F285F80414A4
:1087B000DBB282F8046410F8011F0029F1D170BC0B
:1087C00070470223E2E700BFF0190120F0B40F4B1D
:1087D000C40800F0070700221E5D03EBD005BE4071
:1087E000F6B2C7F1080300278B4228BF0B46C3F13E
:1087F00008049A40C91A46FA04F415F8016F42EACF
:108800000402EED11046F0BC704700BF341F0120B7
:1088100030B5EFF31181802383F312880A4AD2F82E
:108820007835D2F87C45D2F87805D2F87C55CAB2B2
:1088300082F31188013BA84294BF4FF400600020EE
:108840001B1B184430BD00BFF0190120012380F824
:1088500051307047014BD3F880057047F019012063
:1088600001207047024BC3F88425C3F88815704770
:10887000F0190120024BC3F88C25C3F890157047FE
:10888000F019012070477047212870B505D02228C3
:1088900029D0202810D0002070BD0029FBD0072A45
:1088A000F9D1184B18791C685A799B790871002006
:1088B0000C604A718B7170BD0029ECD0072AEAD197
:1088C0001148104B0C680E794D79D0F888258979BC
:1088D0001C601E715D719971002ADCD02146D0F8B0
:1088E00084059047D7E70029D5D0022AD3D1064A7C
:1088F000D2F89035002BCED00988D2F88C05984755
:10890000C9E700BF00000120F019012000207047D6
:1089100003460A2201481A80704700BF0800012060
:108920000346642201481A80704700BF14000120EA
:10893000012901D000207047014BD3F8903018472F
:1089400000000120012901D009F0ACBB014BD3F894
:108950008C30184700000120014BD3F888301847AD
:108960000000012010B40B780A46044603F003030C
:10897000012B05D0022B0BD000205DF8044B704773
:108980008B8843B9204611465DF8044B0CF0B4BF08
:108990008B88832BF6D0034B5DF8044BD3F88030E3
:1089A000184700BF0000012038B5054B04460D46AE
:1089B000DB6F9847294620460AF0DAF8002038BDD8
:1089C0000000012038B5054B04460D469B6F9847C3
:1089D000294620460AF048F9002038BD0000012051
:1089E000F0B4002452004E1C2746030FB0F1204F74
:1089F0004FEA001003F1300503F1370334BF0D5582
:108A00000B5537550234A242EFD1F0BC704700BF7E
:108A1000024808B5FFF7ACFE014808BD1C960608E1
:108A2000F41D0120024808B5FFF7A2FE014808BD69
:108A30002C960608F41D01200B481A220B4B0068E7
:108A40001B680A80C01801D109487047094B0822E9
:108A5000094910B51C68FFF7C3FF042207492046E7
:108A6000FFF7BEFF024810BD107AF01F187AF01F02
:108A7000B0000120147AF01FB2000120C2000120D2
:108A8000024808B5FFF774FE014808BD389606088D
:108A9000F41D012008B520B90448FFF769FE044819
:108AA00008BD0448FFF764FE014808BD4496060867
:108AB000F41D012068960608042301480B807047C6
:108AC000CC00012098B182680C4B12B107229A7039
:108AD000704718780421DA6003281A611A750CBFF0
:108AE00080224FF480729970C3E901227047034BD2
:108AF000012241F2E4715A705A547047DC4F012050
:108B00000378022B0FD0006908B9012070470E4B83
:108B10001B78032B12D080B24FF6F773984294BFA4
:108B2000002001207047084941F6500243688A58E6
:108B3000B3EB422F2CBF012000207047034B98421B
:108B400094BF002001207047DC4F0120F7FFFF0F8A
:108B500030B40378022B13D0104A41F64801436821
:108B600041F63C04555802F5C25100692B40096892
:108B7000023812595B0A01FB003030BC10447047C8
:108B8000064B41F6300441F63401426818595958F1
:108B900000EB410030BC00EB52207047DC4F01205D
:108BA000004870471C1F0120034B93F82805032839
:108BB00094BF002001207047F01901202DE9F843EF
:108BC000884600294FD04718461E284C802507F1BB
:108BD000FF39EFF3118185F31288D4F87825C9B2F3
:108BE000D4F87C05D4F87835D4F87CC581F31188A5
:108BF000634594BF4FF400630023121A1344012B02
:108C00001AD101203DF028F9EFF3118185F3128884
:108C1000D4F87825C9B2D4F87C05D4F87835D4F8DE
:108C20007C7581F31188BB4294BF4FF4006300232D
:108C3000121A1344012BE4D0EFF3118285F312884A
:108C4000D4F87C35D2B216F8011F234483F894156A
:108C5000D4F87C350133C3F30A03C4F87C3582F3BE
:108C600011884E45B5D14046BDE8F883F019012082
:108C7000F8B5002390F8505080F85030DDB110491D
:108C800041F208028A5C032A17D10E4E00F13C041F
:108C900056F8B87C29462046FFF790FF56F8B83CB6
:108CA0002D1A0444DB1B322B01D8002DF2D1B5FA6A
:108CB00085F04009F8BD0120FCE71846FAE700BF3F
:108CC000F0190120E82A0120002280F85120CFE786
:108CD00090F85020531C0244DBB280F8503082F8E8
:108CE0003C1090F851200AB1132B00D9C0E770470F
:108CF000F8B5144641F208030A4A0D46D35C032B2B
:108D00000FD1094E56F8B87C002C0ADD21462846C2
:108D1000FFF754FF56F8B83C241A0544DB1B322BEE
:108D2000F2D9F8BDF0190120E82A01202DE9F0411F
:108D30004379484C002B14BF0122002284F85425AB
:108D400003D184F82835BDE8F08190F8018005460C
:108D50000F4608F1FF3676B2304642F0A3FA0223FE
:108D6000C4F8600584F85C352B78002B45D1ED788C
:108D7000BDBB4FF48071D4F86005C4F868554DF060
:108D8000C5FF4FF47A703DF067F8D4F8680541F0FC
:108D900027FA00220A23D4F86005114650F07CFA25
:108DA000D4F860152C4B8A6812F4C05F0FD18A6822
:108DB00012F080020BD1294B012184F81C2553F8B5
:108DC000B83C84F82815C4F81835BDE8F081013B9B
:108DD000E9D194F81C2584F82835531C84F81C35F7
:108DE000B1E7284641F0A6F8054608B11E23C38026
:108DF0000D21284641F084F8BBE706EB8606414684
:108E000000203E4496F903203EF092F8064630B129
:108E100040683EF07DF8B26884F8742518B90023E4
:108E200084F86C35A3E7431E0D4A02F1D00102EB32
:108E3000431201EB431392F8E810C4F8703500298F
:108E4000EDD11723A2F8E83052F0D6F8012384F8C8
:108E50006C358CE7F0190120A1860100E82A012079
:108E60000000012010B503200C464FF0F7FE032848
:108E70000AD0074B13F8B43C012B4FF012030CBF80
:108E800004480548238010BD12230448238010BDE8
:108E9000E82A0120F8020120E4020120D00201208A
:108EA0002DE9F04FDFF81883BA4D4446DFF82493DC
:108EB0002DED068B89B0CDE9060105920FCD0FC4CB
:108EC0000FCD0FC495E8070019F8AE3C84E8070001
:108ED000042B00F20C81DFE813F037010A010501D1
:108EE000050045019FEDAC8A9FEDAC9AAC4AAD4BB5
:108EF0000598AD49002818BF1346AC4AC8E90621B9
:108F000039EE087ADFEDAA7AF5EE006AA94A28EE72
:108F1000278AA94EB0EE67AA02F11507C6EE879A16
:108F20000025DFEDA68A0292C8F82430079BAB42E9
:108F300000F0D280029B05F1010B13F8014B5FFAA0
:108F40008BF20293002C00F01B81002103E0013121
:108F5000152900F0158101EB41004B0017F800C006
:108F6000A445F4D1484410F8931CCDE903320029FC
:108F700000F00E8120463CF0C9FA824600684EF0AF
:108F8000D7FC9AF805103CF0FFFA0078002840F072
:108F9000F780039B4FEA141E04F00F0C049A09EBB0
:108FA00003010EF1FF34032301F8532C9C4201F816
:108FB000543C00F2C580774901EB4401888D40FAAA
:108FC0000CF111F0010100F0BD800121039201FAC2
:108FD0000CF10139084053F059FE6E4BDFF8F8C12F
:108FE00002211C44039A032394F8344020440CEBE0
:108FF000C00070618371C2719AF8082040F0C4FE0D
:10900000059B002B78D039F8B03C19F8AE1C07EE60
:10901000903AD9F8D8310429F8EEE77AFCEEE77AED
:1090200017EE900AB3FBF0F202F57F4202F1FF0265
:109030004FEA1242B3FBF2F2B2FBF0F083B270D00F
:1090400007EE902AF8EE676A66EE887A28EEE77AED
:1090500019F8AD0C069901903046A9EE267A0091D8
:109060005146C6ED027A86ED037A33F08BFE002D71
:1090700062DD7368D8F8382093425FD0012D5BD051
:10908000D8F85020934259D0022D55D0D8F86820F6
:10909000934253D0032D4FD0D8F8802093424DD027
:1090A000042D49D0D8F89820934247D0052D43D0BD
:1090B000D8F8B020934241D0062D3DD0D8F8C82032
:1090C000D31A18BF01235D46012233741836082DC8
:1090D00006F8072C7FF42AAF394809B0BDEC068B9F
:1090E000BDE8F08F9FED378AB0EE489AFEE69FED1F
:1090F000368AB0EE489AF9E6FAFE697AFCEEE77A2B
:10910000D9F8D8114FF6FF7317EE902A1846B1FB25
:10911000F2F21A44120CB1FBF2F219F8AE1C042957
:109120008ED107EE900A07EE102AF8EE677AF8EE75
:10913000476A67EE8A7A89E70123C4E70023C2E71A
:1091400070615DE771615BE70023174A01219FEDC4
:10915000188A0693154BB0EE489A0591C8E9063275
:109160000F4BCDE60023104A01219FED188A06938C
:109170000E4BB0EE489A0591C8E90632084BBFE69F
:10918000134A0020064BC8F81C20C8F82430A4E776
:109190000B68FFDE78070608ACC5A737ACC5A73655
:1091A00045380408E1BC03082DC4030851380408FD
:1091B0006F12833A3F2A01204800002000007A44C1
:1091C00014000020282930386F12033900000000F5
:1091D000CDBF0308E82A0120C02A0120154BDB6817
:1091E000C3F3022310B4C3F107041A1D042C28BFD3
:1091F0000424062A4FF0FF328CBF033B0023A24019
:10920000002821EA020101FA03F108DB09010A4BF7
:10921000C9B2034483F800135DF8044B704700F0B3
:109220000F000901054BC9B2034419765DF8044BE0
:10923000704700BF00ED00E000E100E0FCEC00E062
:1092400030B5264C0022264841F28731D4F8D83177
:1092500083B0244DA0FB030304F5EE70C4F8DC5189
:10926000DB0C013BC4E97A12C4E978320BF0B8FC9C
:109270001D4B062137201A6C42F020021A641B6C29
:1092800003F020030193019BFFF7A8FFD4F8DC3122
:109290004FF400001549164A4860D96841F00101B1
:1092A000D96099680A40062A06D0B2F5803F03D0FB
:1092B0001A6842F001021A600E4B41F224020020AB
:1092C0000D499A5803F29454C3F89005C2F810025D
:1092D000C3F88805C2E9811403B030BDE82A012033
:1092E00083DE1B43001400400038024000E100E030
:1092F00007000100F0190120042D012038B50F4BA3
:109300000F4AD3F8D831A2FB03239B09013BB3F1E9
:10931000807F10D20B4A0024F0200B4907255360B0
:1093200081F82300214694604FF0FF301560FFF76D
:1093300055FF204638BD012038BD00BFE82A012076
:10934000D34D621010E000E000ED00E0430901227F
:1093500000F01F0084B0013B02FA00F0032B0BD891
:10936000DFE803F015021E0C124B5A6C02435A64DC
:109370005A6C10400090009B04B070470D4B1A6B64
:1093800002431A631A6B10400390039BF4E7094BE6
:109390005A6B02435A635A6B10400290029BEBE7F0
:1093A000044B1A6C02431A641A6C10400190019B22
:1093B000E2E700BF0038024018B10022012140F06E
:1093C000E3BC704718B10022202140F0DDBC70479B
:1093D00000487047202B0120002800F08F80B0F853
:1093E00004C0BCFA8CF3202BC3F11F0200F086806E
:1093F0006F4B2DE9F04F9D18DFF8E48185B00368CD
:1094000008EB820095F838200024DFF8D8E10192BB
:10941000C0F81C1A674A02E00134102C65D04FF0E6
:10942000010909FA04F10CEA010531EA0C01F3D152
:109430004FF0030A04FA09F718684FF00F0B0AFA05
:1094400007F704EA0A0124F0030620EA070089006E
:1094500006F1804618600BFA01F0D3F80CB006F55F
:109460009C362BEA0707DF60DEF8447047F480473C
:10947000CEF84470DEF8447007F480470397039FEA
:10948000B76827EA00004C4FBB421AD007F5806747
:10949000BB4234D0494FBB4235D0494FBB426BD061
:1094A000484FBB4271D0484FBB4269D0474FBB4287
:1094B00078D0474FBB420CBF0727082707FA01F1B6
:1094C0000843B06001341168102C41EA05011160B5
:1094D000516821EA05015160916841EA05019160F6
:1094E000D16821EA0505D56099D1019B984498F887
:1094F0005C3AF02B0CD805B0BDE8F08F704709FA44
:1095000001F10843DDE7022707FA01F10843D8E734
:10951000F021304B264888F85C1AD968019AC1F3CB
:1095200002210244C1F107000B1D92F848400428B3
:1095300092F9482028BF0420062B4FF0FF338CBF40
:10954000033900218340002A6FEA030303F0030379
:1095500003FA01F31EDB204801211B0104F01F0464
:1095600085185209DBB201FA04F485F8003340F89B
:10957000224005B0BDE8F08F0AFA01F10843A0E7E8
:10958000052707FA01F108439BE7042707FA01F1D1
:10959000084396E704F00F041B01104ADBB2224493
:1095A0001376A8E7062707FA01F1084389E700BF09
:1095B00078070608003C0140000002400008024015
:1095C000000C02400010024000140240001802404B
:1095D000001C024000ED00E000E100E0FCEC00E0D7
:1095E000E82A0120003802402DE9F041D0F800E0DF
:1095F0000C46DFF8588084B0DEF804501746DFF8D8
:1096000050C0194605EA0805DDF828800646039390
:109610002C43424644EA0C0CCEF804C00CF062FF26
:1096200078B931680246039B30468F624021CDF8FD
:1096300000800CF087FF003818BF012004B0BDE89F
:10964000F081012004B0BDE8F08100BF009800FC6B
:1096500000200180F8B5134F04460D460AE09B69CF
:10966000DB0602D50CF0FEFED0B9D7F8643A5B1BDE
:109670000A2B08D823682A460A2120469E69B60686
:10968000EDD50020F8BD636C2021002201200B43A2
:1096900084F84020636484F8411084F84220F8BDC7
:1096A0000120F8BDE82A012030B5037883B00446D4
:1096B0001546012B1DD0022B18D1C36841F0800143
:1096C0001BB19A88186812048261606850F02AF809
:1096D00001232A46002160684FF0DEFDE3688BB16C
:1096E0001A6801209B88936103B030BD002003B04D
:1096F00030BD00920A46417990F9040051F024FDF2
:1097000003B030BD0120F2E72DE9F047C94C054612
:1097100094F8681AD4F8700AC1F3400140F066FD6D
:1097200094F8681AD4F86C0AC94301F0010140F0BA
:109730005DFD002D00F0E58005F1FF38BE4E1027DD
:10974000BE4D5FFA88F8D4F8703A33B11A689B8836
:1097500051690B4218BF1B049361D4F86C3A33B1C2
:109760001A689B8851690B4218BF1B049361B4F8B7
:10977000783A002B40F0558194F87A1AD4F87C0A94
:1097800040F034FD4FF0FA0C4FF47A704FF0010EB8
:109790007368C3F30803002B40F01781EFF31183C4
:1097A000002B40F0128154F8B82CA96854F8B83C4A
:1097B0009A42F8D1D4F8A03A9942F4D8D4F89C9AB5
:1097C00000FB09F35B1AB3FBF9F300FB0232736889
:1097D000C3F30803002B40F0B780EFF31183002B95
:1097E00040F0B28054F8B83CD5F808A054F8B81C42
:1097F0008B42F7D1D4F8A01A8A45F3D8D4F89C9AB2
:1098000000FB09F1A1EB0A01B1FBF9F100FB031325
:109810009B1AB3F57A7FDAD3BCF1010CB8D1D4F836
:10982000703A33B11A689B8851690B4218BF1B0408
:109830009361D4F86C3A33B11A689B8851690B4232
:1098400018BF1B049361B4F8783A002B40F0DD8018
:1098500094F87A1AD4F87C0A81F0010140F0C6FC31
:109860004FF0FA0C4FF47A704FF0010E7368C3F3A7
:109870000803002B40F08980EFF31183002B40F0A8
:10988000848054F8B82CA96854F8B83C9A42F8D1AE
:10989000D4F8A03A9942F4D8D4F89C9A00FB09F382
:1098A0005B1AB3FBF9F300FB02327368C3F30803DE
:1098B0004BBBEFF3118333BB54F8B83CD5F808A089
:1098C00054F8B81C8B42F7D1D4F8A01A8A45F3D8C3
:1098D000D4F89C9A00FB09F1A1EB0A01B1FBF9F164
:1098E00000FB03139B1AB3F57A7FDED3BCF1010CA6
:1098F000BCD108F1FF385FFA88F8B8F1FF0F7FF4A8
:1099000022AFBDE8F087EFF3118987F31288D5F80D
:1099100008A02B68DB0303D5C4F898EAD5F808A0A3
:1099200054F8B83C5FFA89F9D4F8981A89F3118889
:10993000D4F89C9A0B4400FB09F1A1EB0A01B1FB9E
:10994000F9F100FB0313CDE7EFF3118987F31288D8
:10995000D5F808A02B68D90303D5C4F898EAD5F840
:1099600008A054F8B83C5FFA89F9D4F8981A89F33A
:109970001188D4F89C9A0B4400FB09F1A1EB0A0171
:10998000B1FBF9F100FB031342E7EFF3118187F319
:109990001288D5F808902B68DA0303D5C4F898EA42
:1099A000D5F8089054F8B83CC9B2D4F8982A81F395
:1099B0001188D4F89C1A1A4400FB01F3A3EB0903A5
:1099C000B3FBF1F300FB02326FE7EFF3118187F392
:1099D0001288D5F808902B68DB0303D5C4F898EA01
:1099E000D5F8089054F8B83CC9B2D4F8982A81F355
:1099F0001188D4F89C1A1A4400FB01F3A3EB090365
:109A0000B3FBF1F300FB0232E1E6D4F8943A002B09
:109A10003FF426AF0023D4F8802A136084F8913AEB
:109A20001EE7D4F8943A002B3FF4ACAE3CF0DEFADB
:109A3000A8E600BFE82A012000ED00E010E000E009
:109A40002DE9F84FC44C4FF0050BC44F4FF01008F0
:109A500094F8681AD4F8700AC1F34001C04D40F080
:109A6000C5FB94F8681AD4F86C0AC94301F00101E7
:109A700040F0BCFBD4F8703A33B11A689B88516946
:109A80000B4218BF1B049361D4F86C3A33B11A68C7
:109A90009B8851690B4218BF1B049361B4F8783A54
:109AA000002B40F0518194F87A1AD4F87C0A40F0E7
:109AB0009DFB4FF0320C4FF47A7001267B68C3F3A4
:109AC0000803002B40F01481EFF31183002B40F0CA
:109AD0000F8154F8B82CA96854F8B83C9A42F8D1D0
:109AE000D4F8A03A9942F4D8D4F89C9A00FB09F330
:109AF0005B1AB3FBF9F300FB02327B68C3F3080384
:109B0000002B40F0B480EFF31183002B40F0AF80C6
:109B100054F8B83CD5F808A054F8B81C8B42F7D1DB
:109B2000D4F8A01A8A45F3D8D4F89C9A00FB09F11E
:109B3000A1EB0A01B1FBF9F100FB03139B1AB3F58A
:109B40007A7FDAD3BCF1010CB8D1D4F8703A33B1D2
:109B50001A689B8851690B4218BF1B049361D4F8A3
:109B60006C3A33B11A689B8851690B4218BF1B04C9
:109B70009361B4F8783A002B40F0DA8094F87A1ABE
:109B8000D4F87C0A81F0010140F030FB4FF0320C38
:109B90004FF47A7001267B68C3F30803002B40F072
:109BA0008780EFF31183002B40F0828054F8B82CAB
:109BB000A96854F8B83C9A42F8D1D4F8A03A99422E
:109BC000F4D8D4F89C9A00FB09F35B1AB3FBF9F3C1
:109BD00000FB02327B68C3F308033BBBEFF3118346
:109BE00023BB54F8B83CD5F808A054F8B81C8B42F5
:109BF000F7D1D4F8A01A8A45F3D8D4F89C9A00FB80
:109C000009F1A1EB0A01B1FBF9F100FB03139B1A67
:109C1000B3F57A7FDED3BCF1010CBCD10BF1FF367A
:109C200016F0FF0B7FF426AFBDE8F88FEFF3118934
:109C300088F31288D5F808A02B68DB0303D5C4F895
:109C4000986AD5F808A054F8B83C5FFA89F9D4F8B6
:109C5000981A89F31188D4F89C9A0B4400FB09F1F7
:109C6000A1EB0A01B1FBF9F100FB0313CFE7EFF31E
:109C7000118988F31288D5F808A02B68D90303D579
:109C8000C4F8986AD5F808A054F8B83C5FFA89F986
:109C9000D4F8981A89F31188D4F89C9A0B4400FBE5
:109CA00009F1A1EB0A01B1FBF9F100FB031345E750
:109CB000EFF3118188F31288D5F808902B68DA0346
:109CC00003D5C4F8986AD5F8089054F8B83CC9B2DE
:109CD000D4F8982A81F31188D4F89C1A1A4400FB0E
:109CE00001F3A3EB0903B3FBF1F300FB023271E7CD
:109CF000EFF3118188F31288D5F808902B68DB0305
:109D000003D5C4F8986AD5F8089054F8B83CC9B29D
:109D1000D4F8982A81F31188D4F89C1A1A4400FBCD
:109D200001F3A3EB0903B3FBF1F300FB0232E4E61A
:109D3000D4F8943A002B3FF429AF0023D4F8802ABA
:109D4000136084F8913A21E7D4F8943A002B3FF459
:109D5000B0AE3CF04BF9ACE6E82A012000ED00E0A3
:109D600010E000E010B4B8B10D4CD4F8A43A102BB8
:109D700005D1052100205DF8044B3BF009BE03EB43
:109D80004302224482F8A91A012182F8A80A0B444E
:109D900082F8AA1AC4F8A43A5DF8044B704700BFD1
:109DA000E82A01202021C078DCE700BF2DE9F04F30
:109DB000BC4C002387B004F6D82894F8EC2AC4F8E9
:109DC000D83AC8E90133C8E903331AB194F8ED3A37
:109DD00084F8D83A94F8EE3A1BB194F8EF3A84F844
:109DE000E73A94F8F23A1BB194F8F33A84F8E23A7D
:109DF00094F8F03A1BB194F8F13A84F8DD3A94F80B
:109E0000F43A013B4FFA83FADBB2BAF1FF3F029317
:109E100000F02581B022A449A44D002302FB0A11C1
:109E20002E4605F1280050311F469B46019356F0FF
:109E3000F9FA039535785146284641F0EBFB814607
:109E4000002840F00F8101370536042FF2D194F835
:109E5000040B039DFFF77AFA4FF44032944E00232F
:109E60000121C4F80C2B3046D4F8002BC4F824BBD5
:109E7000C4F8201BC4F8181B84F8381BC4F8103B26
:109E8000C4F8303BC4F8343BC4F8143B84F8283B96
:109E9000C4F82C3BC4F81C3BC4F8082BFEF7B0F800
:109EA000BAF1000F40F01881019B83F0010919F00D
:109EB000FF0F40F01181A6F1080051F0A3FD01232E
:109EC00008F11408EA78002A40F04081053545453C
:109ED000F8D104EB0A030299022093F9FC2A3DF021
:109EE00027F80546002800F0BA80D0F804804046E4
:109EF0003DF00EF86F4B421E03EB421393F8E870EF
:109F0000002F40F0AC800622A3F8E820002800F0E3
:109F1000A6804046DFF8B8813CF0FAFF51F06CF8BB
:109F2000BBF1010FA9684FF400638CBF4FF480624E
:109F3000002268684FF40055C4F8541B4FF4807138
:109F4000C4F8602B4FF40032C4F8643B0323C4F818
:109F5000500B4046C4F8783BC4F8587BC4F85C7B8F
:109F6000C4F8747BC4F87C7BC4F8807BC4F8685B5D
:109F7000C4F86C1BC4F8702B0DF020F994F8443B26
:109F8000C4F8408B012BC4F8886B059767D0012378
:109F9000D4F8085B84F8443BAB68DE0713D4D4F8EC
:109FA000D8314549AA68B3FBF1F342F0010203EB53
:109FB0004303AA600593059B2BB1059B013B0593C9
:109FC000059B002BF9D1AB68D80748D5D4F8482BAE
:109FD0003A4B134043F48073C4F8483B6B6859050F
:109FE00007D5D4F8483B23F4405343F48053C4F8D6
:109FF000483BD4F8483B13F4805300F05681D4F822
:10A000004C3B23F00603C4F84C3B2D4800232D495C
:10A010006FF02202C4F8900B2B4884F8443B5B4657
:10A02000C4F88C1B05F14C01C4F89C0B2A606E68C7
:10A03000264A46F0806626486E60AE6846F4807612
:10A04000AE600DF033F8234B5A68D20640F016810B
:10A05000D4F8083B9A6812F0405F00F0218107B005
:10A06000BDE8F08F28463FF065FFFB1D032100226D
:10A07000DBB2CDF8049008B18371C2713FF040FFAC
:10A08000307841F0F9FA0BF1010386F802B05FFA7B
:10A0900083FB4FF00703707033714FF00103F370CF
:10A0A000D1E600BFE82A012078070608C035012064
:10A0B000F03501200000012040420F00FEF8FFFFB4
:10A0C000B5210108B9210108A521010808010020D6
:10A0D0003836012000230140B02200217A48482769
:10A0E00056F012FAB0220021774856F00DFA774B5D
:10A0F000384684F8B47BC4F8B03BFFF727F94FF437
:10A10000403000230121D4F8B02BC4F8BC0B7048B8
:10A11000C4F8D01BC4F8C81B84F8E81BC4F8C03BC3
:10A12000C4F8E03BC4F8E43BC4F8C43BC4F8D43BF7
:10A1300084F8D83BC4F8DC3BC4F8CC3BC4F8B82B5B
:10A14000FDF75EFF604851F05DFCB8E694F8440B03
:10A1500000215A1C2F7901280491D2B269783DD090
:10A160004FF00100092984F8440B4ED94FF0030E3B
:10A170006FF01D00D4F808CB4FF007091EFB01005B
:10A18000DCF80CE009FA00F907FA00F02EEA0907FA
:10A19000CCF80C70DCF80C703843CCF80C00062BB3
:10A1A0004FF005001CD86FF0040710FB0373D4F8C0
:10A1B000087B1F2000FA03FC786B01FA03F320EA06
:10A1C0000C007863786B03437B63D4F8083B3F480B
:10A1D000834230D04FF0000384F8443B134675E6C9
:10A1E0000C2B32D86FF0220710FB0373D4F8080B46
:10A1F0001F2707FA03FC076B01FA03F327EA0C0792
:10A200000763076B3B430363DFE7D4F8080B01EBFD
:10A2100041094FF0070ED0F810C007FA09F70EFAFF
:10A2200009FE2CEA0E0CC0F810C0D0F810C047EAA6
:10A230000C070761B3E712291AD01129CAD12549A1
:10A240004B6843F400034B60C4E76FF0400710FB1A
:10A250000373D4F8080B1F2707FA03FCC76A01FA37
:10A2600003F327EA0C07C762C76A3B43C362ACE744
:10A2700018494B6843F480034B60ABE7D4F8082BD4
:10A2800012498A4214D05B68DB063FF5E8AE124BF8
:10A290009A427FF4E4AE9A6812F0405F7FF4DFAE3A
:10A2A0009A6842F080429A60D9E6C4F84C3BACE62A
:10A2B000936813F0405F03D1936843F08043936049
:10A2C000044B5B68CBE600BF9836012000200140BC
:10A2D000A036012000230140002201402DE9F04179
:10A2E000D0F800E00C46DFF8588084B0DEF8045067
:10A2F0001746DFF850C0194605EA0805DDF8288042
:10A30000064603932C43424644EA0C0CCEF804C0A4
:10A310000CF0E8F878B931680246039B30468F624A
:10A320008021CDF800800CF00DF9003818BF012015
:10A3300004B0BDE8F081012004B0BDE8F08100BFA9
:10A34000009800FC002001810A4610B102213FF074
:10A350001BBD7047034690F83C00012800F03E8189
:10A360000220F0B4012483F83D0083F83C40142A15
:10A3700045D8DFE812F04D004400440044007B0063
:10A38000440044004400DA00440044004400AA00B1
:10A390004400440044000601440044004400150009
:10A3A0001A688E68156A0F6825F48015AB4C156223
:10A3B000106A556820F40010D2F854C040EA0650E4
:10A3C000A74E0CEA0404B24244EA072400F00881D4
:10A3D00006F58066B24200F003814E685560546510
:10A3E000D6651062506D0C6940F400605065506D88
:10A3F00020F480605065516D41EA042151650022CE
:10A400000121104683F83D1083F83C20F0BC7047D2
:10A410001A68D1F808C0156A0F6825F00105914C3B
:10A420001562106A5668956920F002002C408C4D28
:10A4300040EA0C00AA4244EA070400F0DD8005F57A
:10A440008065AA4200F0D8804D68566094615563DB
:10A45000106290690C6940F008009061906920F0EA
:10A4600004009061916921439161C8E71A68D1F8AD
:10A4700008C0156A0F6825F010057B4C1562106A3C
:10A480005668956920F020002C40754D40EA0C106C
:10A49000AA4244EA072400F0C38005F58065AA4279
:10A4A00000F0BE804D6856609461956310629069BB
:10A4B0000C6940F400609061906920F480609061C4
:10A4C000916941EA0421916199E71A688E68156AD9
:10A4D0000F6825F48055644C1562106A556820F4A5
:10A4E0000050D2F81CC040EA06305D4E0CEA04046D
:10A4F000B24244EA072400F08D8006F58066B2423D
:10A5000000F088804E685560D46116641062D0698E
:10A510000C6940F40060D061D06920F48060D061A3
:10A52000D16941EA0421D16169E71A68D1F808C00C
:10A53000156A0F6825F480754A4C1562106A5668D2
:10A54000D56920F400702C40454D40EA0C20AA4209
:10A5500044EA070473D005F58065AA426FD04D68C0
:10A560005660D461D5631062D0690C6940F0080070
:10A57000D061D06920F00400D061D1692143D1615C
:10A580003DE71A688E68156A0F6825F48035374CE8
:10A590001562106A556820F40030D2F854C040EAC1
:10A5A00006402F4E0CEA0404B24244EA07041DD0D0
:10A5B00006F58066B24219D04E68556054659665BE
:10A5C0001062506D0C6940F008005065506D20F02D
:10A5D00004005065516D2143516510E7022070471A
:10A5E00025F480254E6945EA8625F6E625F4803572
:10A5F0004E6945EA0625DFE726F4407C20F0080096
:10A600008E69CF684D693843354320F0040045EA30
:10A610000C0619E725F480454E6945EA861571E771
:10A6200026F4406C20F080008E69CF684D6940EAC6
:10A630000710354320F040004CEA850632E726F447
:10A64000405C20F400608E69CF684D6940EA0720C5
:10A65000354320F480604CEA051680E7FF8FFFFE4B
:10A66000000001408CFFFEFFFF8CFFFE8FFFFEFF0E
:10A6700003680B4A23F04003904203600DD0094B5E
:10A6800098420AD01022036823F038031343036072
:10A69000036843F04003036070470822F3E700BFFC
:10A6A00000380040003C00402DE9F8436D4D002388
:10A6B0004FF4F072202107466B4C05F6644085F894
:10A6C000603C55F021FF05F644604FF4F072202104
:10A6D00055F01AFF14F8D30C10B114F8D22C1AB993
:10A6E00000263046BDE8F8833FF024FC804644F85D
:10A6F000C40C3FF061FD06460028F1D0B8F1000F10
:10A7000002D02323A8F806300D2140463FF0F8FB85
:10A7100054F8C40C3FF064FD14F8D20CDFF85081FB
:10A72000013840B240F0BEFD0223202144F8CC0C99
:10A7300004F8D03C4CF0EAFAB8F80A134B4840F061
:10A740001DFD54F8C40C3FF045FDFF218C204FF057
:10A7500097F9814654F8C40C3FF042FD54F8CC0CF4
:10A76000FFF786FFB9F11B0F05D054F8C40C002683
:10A77000FEF728FEB5E7012254F8C43C85F8602CAA
:10A780000BB12322DA80B8F80A13384840F0F6FCFF
:10A7900054F8C40C3FF01EFD40210A204FF070F920
:10A7A000FF218A204FF06CF9034654F8C40CC3F320
:10A7B000801304F8C03C3FF013FD54F8CC0CFFF7B5
:10A7C00057FF14F8D43C012B43D0022B39D0E3B30C
:10A7D00014F8BF3C182B09D114F8C02CB8F80A3370
:10A7E00024F8BC7C24F8BA2C24F8B83CB8F80A1336
:10A7F0001E4840F0C3FCB8F80A131C4840F0BEFCE9
:10A8000054F8C40C3FF0E6FC022100204FF038F968
:10A8100054F8C40C3FF0E4FC54F8CC0CFFF728FFCC
:10A8200014F8AF2C14F8AE3CC2F1200214F8B01C9E
:10A83000C3F1100304F8AD2C04F8AC3C04F8B41CCC
:10A840004FE71023A8F80A33C2E72023A8F80A33F9
:10A85000BEE7002FF5D014F8C03C002B14BF102326
:10A860002023EFE7E82A0120E03B0120103B0120F4
:10A8700000000120F8B5474E16F8AB4C04EB44033A
:10A88000650006EBC30313F8A83C032B77D8DFE879
:10A8900003F0492A1F02254406EBC50555F8A43CE0
:10A8A000002B6ED116F8482C944268D0013404F085
:10A8B00003018A4206F8AB1C61D001EB410402227D
:10A8C000184606EBC40444F8A43C04F8A82CF8BDD0
:10A8D0002B1906EBC30353F8A42C72B1013A0020E4
:10A8E00043F8A42CF8BD2B1906EBC30353F8A42C92
:10A8F000002AF3D1022203F8A82C254406EBC50553
:10A9000015F89C3C013BDBB205F89C3CF3B1224BB3
:10A910000120D3F80C2302F2E733B3FBF2F345F83E
:10A92000A43CF8BD40F06CFD48B31B4A42F20F73E3
:10A930002C440121D2F80C2306EBC404134404F880
:10A94000A81CB3FBF2F344F8A43CF8BD124B601C06
:10A95000032755F8A01CD3F80C23384016F8484CB0
:10A96000531E05F8A87C001B0B4418BF01209A4217
:10A97000B3FBF2F188BF002045F8A41C30B90120D8
:10A98000F8BD013B002045F8A43CF8BD013945F86D
:10A99000A41CF8BDE03B01200000012003689B0AD5
:10A9A000A3F58013522B00D970470E4A134470B59B
:10A9B00093F8604284B00D2C12D800294FF00003A8
:10A9C00009494FF0010514BF1E460226427901EBEA
:10A9D00084106946CDE90065CDE902330AF030F80C
:10A9E00004B070BD780706089C3B01200378012B5A
:10A9F00001D00020704790F90420084902EB420280
:10AA000001EB421292F8D113202901D01846704769
:10AA1000D2F890339869C0F3C0307047E03B012012
:10AA200030B5044683B00D4608480DF107022146B3
:10AA3000FEF73AFE9DF8072035EA020304D02A43C8
:10AA40002146024840F070FC03B030BDDC400120DC
:10AA500070B51B4C82B00E46154694F8FC34022BA0
:10AA60000FD0012B0AD113460091024694F801152C
:10AA700094F9000550F068FB02B070BD002002B0F0
:10AA800070BDD4F808351BB19A88196812048A6120
:10AA90000146D4F800054EF045FE2B463246002113
:10AAA000D4F800054EF0F8FBD4F808352BB11A683D
:10AAB00001209B88936102B070BD0120DCE700BFDC
:10AAC000E03B01202DE9F04F037883B00446022BD0
:10AAD00000F08C80012B04D00025284603B0BDE88F
:10AAE000F08F90F90400554E042886F84035D4BF05
:10AAF00000250125B0F1FF3F08BF45F00105002DFD
:10AB0000EAD100EB40024FEA400C06EB4212D2F8C9
:10AB10009073002FE0D092F8D1E3BEF1200FDBD18B
:10AB2000BF6917F40047D7D192F8D0E3BEF1010F07
:10AB3000D2D04FF04008DFF818E1DFF818B14FF03D
:10AB4000210A94F80590DBF8644A82F8D1A382F8D0
:10AB5000D28306F5A868C2F8D473A2F8BA33C2F853
:10AB6000BCE3B2F8BAE382F8D0331FFA8EF3DFF811
:10AB7000E8E0C2F8B483FF2BC2F8C4E359D8B2F8B6
:10AB8000BAE34FF000781FFA8EFE84442C480094FC
:10AB90004FEA490900EB4C100A4606EB4C144946B3
:10ABA00014301923A4F8B8E3FFF798FB002836D136
:10ABB000D4F890232349536894F8B8630B40224D8E
:10ABC000D4F8C41343EA0903A94243EA064343EA1B
:10ABD0000803536084F8D00303D01C4B994218BF7C
:10ABE000F227136801251F43176076E7C3681BB17E
:10ABF0009A8818681204826160684EF093FD012102
:10AC000060684EF08FFDE3683BB101251A689B88B0
:10AC10002846936103B0BDE8F08F01255DE7B6F8E3
:10AC200042350022013384F8D0239BB2A6F8423586
:10AC300053E74FF0FF0E4FF08078A6E7E03B01208E
:10AC40005C3F0120009C00FCD96C0108E16D01080B
:10AC50000000FFFFE82A0120256F010808480023B3
:10AC6000024611780632022904D00133062BF8D1AE
:10AC70000020704703EB430300EB4300704700BF25
:10AC800024410120F0B59E4C85B02422002104F21D
:10AC9000445055F039FC94F86965002E3AD1354698
:10ACA000D4F880355BB39B6A4BB39648984783686A
:10ACB0002BB303880021DFF874C2013B604666466F
:10ACC0009BB237780636032F1CD001310629F8D104
:10ACD000002201780630022900F0A6800132062AFF
:10ACE000F7D1D4F8A815052909D002FB01C201311A
:10ACF000C4F8A815022000219380107051802846C6
:10AD000005B0F0BD062303FB0141B1F84635013B18
:10AD10009BB2DDE704F5AE6394F86805C4F86C35C2
:10AD200008B90025BCE73FF005F90746C4F87C05E3
:10AD30003FF042FA05460028F3D0013E022370B2EC
:10AD400084F8703540F0AEFA0028EAD0C4F87405F3
:10AD50000FB12023FB800D2138463FF0D1F8D4F805
:10AD60006C350126D8683FF03BFAD4F86C352021C9
:10AD700058684BF0CBFF644BD4F86C2584F8A4657D
:10AD80000026C4F8A02593E80300009032208DF837
:10AD900004103BF061F8052302AA6946D4F86C055B
:10ADA0008DF80A608DF8096040F06AFA9DF80A2073
:10ADB0009DF8090012029DF80B10544B42EA004224
:10ADC0000A439A4200F0948032DCA3F5F1139A42D0
:10ADD0005FD043DD4E4B9A4253D002339A4263D147
:10ADE0004FF400724FF48073A4F88425A4F89035D2
:10ADF000B4F890250020B4F884354FF48071120225
:10AE000084F89205A4F8861502FB03F3C4F888259C
:10AE1000B3F1807FC4F88C3559D801223D4B84F8BA
:10AE20009925C4F880353BE7062101FB02C261E7A2
:10AE3000394B9A4235DC053B9A4235DD374B13449A
:10AE4000032B4DD801A252F823F000BF93AE0008A7
:10AE500083AE000875AE0008E1AD0008A3F522033B
:10AE6000013B9A423CD02EDD2D4B9A4209D0013352
:10AE70009A4219D14FF48073A4F88435A4F8903520
:10AE8000B6E780224FF48073A4F88425A4F89035A7
:10AE9000AEE740224FF48073A4F88425A4F89035DF
:10AEA000A6E7204B9A42E5D0002394F868051D469A
:10AEB000A4F88435A4F89035C4F88835C4F88C35E6
:10AEC00040F03AF9ECE6184B9A42D3D0ECE7012374
:10AED000B721D4F8A00584F898354EF013FD9CE70F
:10AEE00020224FF48073A4F88425A4F890357FE7DE
:10AEF0004FF480621023A4F88425A4F8903577E7F6
:10AF0000E03B0120604101202C0A06081640E000C9
:10AF10001720C200340A06081940EF00EABF10FFEC
:10AF200017BA20001870EF001860010024410120BA
:10AF30002DE9F04F4021BA4C0027042341F23C0593
:10AF400004F694564FF0A042616194F8BD030221CB
:10AF50008BB06360C4F8006464512260276327618A
:10AF6000E7626762A161E160C4E90777002800F049
:10AF70005F810321164684F8BD13936823F0010313
:10AF80009360F368304643F04003F36009F088FBB8
:10AF9000B36B012F054643F48033B36317D005B379
:10AFA000022384F8BD339F4B13F8B45C012D00F0ED
:10AFB000FB8023688021012059625A6A42F4800292
:10AFC0009A62FDF7ADFB00200BB0BDE8F08FB368CF
:10AFD00043F00603B360B36843F02003B360002D71
:10AFE000DED123683220DA6822F0C042DA60DA6803
:10AFF00042F08042DA6009F0C9F8606848B32A4636
:10B0000001272946C2EBC203561C04EB830383F8D5
:10B010003C20A3F84220F2B283F83D70824283F8CC
:10B020003F101965C3E91111ECD300221146C2EBA0
:10B03000C203561C04EB830383F8FC21F2B283F8AD
:10B04000FD11824283F8FF11C3F81012C3E9811188
:10B05000EDD300222368D4F80CC01646D4F8108033
:10B06000D4F82CE0D4E90671019102F140010132DB
:10B0700003EB81010F2A4E60F7D19A6BBEF1000FEE
:10B0800040F0408122F400129A631A6842F04002B4
:10B090001A601A6842F080021A600022012F03F53C
:10B0A0000066C3F8002ED3F80028C3F80028D3F8B0
:10B0B000002800F01E81032F00F01B8142F00302E4
:10B0C000C3F800284FF48461574A196102E0013A3D
:10B0D00000F02F8119698F06F9D41021524A1961A5
:10B0E00002E0013A00F023811969C906F9D4002170
:10B0F00031617161F161E0B103F510624FF0904A86
:10B100004FF0006B0F464FF67F399C4607E0176003
:10B1100001311761C2F808902032814261D0136872
:10B12000002BF4DA11B1C2F800A0F1E7C2F800B0C8
:10B13000EEE73269B8F1010F22F48072326100F05B
:10B14000EA8000216FF0804299615A61B8F1000FE6
:10B1500003D19A6942F010029A619969334A0A430D
:10B160009A61019A1AB19A6942F008029A61BEF195
:10B17000010F00F0CB80002D7FF412AF0121626A35
:10B1800084F838508A4284F8BD1300F0D480736884
:10B19000032043F00203736008F0F8FF214B13F81B
:10B1A000B45C012D7FF405AF03204DF057FD03285B
:10B1B0003FF4FFAE23688022284640215A625A6A33
:10B1C00042F400129A62FDF7ABFA20210220FDF74B
:10B1D000A7FA40210320FDF7A3FA00200BB0BDE839
:10B1E000F08F002163460CF530624FF0904A4FF02B
:10B1F000006B0F464FF67F39844607E01760013138
:10B200001761C2F808902032614592D0106800287A
:10B21000F4DA11B1C2F800A0F1E7C2F800B0EEE72D
:10B22000F0190120E82A0120400D030000383C807D
:10B2300000F0FF054B4B03204FF4C05684F8BC537D
:10B240001A6B42F001021A630A221B6B069105A9D0
:10B2500003F00103089044480493049B0795059666
:10B26000099208F0C9FCE36A012B71D03D4B06211D
:10B2700043205A6B42F080025A635A6B02F08002FC
:10B280000292029A5A6C42F480425A645B6C03F454
:10B2900080430393039BFDF7A1FF032326683349F3
:10B2A0000820A269886084F8BD33012AB368276941
:10B2B00023F00103B3607FF464AEB26B2C4B22F435
:10B2C0008032616BB2630129F26803EA0203F36022
:10B2D000F36823F44013F36003D1F36843F480135D
:10B2E000F360304609F0DCF9012F05467FF457AED4
:10B2F0006DE6BCF1000F3FF4E3AE42F00102C3F88B
:10B300000028DFE642F400129A63C6E69969194AFA
:10B310000A439A612FE718490020184A31636FF0F9
:10B320008041376B3A4332639861596115E70125D3
:10B33000DDE60125D1E684F8F4539969C4F8FC23CD
:10B3400041F000610E4A9961596D0A435A651EE742
:10B350004FF4007305A904480593CDE9065508F09C
:10B360004BFC83E7003802400000024000E100E0AF
:10B37000BFFFBDFF0400004000018000030001008A
:10B380000300001010B5194C94F8AE0590B9184B95
:10B3900083F85505C3F8580594F8B135012B1FD033
:10B3A000D4F8B43503B313495B68A1F10C00BDE8D0
:10B3B000104018473EF0BEFD94F8B0250C49003A05
:10B3C000C1F8580518BF012281F855250028E3D09F
:10B3D0001F22C280FDF7F6FF94F8B135012BDFD1B3
:10B3E000054BC4F8B435DEE710BD00BFE03B0120DB
:10B3F000F0190120984101201003012099B10A6B36
:10B40000824216D9154BD3F8FC25914221D34C39F1
:10B4100091421ED30B6B9842F9D38B6B9842F6D8AE
:10B420000B46184670470D4BD3F8FC150A6B90423B
:10B4300012D30B680BB9F4E70A6B90420B4602D3A8
:10B440008A6B9042EDD951F84C3F002BF4D118464D
:10B4500070470023184670470A46D8E7E03B0120B2
:10B460002DE9F047CC0143D1034622494FF0FF328A
:10B47000022443F8081B7E2642601846DFF87880D5
:10B480002644051D6FF07047D8F800964FF0010A6A
:10B49000013E494608E0A3421CD0631C45F8043C29
:10B4A000321B1C460435CAB10B6BA34202D88B6B0E
:10B4B000A34204D22046FFF7A1FF014690B10A79CA
:10B4C0004B6B002AE7D1A34204D0E6D2631C45F8B7
:10B4D000042CE5E7631C45F8047CE1E7C8F8001696
:10B4E000BDE8F087321B631C494645F804ACD8E739
:10B4F0008026C3E7F8FFFF0FE03B0120F0B50023F3
:10B500000E680DE0BCF1050F17D9BEF1050F18D874
:10B510000A2C16D103EB830316F8010B04EB43034B
:10B52000A0F13005A0F1610CA0F1410EA0F13704AB
:10B53000EFB2092FE6D82C46ECE7A0F157040A2C0D
:10B54000E8D00E601360F0BD036870B55E6A26B186
:10B5500033460522BDE87040184704460D464E1D8F
:10B5600000E023689B68204698470028F9D02368AC
:10B57000204615F8011B1B689847B542F1D170BDF4
:10B580002DE9F0470023194D84B0074695F90D9633
:10B5900005F214664FF0B60A00EB010805F6B40593
:10B5A0001C46D6F800C0304600226946E036BCF1A1
:10B5B000000F14D09CF838C0BCF1140F0FD019F153
:10B5C000020F01D0CC450AD1CDE90244CDE9007883
:10B5D000ADF808A08DF80E4031F0CEFF0346B5421D
:10B5E000DFD1184604B0BDE8F08700BFE03B012082
:10B5F0002DE9F743A0230124114E18255FFA84F8A2
:10B60000FF2B14DCE9B2D6F8B4085F1CDBB2C1F141
:10B610001C02C1F11B0180F80B808272C9B2026862
:10B6200000930023D2F818904246C8473B46013D9C
:10B63000E6D10134052CE0D103B0BDE8F08300BFB2
:10B64000E03B012010B50A4C94F8D108003818BF2F
:10B650000120FFF729F850B1064904F6B8003FF081
:10B66000FBFC04F6B80012F049F904F6B80010BD6E
:10B67000E03B0120600A06082DE9F04F914C164688
:10B680000B2287B094F85A8B054694F865AB89462F
:10B690004046114602951D469DF8407039F0C6FFA0
:10B6A000C245834640F0BC80039040463EF042FCD9
:10B6B00017F008030246019300F0A580BBF1000FCC
:10B6C00000F09D809BF80710890700F19880C4F86E
:10B6D00024B9C4F82009C4F81C09002800F0EE8041
:10B6E00040F60B3105F0020AC1804FF48073DFF899
:10B6F000F4810299584608EB030284F8E4580025C7
:10B70000C4F80C19C4F8F82831466F4AC4F8EC386C
:10B71000C4F8E028C4F8F038C4F8E86884F8E5789C
:10B72000C4F81099C4F8F488C4F80059C4F8FC5857
:10B73000C4F80859C4F80459C4F83C5B84F8405B69
:10B74000A4F8345B31F04EF9D4F8240907F0010174
:10B75000FFF724F95D4A5E4BD4F82409C4F8485B2E
:10B76000C4F84C2BC4F8443BBAF1000F1CD0D4F8F9
:10B770002C79CFB13A6803689A4215D0012331463B
:10B78000384684F8413B31F02DF908F50572294619
:10B79000D4F82C094BF02AFF2A4608F50771D4F893
:10B7A00024094BF023FF07E04A4A002302F1080175
:10B7B00084F8413B4BF01AFFD4F824391B689B0AEC
:10B7C000A3F58013522B32D8434A134493F86022D6
:10B7D0000D2A2CD8414B03EB8213C4F82839019B66
:10B7E0005BB33F4831F020F93D4807B0BDE8F08F2A
:10B7F000039BCDE9040113B1D879830725D5002037
:10B8000007B0BDE8F08F15F00101F1D105F0020C91
:10B810005FFA8CFABAF1000F32D1D4F824B964E798
:10B820000B220C21504639F001FF03903DE7002325
:10B83000C4F82839019B002BD3D1294831F0EAF80C
:10B840000121274831F016F9CBE7504605F0020AEE
:10B850003EF070FB039AD4460599C4F82429049A53
:10B86000C4F81C09904202D1BAF1000F1CD1002883
:10B87000CED040F60C3EA0F806E0BAF1000FCCD0D6
:10B88000B8F1000FBBD0C4F8202991B9BBF1000F6B
:10B89000B5D0C4F824B95FFA8CFA002A3FF425AF7A
:10B8A00040F60B31D18020E7B8F1000FA7D0C4F8E3
:10B8B0002029C4F82CB9D4F824B9ECE705F0020A21
:10B8C00013E700BFE03B0120B00A060859C3030894
:10B8D0008DCA030824470120780706089C3B0120F5
:10B8E000C044012010450120094B13F8AE3C042B45
:10B8F00008D9053B032B08D801231A4600B1037071
:10B900001046704700230122F8E700231A46F5E7A6
:10B91000E82A01202DE9F0479AB004460D46174663
:10B920009846DDF89090DDE9226A02E020683BF05D
:10B930005DFB20683BF062FB0028F7D101466422E2
:10B9400001A854F0E1FD264B8DF80450CDF85CA021
:10B950000293002D40D0AB1E012B3FD9042D14BF04
:10B96000002303231F4A8DF80530012352F8B82C19
:10B97000039616448DF85B30CDE90594049637B1F3
:10B980004246394607A854F04DFD8DF85A80164EB0
:10B99000002396F8B69B1893B9F1000F19D196F8C9
:10B9A000B50B642201A902FB006000F6B83054F028
:10B9B00039FD012386F8B59B86F8B63B236843B171
:10B9C00043463A46294620461AB0BDE8F04715F0EE
:10B9D0005FB91AB0BDE8F0870523C3E70223C1E7CA
:10B9E00054470120E82A0120E03B01209FED747AB2
:10B9F00007EE901A20EE070AF8EE677A27EE800A23
:10BA0000FDEEC07A17EE903A2033402B00F2C8804A
:10BA1000DFED6C7AB4EEE70AF0EE407AF1EE10FA60
:10BA20000CDD9FED696ADFED696AB0EE677A77EE4B
:10BA3000C67AB4EEE67AF1EE10FAF6DC9FED647A9F
:10BA4000F4EEC77AF1EE10FA0CD59FED5F6ADFEDE8
:10BA5000616AB0EE677A77EE867AB4EEE67AF1EE56
:10BA600010FAF6D49FED5C7AF4EEC77AF1EE10FA94
:10BA700040F386809FED537A77EE677A67EEA75A98
:10BA80009FED565A9FED566AB6EE007ADFED556A85
:10BA9000A5EE856A27EEA55AE5EE866AE5EE267ADA
:10BAA00027EE877ADFED4C6A70EE267ABDEEE76A04
:10BAB00016EE103A2033402B6FD8B4EEE60AF1EEC2
:10BAC00010FA0CDDDFED405A9FED406AF0EE676A38
:10BAD00077EEE57AF4EEC66AF1EE10FAF6DCDFED09
:10BAE0003C6AF4EEE67AF1EE10FA0CD5DFED365A48
:10BAF0009FED386AF0EE676A77EEA57AF4EEC66AD3
:10BB0000F1EE10FAF6D4DFED346AF4EEE67AF1EEF7
:10BB100010FA48DDDFED2B6A76EEE77A67EEA75A7A
:10BB2000DFED2E4A9FED2E6AB8EE005ADFED2D6A4A
:10BB3000A5EEA46A67EEA54AE5EE866AE4EEA67A6B
:10BB400067EE857AC7EE206A002383614361036252
:10BB5000B7EE006AC36176EE865A76EE666A86EEC6
:10BB6000257A67EE277A80ED007A66EE876A80EDA7
:10BB7000027AC0ED017AC0ED037AC0ED046A704725
:10BB80009FED197AF4EEC77AF1EE10FA7FF576AFF1
:10BB90009FED0F7A77EE677A70E7DFED147AD1E7E1
:10BBA0009FED127A7EE7DFED106AF4EEE67AF1EEB1
:10BBB00010FAB3D5DFED066A76EEE77AAEE700BF9E
:10BBC00027D4D236DB0F4940DB0FC940E4CB164106
:10BBD000DB0F49C0E4CB16C1DB0FC93F92E741B987
:10BBE0009730083C15A82ABEDB0FC9BF0000000033
:10BBF00030B40023314D32494CF25034C5F8383C52
:10BC0000304AD1F8640A04E0D1F8643A1B1AA3421E
:10BC10000FD8D368DB03F7D4D16811F4F9710BD1D5
:10BC2000D06810F0010002D001230846D36030BC78
:10BC30007047032030BC7047D3689B0705D5D5F803
:10BC4000383C43F02003C5F8383C1E4BDB68DC066B
:10BC500005D5D5F8383C43F01003C5F8383C194BEE
:10BC6000DB68980605D5D5F8383C43F00803C5F8DD
:10BC7000383C144BDB68590605D5D5F8383C43F001
:10BC80000403C5F8383C0F4BDB681A0605D5D5F818
:10BC9000383C43F00203C5F8383C0A4BDB68DB054F
:10BCA00005D5D5F8383C43F04003C5F8383C054B82
:10BCB0004FF4F9720120DA6030BC7047E03B01209C
:10BCC000E82A0120003C02400C480D4BD0F8541CDF
:10BCD00010B48A1E0B4C2231C0F8443CB0F86E3CC4
:10BCE0001B01A4FB03C3DB08A3F5B06322F8023FEA
:10BCF0009142F3D15DF8044B704700BFE03B012057
:10BD0000DD970208CDCCCCCC70B5084C251D2E4655
:10BD100014F8010B31F002FE28B10378B44205F8A3
:10BD2000013BF5D170BDFF23F8E700BF704801204B
:10BD30002DE9F0471C4F01264FF03C094FF0000859
:10BD400007F10805B24617F8010B3EF0F3F8044678
:10BD500090B180F80690C671FB7803F07F02012A4B
:10BD600017D013F0800F20460CD185F804803EF0E8
:10BD700031FA85F805802C6001360835052EE2D1B0
:10BD8000BDE8F08785F804A03EF02AFA85F805A002
:10BD9000F1E71B0604D42046FDF70EFBFB78E0E735
:10BDA0003EF01EFAF7E700BF784801202DE9F04F7A
:10BDB000DFF81C8185B0DFF81CA1012608F10C0713
:10BDC000DFF81491AAF1940B18F8013B002B64D012
:10BDD0001D0903F00F01013D032D6CD809EB45024D
:10BDE000908D40FA01F414F0010467D001224D4413
:10BDF00003938A40334C013A104050F047FF95F8C6
:10BE000034200421039B104404EBC0047C61E671E0
:10BE1000A171002102E0013115293ED001EB410062
:10BE20004A001BF800509D42F5D15044039210F88F
:10BE3000931C002944D0184639F068FB0546006879
:10BE40004BF076FD697939F09FFB03782BBB039AA1
:10BE50000421524402F8536C02F8541C04B32046E7
:10BE6000194C2A7A022103933DF08EFF2946039B49
:10BE7000B4F8C25C3846B4F8C04C144ACDE900436B
:10BE8000B2FBF5F301369BB230F07CFF0123F6B232
:10BE9000183707F8073C092E96D105B0BDE8F08F9A
:10BEA000094B2946094A3846B3F8C25CB3F8C03C8E
:10BEB000CDE90034E4E700247C61AAE77C61A8E7CF
:10BEC0000B68FFDEC02A0120E03B012040420F004A
:10BED000A4480120E82A0120780706088E4B2DE9A6
:10BEE000F04193F8902D82B00190002A40F00E812D
:10BEF00093F8B42DB7EE007AB3F8B87D012107EEC0
:10BF0000902AB3F8B60DF0EE475ADFED846AB8EE2A
:10BF1000E76A07FA01F507EE900AB3F8B20D804C14
:10BF2000E6EE665A8542A6EE267AA4F80871F8EE87
:10BF3000E77AB8BF054683F8901DAEB267EEA67AE1
:10BF4000A4F80C61C4ED3F5A84ED407AC4ED417A07
:10BF5000002A00F0D880DDED017AADB29FED710AC4
:10BF6000F8EE677A6D0080EE270A51F055FF8046A3
:10BF7000B0FBF5F5012DB8BF0125EDB2B0FBF5F32F
:10BF80009BB284F8105100EE103ABBEEED0A84ED3E
:10BF9000450A51F041FF644BDFED646AA3FB0838AA
:10BFA000DFED630A9FED636A00234FEAD8089FED37
:10BFB000621ADFED625A07EE908ADFED611A9FED9B
:10BFC000612AF8EEE77ADFED602A9FED603ADFED57
:10BFD000603A86EEA77A5F49B7FBF0F00228B8BF57
:10BFE000022084F8180184ED477A07EE903AB8EE03
:10BFF000E77AF0EE467AE7EE207AFDEEE76A16EE93
:10C00000902A2032402A7BD8B4EEC17AF1EE10FAA1
:10C010000CDDDFED516A9FED517AB0EE675A77EE95
:10C02000E67AB4EEC75AF1EE10FAF6DCF4EEE57AF1
:10C03000F1EE10FA0CD5DFED486A9FED497AB0EECB
:10C04000675A77EEA67AB4EEC75AF1EE10FAF6D434
:10C05000F4EEC67AF1EE10FA4ADD73EEE77A67EE97
:10C06000A76AB0EE424AB7EE007A67EEE64AA6EE5D
:10C07000A14A77EE677AB0EE627AB6EE005AA6EE83
:10C08000847AE4EE877A67EE857A0133E1EC017A0F
:10C09000202BAAD107EE905AB7EE006A314A102041
:10C0A000F8EEE76A07EE906A2F4B02F12806F8EEE9
:10C0B000677A202186EE267A84F82156C4F8C427B0
:10C0C00002F1A8051422C4F8C067C4F8D057C3ED24
:10C0D000AC7AC3EDAD7AC3EDAE7AA4F8BC07A4F890
:10C0E000CC17A4F8C82783ED007A02B0BDE8F08130
:10C0F000F4EEC37AF1EE10FA48BF75EEE77AAEE7D8
:10C10000F6EE007AC1E7194B1A7024E7044C94F854
:10C110001051B4F80C61BDE7E03B01200AD7233C85
:10C120001400002000247449ABAAAAAADB0FC9415D
:10C130003C8C4F3EDB0FC93F0100F840DB0F49C08C
:10C1400092E741B99730083C15A82ABEDB0FC9BF5A
:10C15000DB0F494034010020DB0FC940E4CB16411E
:10C16000E4CB16C1E00A06083806002000000020D3
:10C170002DE9F843204D0023204E4FF0050895F897
:10C18000BF7D05F6BC5506F66C2486F8687A15F86E
:10C19000010B03F1010908BB20604B460434032B5B
:10C1A000F5D1F943D6F86C0A01F001013EF01EF812
:10C1B00096F8681AD6F8700A81F00201C1F34001BE
:10C1C0003EF014F896F8681AD6F8740A81F0040163
:10C1D000BDE8F843C1F380013EF008B83DF0AAFE87
:10C1E00020605FFA89F310B180F80680C37120687F
:10C1F000FDF7E2F8D1E700BFE03B0120E82A01208B
:10C200002DE9F0412A4C82B02A4DB4F8C46DA5F84E
:10C21000786AEEB994F8C00D3DF08CFE94F8C12D0B
:10C22000C5F87C0A003A18BF012285F87A2A48B17D
:10C2300094F8C21D2B220029C28014BF11210121B4
:10C240003DF05EFE002002B0BDE8F0413EF064BD6E
:10C2500094F8C08D00222B21404639F0E7F90746BB
:10C2600040463DF067FE00B117B902B0BDE8F0816D
:10C270002B22C5F8940A4FF00008C280397AFEF7E5
:10C2800063F80D4ACDF804803946A4F8C66D05F56B
:10C290002860B2FBF6F3C3F34F049BB2009430F076
:10C2A00071FDD5F8803AC3F8008085F8918ADCE703
:10C2B000E03B0120E82A012040420F002DE9F84F21
:10C2C000254B002693F8D42D03F6CB5703F6E854FC
:10C2D00083F8C82D5FFA86FB4FF0010917F8010FAC
:10C2E00001360BEB090A49464FF000085FFA8AFA5B
:10C2F000524639F09BF9054640B3387804F80E8C65
:10C3000004F80D8C04F80FBC04F8109C44F8045C8D
:10C310003DF010FE18B180F8069080F807A0297A49
:10C32000FEF712F80D4A002128464BF08FFA0C4B0D
:10C33000221D2146236028460A4BC4E901384BF0F0
:10C3400055F942466979286830F078FC082E04F1E6
:10C350001C04BFD1BDE8F88FE03B012040420F0034
:10C360000DCD0308BDBA030870B52C4C00222C4B30
:10C37000022194F8000FC4F8F83EC4F8B82EC4F8AF
:10C38000BC2EC4F8C02EC4F8F42EA4F8FC2E39F04C
:10C390004DF9002840D0234B0546026803F1C00048
:10C3A000597C11B159688A422BD018338342F7D196
:10C3B000002394F8000FC4F8E45D84F8D83D3DF004
:10C3C000B9FD08B10223C380297A0026FDF7BCFF1E
:10C3D0002846154A00214BF039FA144A1448154BE7
:10C3E000111FC4F8E80D2846C4F8EC3DC4F8F06D00
:10C3F0004BF0FCF8324669792868BDE8704030F0AF
:10C400001DBC926A0C4801320C49D0F8D831B3FBFC
:10C41000F2F381F83433CBE770BD00BFE03B01207D
:10C4200000FFFF004800002040420F00CC490120DF
:10C43000E5BA030881BC0308E82A012000000120B6
:10C440002DE9F04FC34D85B00E46C34F0446C022C0
:10C4500005F134000021019654F056F897F8013F99
:10C46000002B70D097F8023F002B00F08B80DFF894
:10C47000089319F8A03C012B00F0AE80022B00F0CD
:10C480008E80B64BB64E1C46029319F8AA7C0FCE8E
:10C490000FC40FCE0FC4391EB24A19F8AE3C18BFF4
:10C4A0000121C5F83C29072B85F85C1996E807009F
:10C4B00084E8070000F21381042B00F21D81DFF8ED
:10C4C000D0820026DFF8B8B2019B5FFA86FA03211A
:10C4D000B3420AF101072BDD1BF8014BFFB22046E6
:10C4E0003A4639F0A3F8034620461C4613B33DF004
:10C4F00021FDC8F8140018B14FF00303C771837110
:10C5000019F8AD3C19F8AE2C002B00F0F380E3795C
:10C5100083F001035146204601364BF021FE48B11D
:10C520004FF00103082E08F1180808F8073CCBD19A
:10C53000029B06E08C4900238C4AC5F84019C5F8D7
:10C540004829C5F85839D5F8583963B10022012176
:10C55000019883F82D1083F82C001A6383F82E209D
:10C5600005B0BDE8F08F824E824C0FCE0FC40FCEC7
:10C570000FC496E80700A4F1200384E80700C5F87B
:10C580005839EDE77C4B2046019913F8AC2C003A62
:10C5900018BF0122FCF784FCC5F85809D3E719F845
:10C5A000AA3C002B3FF46DAF19F8AE3C082B13D119
:10C5B00005F624136A4E6B4F1C460293012385F83F
:10C5C0005C390FCE0FC40FCE0FC496E80700C5F834
:10C5D0003C7984E8070085E0019B0026DFF8B4C1C0
:10C5E000664CB046C5F8603987F8046FBCE80F00A8
:10C5F0000FC4BCE80F000FC419F8AA2CA4F6DC0A7B
:10C6000019F8AE1C04F15C0B921B5D4B87F83C1FC4
:10C6100018BF01220293CDF80CA085F85C299CE894
:10C62000070084E8070040E0E27982F0010A0AF09E
:10C63000010495F85C19013487F8034F09B18AF0B9
:10C64000010A30463DF0B8FD002865D0002E70D0BC
:10C65000B088610108F101084FF00303B0FA80F0DF
:10C6600041F00D01CBF80C60C0F11F008BF810A059
:10C67000CBF81410CBF8040086F80780B37130466D
:10C680003DF03EFC1AF0010F304625D03DF0A2FDF2
:10C69000039BB8F1080FDBF80C200BF1200B03F122
:10C6A000180343F8042C039320D0D5F860294245A1
:10C6B0001CDD029B13F8016B3046029338F0E8FF53
:10C6C000044630463DF036FC19F8AD2C0646002AEB
:10C6D000AAD194F807A0AAE73DF082FDD8E7082B7D
:10C6E0007FF4EDAE274BC5F86439E8E62348C5F87A
:10C6F000580928E7E3790DE719F8AB3C224A012BEA
:10C70000C5F8642905D09A1E53425341002F18BF23
:10C71000002385F86839D2E61C4B01221249C5F87E
:10C720000839124BC5F80C1987F8042FC5F81439CD
:10C73000DDE761014FF0FF3308F10108CBF80C6031
:10C7400041F00D01CBF804308BF810A0CBF8141099
:10C7500095E700BF14000020E03B012038090020CD
:10C76000340C06084D5A05084D38040845380408AD
:10C77000080C0608E84A0120E82A012004090020E4
:10C780003F2A012081330000B533000051380408EE
:10C7900048000020600C0608F8B5704F97F8680C48
:10C7A0003DF0C8FB97F8695C58B12D230446C3805F
:10C7B000FCF708FE0A2039F033FA20463EF0E0FA92
:10C7C00018B9D7F8403FDA0000D5F8BD013D092D72
:10C7D000FBD897F8674CD4B9402032F091FD00287F
:10C7E000F3D090F9043097F83D1C092BC8BF143BD7
:10C7F0000A293B4493F8504B00F0A28093F85B3B2E
:10C8000097F8662C002A08BF1C46002CDDD0204675
:10C810003DF090FB0546002800F08B802D23C3805F
:10C82000FCF7CAFD012108463DF0E8FC2B68AA8808
:10C830009A613C2039F010FB002101203DF0DEFC24
:10C8400097F8693C002B38D00026454C94F8681ABC
:10C85000D4F86C0AC94301F001013DF0C7FC94F81B
:10C86000681AD4F8740A81F00401C1F380013DF024
:10C87000BDFC7820002D38D0AB8801362A681B0417
:10C88000936139F0CDF994F8681AD4F86C0A01F084
:10C8900001013DF0ABFC94F8681AD4F8740AC1F3B6
:10C8A00080013DF0A3FC2B68AA8878209A6139F0BA
:10C8B000B7F997F8693C9E42C8DB97F8673C83BBA1
:10C8C00097F8683C002B80D197F86A3C012B7FF4E5
:10C8D0007CAFD7F8403F13F080537FF476AF87F8F2
:10C8E000693CBDE8F84042F025BE7820013639F0B9
:10C8F00097F994F8681AD4F86C0A01F001013DF038
:10C9000075FC94F8681AD4F8740AC1F380013DF0FC
:10C910006DFC782039F084F997F8693C9E4295DBEC
:10C92000CBE7322039F098FA284600213DF0E8FAAA
:10C93000C6E7FCF741FD012108463DF05FFC78E7C2
:10C94000D7F8443F5B057FF540AF12F043FA00286B
:10C950007FF43BAF002C7FF45AAF36E7E03B012079
:10C96000E82A0120094BD3F8480FD3F84C2FD3F80D
:10C97000503F904202DC114602460846984204DDD0
:10C980009A42B8BF1A46104670477047E03B0120F4
:10C990000B6810B414681B1B036054684B681B1BA6
:10C9A0005DF8044B43608B6892689B1A8360704704
:10C9B0002DE9F047041E0D4612DB092C26DC0B4640
:10C9C000814A82480021A0FB04605970C00800EB36
:10C9D0008000A4EB4000125C28461A70BDE8F08786
:10C9E00064422D23092C01F8013B24D8764A774B69
:10C9F0000020A3FB046348702846DB0803EB830395
:10CA0000A4EB4303D35C0B70BDE8F0876F4B632C42
:10CA1000A3FB04264FEAD60621DC0B466A4A6B4983
:10CA2000A1FB0601C90801EB8101A6EB4101515CA4
:10CA300003F8011BC5E7654A632CA2FB04364FEAE5
:10CA4000D60637D8604A614BA3FB0603DB0803EB2D
:10CA50008303A6EB4303D35C01F8013BC7E7A3FBC9
:10CA60000627B4F57A7F4FEAD7070DD20B46564A10
:10CA70005649A1FB0701C90801EB8101A7EB410160
:10CA8000515C03F8011BCAE7A3FB072842F20F72AF
:10CA900094424FEAD80836D80B464B4A4B49A1FB83
:10CAA0000801C90801EB8101A8EB4101515C03F8C1
:10CAB000011BDDE7A2FB0637B4F57A7F4FEAD70703
:10CAC0000CD2414A414BA3FB0703DB0803EB830372
:10CAD000A7EB4303D35C01F8013BB4E7A2FB0739A2
:10CAE00042F20F739C424FEAD90921D8364A374B9C
:10CAF000A3FB0903DB0803EB8303A9EB4303D35C2C
:10CB000001F8013BDEE7A3FB0829314A94424FEAD2
:10CB1000D90921D80B462C4A2C49A1FB0901C90887
:10CB200001EB8101A9EB4101515C03F8011BB5E761
:10CB3000A2FB093A264B9C424FEADA0A21D8224A44
:10CB4000224BA3FB0A03DB0803EB8303AAEB43039B
:10CB5000D35C01F8013BCAE7A3FB09231D4A9442B9
:10CB60004FEAD30A21D80B461849174AA1FB0A01FC
:10CB7000C90801EB8101AAEB4101515C03F8011BDB
:10CB8000CAE7A2FB0A38134B9C424FEAD80813D8D5
:10CB90000E4B0D4AA3FB0803DB0803EB8303A8EB52
:10CBA0004303D35C01F8013BCAE70A22BAFBF2F067
:10CBB00046F04EFC0346D7E70A22B8FBF2F046F0F7
:10CBC00047FC0146E4E700BF8C960608CDCCCCCCF0
:10CBD0009F8601003F420F00344870B490F8543FE4
:10CBE000A3F13001092958D800F6547400F6637097
:10CBF000224612F8015FA5F13001092904D88242CA
:10CC0000F7D1002070BC7047141B022C4BDD284864
:10CC1000002101E010F8013B01EB8101161A0446E6
:10CC200003EB4103022EA3F1300303F0FF01F1DC1B
:10CC3000204B03FB01F1A2424FF000030ED903EB9E
:10CC4000830314F8016B5B00A242A3F13003334469
:10CC500003F0FF03F3D1184800FB03F32E2D06D099
:10CC60001648A0FB032370BC01EB93007047013210
:10CC70000425002404EB84041078013D303864005E
:10CC80000928A4B2204401D8013284B215F0FF056E
:10CC9000F0D1642202FB0433E2E700211D4600F6D6
:10CCA00054720B46DAE70021054CC4E7E03B012053
:10CCB000354B01208096980040420F00ABAAAAAAEB
:10CCC000344B012038B50D460446FF2100682A4642
:10CCD00053F01AFC22682A44226038BD0C461646DE
:10CCE000054683B530F088FE204630F085FE0021F1
:10CCF000204B0846002E08BF1E463DF07FFA00215B
:10CD000001203DF07BFA28463AF078F9B0B10121D4
:10CD100000203DF073FA28463AF068F907462046AD
:10CD20003AF068F90028FAD0394620463AF06AF914
:10CD30003846B047002108463DF060FA20463AF0F8
:10CD40005DF90028DFD0012100203DF057FA204690
:10CD50003AF04CF90146284601913AF04BF9019915
:10CD60000028F8D028463AF04DF9002108463DF059
:10CD700045FAC8E739C20308F0B5002289B0DFF8E8
:10CD800098C004AF13460A604A603E468A60CA6093
:10CD90000A610268C2F3855040FA03F43546E4079D
:10CDA00004D513F80C4005F8014B2E460133062B31
:10CDB000F2D1174DC2F303240023C2F305302C44F3
:10CDC00005F2245C33700DF1190694F81C458DF8BA
:10CDD000184040FA03F43546E40704D513F80C4034
:10CDE00005F8014B2E460133062BF2D10023C2F386
:10CDF000834506AC0846337002F00F030549C2F3C1
:10CE000003120097CDE9014549F086FB09B0F0BD5A
:10CE100078070608B49606088C0C060870B5094C0D
:10CE20000546D4F8642F62B1002601362D21D4F8CE
:10CE3000640F3EF0B3FAAE42F7DBBDE870403FF05E
:10CE40005DBC70BDE03B012038B50546084643F0A7
:10CE500027FA041E0D4B0FDB93F86C2A944205DA77
:10CE600021460B4840F002FC204638BDFF2C03D180
:10CE7000084840F0FBFBF7E793F86C2A2846064980
:10CE80004FF0FF34013A3FF0E1FBEDE714000020E2
:10CE9000C3960608D4960608E7960608114A01309C
:10CEA000002302EBC000F0B4D0F830C50E4E336062
:10CEB0003361336233633364336533663367BCF1A4
:10CEC000000F0DD090F82C7557B13F0100240CEBEA
:10CED0000403351910340FCBA74285E80F00F6D1B3
:10CEE000F0BC704778070608484B0120024BFF2131
:10CEF000D3F860054CF016BCF0190120002310B5E2
:10CF0000104CC4F82435FFF7F1FFFD21D4F860057B
:10CF10004CF008FCFFF7EAFFFF2808D1FFF7E6FF17
:10CF2000FF2804D10423022084F8283510BD064AC6
:10CF30000923002052F8B82C84F82835C4F81825A5
:10CF400010BD00BFF0190120E82A01202DE9F843A7
:10CF50001C4C05468946904694F828651F46042EC9
:10CF600008D0082E02D00020BDE8F883FFF7C6FFE6
:10CF70000228F8D1D4F868053DF02CF994F81E3554
:10CF8000BBB96902112006F0CBFBC0B90E4A0523DC
:10CF90000120C4F8049552F8B82CC4F80855C4F818
:10CFA0001085C4F81475C4F8182584F82835BDE830
:10CFB000F8832946112006F0B3FB0028E6D006F0DE
:10CFC000DFFBD0E7F0190120E82A012070B51F4CE3
:10CFD00006460D4694F82835042B09D0082B25D198
:10CFE000D4F8203583422FD0FFF788FF02281DD1C7
:10CFF000D4F868053DF0EEF80021372006F090FBEC
:10D000002946172006F08CFBC0B994F81E357BB971
:10D010007102192006F084FB80B908230220C4F8AD
:10D020002455C4F8206584F8283570BD012070BDF2
:10D030003146192006F074FB0028EED006F0A0FB64
:10D0400006F0DAFB032070BD022070BDF01901204C
:10D050002DE9F043054691B00E4690461F464A4CD6
:10D0600094F8280504280ED0082808D1D4F82035D3
:10D07000AB4200F08480FFF741FF0228F0D001208E
:10D0800011B0BDE8F083D4F868053DF0A3F894F83A
:10D090001E35002B63D16902182006F041FB0028E1
:10D0A00067D194F82895FFF721FFB9F1080F0CBF5D
:10D0B000FC21FE21D4F860054CF034FB94F86C257B
:10D0C000002A4ED094F874250021D4F860354FF032
:10D0D000400E52064FF4806C4FF400700C330A92ED
:10D0E000D4F87025CDF80CE0CDF818C00990049163
:10D0F000106805910F91CDE90711CDE90B11CDE92C
:10D100000D11117ACDE9013606F056FFD4F87035CD
:10D1100001AA197A186806F009FFD4F870351B497E
:10D120001A7A1868895CD4F86025435843F00103E3
:10D130004350536843F0020353600122062300204A
:10D14000C4F80465C4F80855C4F81085C4F814750B
:10D1500084F80C2584F8283511B0BDE8F083294601
:10D160009AE74FF480733146D4F860054CF094F898
:10D17000E3E706F005FB06F03FFB032080E7FFF73F
:10D18000B5FEFC2196E700BFF0190120A40D0608AA
:10D1900070B5092405460E46FFF7A8FEFF2803D107
:10D1A000013CF9D1012070BDFE2801D0022070BDE4
:10D1B000064833462A460021D0F860054CF06CF84A
:10D1C000FFF794FEFFF792FE002070BDF0190120DA
:10D1D0002DE9F047CD4C86B094F85465002E00F050
:10D1E0008F8194F8282504F24458C94F531E082B08
:10D1F0005CD8DFE813F06D00970025015B00490063
:10D200000900D6005B00C20094F86C25002A40F0AB
:10D21000818194F80C554FF48073D4F80415D4F838
:10D22000600501EB05214CF037F894F80C3501331B
:10D23000DBB2022B84F80C3535D1D4F8600500E060
:10D24000C3688368DB07FBD400214CF06BFA002134
:10D25000D4F860054CF066FAFFF748FE00F01F00B6
:10D26000052800F0218206F0C7FAD4F81055002DE9
:10D2700000F0AB810022D4F81435D4F80815012051
:10D28000A84794F82825B1E74FF40071D4F80405B5
:10D29000FFF77EFF012800F07F81022800F08481E3
:10D2A000002800F0988194F82825531EDBB2022B49
:10D2B00000F21C81964BD4F8182553F8B83C9B1A01
:10D2C000C82B00F24E810026304606B0BDE8F0873C
:10D2D000D4F868053CF07EFF0021084606F020FAED
:10D2E000054606F04DFA012DDDD14FF00009D4F8C6
:10D2F000680584F81D953CF06DFF40F2AB110820E5
:10D3000006F00EFA052800F06381012800F0348150
:10D3100006F036FA94F81D35002B00F0C181022387
:10D3200084F82835D4F868053CF054FF94F81D358E
:10D3300000213720022B0CBF4FF080450D4606F030
:10D34000EFF92920294606F0EBF9054606F018FA10
:10D35000002DA8D194F81D35022B00F0618184F8CE
:10D360001E55D4F868053CF035FF0021092006F071
:10D37000D7F9B0B306F004FA95E70825FFF7B6FD34
:10D38000FF2800F0AA81013DF8D1D4F8183557F8EC
:10D39000B82CFA33934286D206F02EFA94F8282558
:10D3A00024E7FFF7A3FDFF284FF0080505D0013D56
:10D3B000EBD0FFF79BFDFF28F9D1D4F824350022EC
:10D3C000012B84F81C2540F28E81D4F82025013BE6
:10D3D00008210132C4F8243584F82815C4F8202522
:10D3E00072E710214046FFF7D3FE05460028C1D161
:10D3F00001217F20FBF7EAF901288146BAD12846AE
:10D400000221FBF7E3F9002800F02B810128B1D1BC
:10D4100016213A20FBF7DAF901308002C4F82C0516
:10D4200006F0AEF9D4F868053CF0D4FE00210A20DD
:10D4300006F076F9002840F00D81032384F82835A2
:10D44000102102A8FFF7A4FE00287FF42CAF9DF85E
:10D4500015309DF816201B019DF809009DF80A5013
:10D4600002F00F01DBB245EA0025DDF8110043EAC6
:10D4700012139DF8102000BA84F8401503F5FA63E2
:10D480009DF80B10C4F83805A4F83E3513099DF833
:10D49000080002F00F0284F83C35039BA4F83055D5
:10D4A000C4F8343584F83D2584F8320584F8331502
:10D4B00006F066F994F81E3573B9D4F868053CF0A7
:10D4C00089FE4FF40071102006F02AF9054606F097
:10D4D00057F9002D7FF460AFD4F86005FDF7C8F868
:10D4E00000230422C4F8243584F82825042A18BF10
:10D4F000082A0CBF01260026304606B0BDE8F0879A
:10D50000304684F8286506B0BDE8F087F0190120A0
:10D51000E82A0120D4F87025137C10681F2B73D9DA
:10D52000203B202241689A4011403FF4CCAE1021AC
:10D53000C26001FA03F3C360D4F860058368DD07B5
:10D5400003D5C3688368D907FBD4836813F4C05F2D
:10D55000FBD183681A06F8D4436823F002034360C2
:10D560006FE606F049F994F82865082E18BF042ED6
:10D570000CBF01260026A7E60423494602AAD4F8D8
:10D5800060054BF089FE9DF80B30AB2B7FF4C0AEED
:10D59000022384F81D35BBE6D4F8183557F8B82CAB
:10D5A00064339342BFF47FAE06F0EAF806F024F944
:10D5B000D4F810554DB10022D4F81435D4F808151C
:10D5C0001046A84794F8282510E694F828250DE67B
:10D5D00084F81D559CE6019006F0D2F804230198CA
:10D5E000D4F8105584F81C0584F82835002D3FF434
:10D5F0006BAED4F81435D4F80425D4F80815A84730
:10D6000094F82825531E51E6202201689A401140C3
:10D610003FF459AE1021826001FA03F383608BE777
:10D62000D4F868053CF0D6FD29463A2006F078F893
:10D6300029460546042302AAD4F860054BF02CFEC7
:10D6400045B906F09DF8029B1BBAC3F3807384F8BA
:10D650001E3586E606F094F806F0CEF894F82825F4
:10D66000C4E504212C20FBF7B1F8032105464E2028
:10D67000FBF7ACF882460C213620FBF7A7F80AF13D
:10D68000020A431C09FA05F503FA0AF3A3FB050194
:10D69000430A43EAC153C4F82C3506F071F8C1E6D9
:10D6A0001E4684F828350FE6174B0722D4F810657C
:10D6B00053F8B83C84F82825C4F81835002E3FF4F8
:10D6C00003AED4F814350120D4F80425D4F8081595
:10D6D000B04794F82825531EE8E506F051F80423D6
:10D6E00084F82835F0E508D0042384F8283506F0BE
:10D6F00047F894F82825531ED8E5FFF7FFFB0228CA
:10D700007FF4D1AD36E600BFE82A012038B50F4CD2
:10D71000034694F8EF1F04F6E87084F8EB3F01F03D
:10D720003F0101F10A058B1C083184F8EA5F2544AA
:10D7300084F8ED3F1FF02EFC85F8E60F94F8EA3FE1
:10D74000000A1C4484F8E70F38BD00BFE03B01200D
:10D7500038B51E4C096854F8E45C0068491B1C4D40
:10D76000DFED1C6A00EE901A54F8E81CD5EDCE7A75
:10D770001C46F8EEE00A401A60EEA70A07EE900A8F
:10D78000F8EEE77A20EEA07AB1EE670AA7EEA77A64
:10D79000F1EEC77A67EEA67AFCEEE77AC2ED007A80
:10D7A00048F09EFF9FED0C7ADFED0C7AE0EE077AF1
:10D7B000FDEEE77A17EE902A002A02DBC4ED007A2C
:10D7C00038BD48F6A0431344236038BDD84C01202F
:10D7D000000001202C7D8E3FA00CB34500A00C461C
:10D7E00038B50A4C002501228021204631F074FD15
:10D7F00030B194F9040031F0A3FD08B1006838BDE0
:10D8000001350C34072DEED10020F8E7084C01203B
:10D8100038B5041F00F1080554F8043FD81780EA12
:10D82000430019F001F8A542F6D138BD084B4FF678
:10D83000FF70002103F5276210B40024C3F81C0B0D
:10D84000C2F8A410C3F8184B5DF8044B704700BF32
:10D85000140000202DE9F041BB4CDFEDBC7AD4F878
:10D86000242B94F8053B07EE102A2DED028BB8EE21
:10D87000478A28EE278A002B45D094F8707A002F2B
:10D8800040F0B680B24E0025DFEDB28A4FF00008BE
:10D8900094F8283B2B41DB0712D594F8043B1BBBC3
:10D8A000B4F8063B07EE103A002F46D0B8EE477AA0
:10D8B000C8EE877A77EE887A88EE277A86ED027A44
:10D8C00001352436042DE3D194F8095BB4F80C6BD0
:10D8D000B5BB2FB994F8203B84F8307B84F82C3BFF
:10D8E000BDEC028BBDE8F081B4F8063B301DD4F8E6
:10D8F000241B00EE103AB8EE400ACFB941F056FEB4
:10D9000094F8707ADCE794F8041B94F8212BB1FAB0
:10D9100081F1D4F8100BB4F8065B49092AF09EFE99
:10D9200080B28542A4F8060BA7D094F8707AA9E7D4
:10D9300052F012FF94F8707AC2E7C6F80480B5E797
:10D94000854A94F80A3B52F8782C92F883201343C6
:10D950005ED1A5F1010194F8212BD4F8100BB1FA96
:10D9600081F149092AF07AFE80B2A4F80C0B002F4D
:10D9700061D194F8203B84F8305B84F82C3B00287C
:10D98000AED007EE900A0123B8EE678A9D42DFED24
:10D99000717A84F8343BC7EE888A00F08B80022DC0
:10D9A0009ED1D4F8241BB0EE480A6C4841F0FEFD2D
:10D9B00094F8303B012B00F0C180022B90D1B0EEE7
:10D9C000480AD4F8241B664841F0F0FD94F8303B37
:10D9D000012B00F0AE80022B82D1B0EE480AD4F8C1
:10D9E000241B6048BDEC028BBDE8F04141F0DEBD78
:10D9F00094F8095BB4F80C6B002D3FF471AF564AF4
:10DA000094F80A3B52F8782C92F88320134304D000
:10DA1000002F7FF465AF3046ABE7A5F1010194F824
:10DA2000212BD4F8100BB1FA81F149092AF016FE26
:10DA300080B2A4F80C0BB0423FF452AF00283FF480
:10DA40004FAF94F8303B002B3FF44AAF07EE900AFB
:10DA5000012BB8EE678ADFED3F7AC7EE888A47D0A0
:10DA6000022B7FF43DAFD4F8241BB0EE480A3B48AC
:10DA700052F072FE94F8303B012B52D0022B7FF40F
:10DA80002FAFB0EE480AD4F8241B354852F064FE9C
:10DA900094F8303B012B47D0022B7FF421AFB0EE3E
:10DAA000480AD4F8241B2F48BDEC028BBDE8F04196
:10DAB00052F052BE2C4A0021D2ED007A134678EE85
:10DAC000A76A43F8041F87EEA67A83ED017A78EE01
:10DAD000A76A0021996087EEA67A83ED037A77EE34
:10DAE000A88A00221A6187EEA87A83ED057AF7E604
:10DAF0001D4A1346F3EC017A78EEA76A87EEA67A00
:10DB000083ED017AD2ED007A78EEA76A87EEA67AE5
:10DB100083ED037A77EEA88A87EEA87A83ED057AFB
:10DB2000DEE6114A131DEDE70F4A131DD2ED007A10
:10DB3000F0E70D4A131DD2ED007AD0E70A4A131D13
:10DB4000D2ED007AC3E700BF14000020BD37863550
:10DB5000840A002083F9223ED84C01204C0B00207F
:10DB6000700B0020940B0020B80B0020012816D069
:10DB70002E4B93F8C03B012B2AD02D4BF6EE006ABA
:10DB8000BEEE007ADFED2B7A03EB800010ED170A72
:10DB900080FE660A80FE070A20EE270A7047244AA4
:10DBA000F6EE006A214BBEEE007A12ED160ADFEDAA
:10DBB000217A93F8C43B80FE660A80FE070A20EEB5
:10DBC000270A23B1B5EEC00AF1EE10FA03DC704764
:10DBD0009FED190A704707EE903A32F9721C32F93C
:10DBE0005E3CDFED166AF8EEE77ACB1A07EE103AE4
:10DBF000B8EEC77A27EE267AB4EEE77AF1EE10FA9D
:10DC0000E6DA77EEC77AB2EE047AF4EEC77AF1EE8E
:10DC100010FADCD8B1EE047A67EEA67A30EE470A45
:10DC2000A7EE807AB0EE470A704700BF14000020CC
:10DC3000D84C01200000484300000000CDCCCC3D72
:10DC4000F8B5774B40F6030133F8502C0A402DED20
:10DC5000048BB0EE408A04D0B0EE480ABDEC048BD1
:10DC6000F8BD03EB4003B5EEC00ADFED6E6AF7EED8
:10DC7000007A33F9741CBFEE007A33F9603CF1EEA0
:10DC800010FA694E4FEA8007A1EB030306EB80040C
:10DC9000C8BF012100EE103AD8BF4FF0FF31D4F8D1
:10DCA000C85BB8EEC00A20EE260AB5EEC00AF1EE57
:10DCB00010FACCBF4FF0010C4FF0FF3C77FE877A93
:10DCC0006B1A18BF0123002D08BF0023002B49D178
:10DCD00006F53D62F0EEC06A92ED007AF4EEC76A96
:10DCE000F1EE10FA07DD614508BF002D0CBF0123DE
:10DCF000002300F08580002D42D0B0EE408A4B4AD0
:10DD0000DFED4B8AD2ED006A97EE278A9FED497AC4
:10DD1000DFED497A28EE268A88FE478A88FE278A20
:10DD2000002B61D196F8183C984295D1434C14F8D9
:10DD3000BF3C262B90D1B2EE049A20EE090A50F097
:10DD40006BF8B0EE480A24F8BA5C24F8BC0C50F02A
:10DD500063F828EE890A24F8B80C50F05DF824F82E
:10DD6000B60C79E706F53D63F0EEC06AC4F8C82B3F
:10DD700093ED007AF4EEC76AF1EE10FA3EDC13463A
:10DD800006EB80029FED2E6AD2ED6F7AF0EEE76A25
:10DD9000F4EEC66AF1EE10FA2DDC9FED2A6A66EE0B
:10DDA000866A294AF0EE408AB7EE006A92ED005A80
:10DDB000FFEE005A67EE857AE6EEA78AF5EEC08A96
:10DDC000F0EEE87AF1EE10FAF4EE477ACCBF0124D7
:10DDD0004FF0FF3436FE256AF1EE10FA01DDA14264
:10DDE00014D00025002B9DD00744184B002203EBD4
:10DDF00087035A6096E7F7EE006AD2E76145BED125
:10DE0000F21965460123C2F8C8CB74E7B0EE688A00
:10DE100052ED017A002597EE068A28EE278AE3E77D
:10DE2000D84C0120CDCCCC3D14000020E80B0020C4
:10DE30000000000000007A4400007AC4E03B0120AA
:10DE4000FFFFF9436F12033BEC0B0020F00B0020A7
:10DE500030B46B4C0A7804EB80016A4D534207EEF4
:10DE6000902A51ED176A07EE103A51F84C3CB8EE83
:10DE7000E76A85FB0315DB17B8EEC77AC3EB6513BA
:10DE800007EE903AF8EEE77AE6EE267AF4EEC77AF5
:10DE9000F1EE10FA05D407EE102AF8EE476A86FE76
:10DEA000E77A04EB400040F6010134F8502C30F9D9
:10DEB000743C30F9600C1142DFED536AA3EB0003B0
:10DEC00007EE903AF8EEE77AA7EEE67A06D04F4BE7
:10DED00093ED000A30BC27EE000A704734F9743C19
:10DEE00034F9722C002B54ED107A14ED116AB8BF7E
:10DEF0005B42002A87FE866A4549B8BF52429BB200
:10DF000091F8200C92B29342B8BF134607EE903AB4
:10DF1000F8EEE77A67EEA67A60BB01F62C43F7EEDF
:10DF2000005AD3ED006AF4EEE56AF1EE10FA54D42B
:10DF300001F62441D1ED007ADFED365AF4EEE57AB0
:10DF4000F1EE10FA46D9DFED344AB7EE005AC4EECE
:10DF5000A76AF0EE457AE6EE667AC7FEC56AC6FEA7
:10DF6000A56A2E4BD3ED007A67EE277A30BCA7EE78
:10DF7000A60A704701F624439FED265AD3ED005AB6
:10DF8000F4EEC55AF1EE10FA21DD01F62841D1ED8B
:10DF9000004AF4EEC54AF1EE10FA18DDDFED206A12
:10DFA00074EEE77AB7EE004A26EE266AC7EEA46A58
:10DFB000C6EE257AC6FEC46AC6FE856A77EE847A06
:10DFC00066EEA76AC6FEC46AC6FE856AC9E7F0EEB9
:10DFD000456AC6E7F0EE656AC3E775EEE65ADFED1F
:10DFE000114A9FED115A01F6244165EEA45AD1ED74
:10DFF000004A75EE677AE5EEA76A66EEA47A9BE7BB
:10E00000D84C01201F85EB51CDCCCC3D300C0020ED
:10E0100014000020000000000000C842440C002052
:10E020000000C8C2610BB63B000034432DE9F04F3D
:10E030000C4F17F8BF5C102D2DED048B83B000F052
:10E040006184094C002694F8B987B8F1060F00F2F4
:10E050004484DFE818F0D304940565040B00D8006D
:10E06000A8056903E03B012014000020E34B102DBC
:10E070001A4693ED037AD3ED057AB2EC011A27EE36
:10E08000073A67EEA73A93ED077A92ED006AD3ED6F
:10E09000097A27EE074AD3ED0B6A66EE062A93ED5E
:10E0A0000D7A67EEA74AD3ED0F7A26EEA65AD3ED86
:10E0B000021A67EE075A93ED042A27EEA76AD3EDFA
:10E0C000116AE1EE012A93ED137AA1EEA13AD3EDA4
:10E0D000157AE2EE023AD3ED060A66EEA66A93EDF1
:10E0E000081A27EE077AD3ED0A1A67EEA77A93ED9E
:10E0F0000C2AA0EEA04AE1EE014AD3ED0E0AA1EEF1
:10E10000A15A93ED101AE2EE025AD3ED121A93EDD2
:10E11000142AA0EEA06AE1EE016AE2EE027AA1EE14
:10E12000A17AB1EEE22AF1EEC32AB1EEE33AF1EEC2
:10E13000C43A03ED202AB1EEE44A43ED1F2AF1EE82
:10E14000C54A03ED1E3AB1EEE55A43ED1D3AF1EE34
:10E15000C65A03ED1C4AB1EEE66A43ED1B4AF1EEE6
:10E16000C76A03ED1A5AB1EEE77A43ED195A03ED87
:10E17000186A43ED176A03ED167A93ED177AD3ED1B
:10E18000197A67EE075AD3ED1B6A27EEA76A93ED5B
:10E190001D7AD3ED1F7A66EEA66AD3ED164A27EEF6
:10E1A000077A93ED185A67EEA77AE4EEA45A93ED36
:10E1B0001A4AA5EE056AD3ED1C4A93ED1E5AE4EE09
:10E1C000046AA4EEA47AE5EE057AB1EEE55AF1EE22
:10E1D000C65AB1EEE66AF1EEC76A03ED155AB1EE22
:10E1E000E77A43ED145A03ED136A43ED126A03ED27
:10E1F000117A00F0758794F8B98708F101085FFA81
:10E2000088F884F8B98794F818310F2B00F3B68793
:10E210007B490D2B03F1010C01EB830200F2C38754
:10E2200001F2844A02F5C6620AEB8301D2ED007A5C
:10E2300091ED6C7AB4EE677AF1EE10FA05DDB5EE89
:10E24000C07AF1EE10FA00F346870020DFED6D7A18
:10E250000AEB8C02D2ED6C6AF4EE476AF1EE10FA2A
:10E2600008DDF4EE676AF1EE10FA03DDF0EE667A8F
:10E270005FFA8CF0D91C03F1020C0E29624600F300
:10E28000EE800AEB830292ED6E7AB4EE667AF1EEDE
:10E2900010FA08DDB4EE677AF1EE10FA03DDF0EE65
:10E2A000477A5FFA8CF00AEB8302D2ED6F6AF4EEE4
:10E2B000476AF1EE10FA07DDF4EE676AF1EE10FA44
:10E2C00002DDF0EE667AC8B2591D03F1040C0E2986
:10E2D000624600F3C4800AEB830292ED707AB4EEDA
:10E2E000667AF1EE10FA08DDB4EE677AF1EE10FA14
:10E2F00003DDF0EE477A5FFA8CF00AEB8302D2ED91
:10E30000716AF4EE476AF1EE10FA07DDF4EE676A1F
:10E31000F1EE10FA02DDF0EE667AC8B2D91D03F113
:10E32000060C0E29624600F39A800AEB830292EDF6
:10E33000727AB4EE667AF1EE10FA05DDB4EE677A21
:10E34000F1EE10FA00F3E7860AEB8302D2ED736A6E
:10E35000F4EE476AF1EE10FA05DDF4EE676AF1EECD
:10E3600010FA00F3D38603F1090103F1080C0E291A
:10E37000624674DC0AEB830292ED747AB4EE667A3C
:10E38000F1EE10FA05DDB4EE677AF1EE10FA00F363
:10E39000CD860AEB8302D2ED756AF4EE476AF1EEA0
:10E3A00010FA05DDF4EE676AF1EE10FA00F3B986B3
:10E3B00003F10B0103F10A0C0E2962464FDC0AEB54
:10E3C000830292ED767AB4EE667AF1EE10FA05DD0C
:10E3D000B4EE677AF1EE10FA00F3B3860AEB83022B
:10E3E000D2ED776AF4EE476AF1EE10FA0CDDF4EE46
:10E3F000676AF1EE10FA00F39F8605E068080020D6
:10E40000B40100200000000003F10C01012B0A46BA
:10E4100025DC0AEB830292ED787AB4EE667AF1EEAF
:10E4200010FA07DDB4EE677AF1EE10FA02DDF0EED5
:10E43000477AC8B20AEB8302D2ED796AF4EE476AF2
:10E44000F1EE10FA09DDF4EE676AF1EE10FA04DD80
:10E4500003F10D00F0EE667AC0B203F10E0202F194
:10E460006C030AEB82010AEB830CD1ED6B6A9CED25
:10E47000007AF4EE476AF1EE10FA07D5B4EE677A47
:10E48000F1EE10FA02DDF0EE477AD0B20F2A02F177
:10E49000010C00F0F3830AEB83030AEB8201D3ED56
:10E4A000006A91ED6D7AF4EE476AF1EE10FA05D547
:10E4B000B4EE677AF1EE10FA00F37D860E2A02F1CF
:10E4C000020300F0DB830AEB830191ED6C7AD1ED5E
:10E4D0006B6AF4EE476AF1EE10FA05D5B4EE677A8E
:10E4E000F1EE10FA00F371860F2B03F1010200F038
:10E4F000C5830AEB820191ED6C7AD1ED6B6AF4EE83
:10E50000476AF1EE10FA05D5B4EE677AF1EE10FA2B
:10E5100000F364860F2A02F1010300F0AF830AEBD7
:10E52000830191ED6C7AD1ED6B6AF4EE476AF1EEFE
:10E5300010FA05D5B4EE677AF1EE10FA00F35786BB
:10E540000F2B03F1010200F099830AEB820191ED98
:10E550006C7AD1ED6B6AF4EE476AF1EE10FA05D5EC
:10E56000B4EE677AF1EE10FA00F34A860F2A02F150
:10E57000010300F083830AEB830191ED6C7AD1ED06
:10E580006B6AF4EE476AF1EE10FA05D5B4EE677ADD
:10E59000F1EE10FA00F340860F2B03F1010200F0B8
:10E5A0006D830AEB820191ED6C7AD1ED6B6AF4EE2A
:10E5B000476AF1EE10FA05D5B4EE677AF1EE10FA7B
:10E5C00000F336860F2A02F1010300F057830AEBAD
:10E5D000830191ED6C7AD1ED6B6AF4EE476AF1EE4E
:10E5E00010FA05D5B4EE677AF1EE10FA00F3298639
:10E5F0000F2B03F1010200F041830AEB820191ED40
:10E600006C7AD1ED6B6AF4EE476AF1EE10FA05D53B
:10E61000B4EE677AF1EE10FA00F31C860F2A02F1CD
:10E62000010300F02B830AEB830191ED6C7AD1EDAD
:10E630006B6AF4EE476AF1EE10FA05D5B4EE677A2C
:10E64000F1EE10FA00F31C860F2B03F1010200F02B
:10E6500015830AEB820191ED6C7AD1ED6B6AF4EED1
:10E66000476AF1EE10FA05D5B4EE677AF1EE10FACA
:10E6700000F30F860F2A02F1010300F0FF820AEB7C
:10E68000830191ED6C7AD1ED6B6AF4EE476AF1EE9D
:10E6900010FA05D5B4EE677AF1EE10FA00F30286AF
:10E6A0000F2B03F1010200F0E9820AEB820191EDE8
:10E6B0006C7AD1ED6B6AF4EE476AF1EE10FA05D58B
:10E6C000B4EE677AF1EE10FA00F3F5850F2A02F145
:10E6D000010300F0D3820AEB830191ED6C7AD1ED56
:10E6E0006B6AF4EE476AF1EE10FA05D5B4EE677A7C
:10E6F000F1EE10FA00F3E8850E2B40F0BF82B84B24
:10E7000093ED007A53ED016AB4EE667AF1EE10FAF9
:10E7100040F3B482B4EEE77AF1EE10FA40F3AE8241
:10E72000F0EE477A0F20ACE294F8BA2794F834362A
:10E73000DFF8C0E203F5937CC3F120030CEB421C2D
:10E7400013F0FC0FC3F385005FFA83F80EEB8C0C1B
:10E7500000F00D8501300CF11003AEF170010EF2E6
:10E7600044624FEA00190CEB001013ED026A1033FB
:10E7700011ED027A103253ED076A103153ED057A2C
:10E7800026EE076A51ED074A13ED087A834211ED30
:10E79000085A66EEA46A51ED055A27EE057A02ED95
:10E7A000066A67EEA57A42ED076A02ED087A42ED45
:10E7B000057ADAD18B49A9F1100301F2B4629C44C5
:10E7C000C818134418F003021BD0DCED007A013A9C
:10E7D00090ED007A67EE877AC3ED007A11D0DCED18
:10E7E000017A012A90ED017A67EE877AC3ED017A0A
:10E7F00007D0DCED027A90ED027A67EE877AC3EDFE
:10E80000027A94F83406002863D094F8BA370EEBF5
:10E81000880C5FEA90090EEBC31E0CF2346C01EB1E
:10E8200088080EF5936E35D009F101090EF1100339
:10E8300008F110010CF110024FEA091A0EEB091948
:10E8400013ED026A103311ED027A103253ED076AAC
:10E85000103153ED057A26EE076A51ED074A13EDA4
:10E86000087A4B4511ED085A66EEA46A51ED055A37
:10E8700027EE057A02ED066A67EEA57A42ED076A91
:10E8800002ED087A42ED057ADAD1AAF110039E442E
:10E8900098449C4410F003001BD0DEED007A013850
:10E8A00098ED007A67EE877ACCED007A11D0DEED34
:10E8B000017A012898ED017A67EE877ACCED017A2A
:10E8C00007D0DEED027A98ED027A67EE877ACCED1A
:10E8D000027A102D7BD094F8B98708F10108424BD9
:10E8E000A3FB0823A8EB030203EB52039B08C3EB33
:10E8F000C303A8EB030384F8B93703B0BDEC048B62
:10E90000BDE8F08F37F02AFA384C17F8BF5C06469E
:10E9100094F8B987102D08BF27F8BC8CFFF795BB7A
:10E92000DFF8CC80DFF8D0E0B0EE006AD8ED005A16
:10E93000F6EE006ADEED007A0EF18C03B4F8BC0747
:10E9400077EEA77AD4F8D0170138B0EE664A1031C6
:10E95000B0EE677A08EBC002E5EE867A083A95EEEB
:10E96000867A67EEA67A27EE267ACEED1F7A8EEDAE
:10E97000207AD2ED036A0138D2ED027A01F1080162
:10E9800053ED215AA2F1080253ED224A03F1080384
:10E9900035EEE67A11ED036A37EEE45A77EEA47AA3
:10E9A00076EEA56A51ED045AA6EE057AE5EE857A73
:10E9B000A5EEE67AE6EE267A27EE047A67EE847A0A
:10E9C00003ED037A43ED047AD3D1102D83D137F0D0
:10E9D000C5F9801B94F8B98727F8BA0C7DE700BF0A
:10E9E000240800203401002025499224140000202E
:10E9F000E8070020B4010020EC070020B4F8BC3781
:10EA00009A485908D4F8C02700EB8308DB084FEA7E
:10EA1000810C00EB810A00F0A38003F1010E0CF1E0
:10EA2000100C0AF1100310300AEB0E1AC44402F164
:10EA3000100908F1100E5EED047A103310ED041A7F
:10EA400009F110095CED041A103013ED086A71EE3B
:10EA5000278A5EED032A31EE671A1CED032A36EE93
:10EA6000218A5EED013A71EEC61A13ED064A0EF1E7
:10EA7000100E53ED054A0CF1100C5EED066A53EDD5
:10EA8000075A5CED067A1CED057A35EE820A10ED28
:10EA9000063A72EE655A10ED075A74EE270A10ED29
:10EAA000056A77EEC47A40ED088A35EE229A36EE92
:10EAB000232A35EE625A73EE268A00ED079A74EE29
:10EAC000872A00ED052A37EE647A40ED068A73EE58
:10EAD000666A43ED052A36EE636A03ED088A03EDA4
:10EAE000070A43ED060A534559ED074A19ED084A4E
:10EAF00024EEC12A24EE653A65EE242AA5EE042A06
:10EB000061EE843AB0EE435AE1EE042AE5EEA43A0F
:10EB1000A1EEA45A0EED072A4EED082A4CED073A55
:10EB20000CED085A59ED055A19ED065A26EE253A0C
:10EB300065EEE63A27EE854A65EE474AE6EE053A87
:10EB4000A6EE853AA7EE254AE7EEA54A0EED063A6F
:10EB50004EED053A0CED054A4CED064A7FF46BAFDD
:10EB600089B242480191F9F7F5FA01994046D4F883
:10EB7000C027F9F7EFFA102D7FF4ADAE27E7DFF8E5
:10EB8000EC80D4F8C4274046B4F8C8174DF0AAFA70
:10EB900017F8BF5C102D00F0FE8294F8B9370133EE
:10EBA00084F8B937BEE6324B1B78002B00F0688240
:10EBB000304A94F8BA3702F1DC08D4ED3F7A03EB1F
:10EBC000C300D4F8A41108EB8303D4ED410A02EB8F
:10EBD000800093EDAC0AD0F81CA0D0F8209020EE75
:10EBE000270A90ED054AD0F818B0FCF7FFFE80ED3B
:10EBF000054A6C32C0F818B0C0F81CA0C0F82090CC
:10EC000094F8BA37D4ED407A08EB8308D4F8A4110D
:10EC100003EBC30098EDAC0A02EB800020EE270A5C
:10EC2000D0F814A0D0F81890D0F81C80026AFCF735
:10EC3000DDFE102DC0F814A0C0F81890C0F81C809C
:10EC4000026200F0A08294F8BA270B4B013294F8CC
:10EC5000B907A3FB0213013003F4FF7184F8B9076D
:10EC600001EB5303D21A84F8BA275FE5E8070020C6
:10EC7000000000205C050020ABAAAAAA002800F032
:10EC80004E81431E012B40F3C4820AEB8002811E99
:10EC900092ED6B7A1346D2ED6A6AF4EEC76AF1EE32
:10ECA00010FA00F3828001297FD093ED697AC21EA9
:10ECB000B4EEE67AF1EE10FA00F34982012A00F090
:10ECC0004682D3ED686A021FF4EEC76AF1EE10FACD
:10ECD0006BDC012A69D093ED677A421FB4EEE67AC5
:10ECE000F1EE10FA00F33382012A00F03082D3ED06
:10ECF000666A821FF4EEC76AF1EE10FA55DC012A4B
:10ED000053D093ED657AC21FB4EEE67AF1EE10FAB5
:10ED100000F31D82012A00F01A82D3ED646AA0F18B
:10ED20000802F4EEC76AF1EE10FA3EDC012A3CD08C
:10ED300093ED637AA0F10902B4EEE67AF1EE10FAEF
:10ED400000F30582012A00F00282D3ED626AA0F18D
:10ED50000A02F4EEC76AF1EE10FA26DC012A24D08A
:10ED600093ED617AA0F10B02B4EEE67AF1EE10FABF
:10ED700000F3ED81012A00F0EA81D3ED606AA0F191
:10ED80000C02F4EEC76AF1EE10FA0EDC012A0CD088
:10ED900093ED5F7AA0F10D02B4EEE67AF1EE10FA8F
:10EDA00000F3D581022A07FE267A431C0E2B00F3BE
:10EDB0003C820AEB800100F1020CD1ED6D6A0A463B
:10EDC00091ED6E6AB4EEE66AF1EE10FA00F36E8130
:10EDD000BCF10F0F00F08E80D2ED6F6AC11CB4EE53
:10EDE000E66AF1EE10FA00F15F810F2900F0B281BE
:10EDF00092ED706A011DB4EEE66AF1EE10FA00F3CE
:10EE000055810F2976D0D2ED716A411DF4EEC66AA4
:10EE1000F1EE10FA00F348810F2900F09B8192ED8A
:10EE2000726A811DB4EEE66AF1EE10FA00F33E81DB
:10EE30000F295FD0D2ED736AC11DF4EEC66AF1EE00
:10EE400010FA00F331810F2900F0848192ED746A89
:10EE500000F10801B4EEE66AF1EE10FA00F3268143
:10EE60000F2947D0D2ED756A00F10901F4EEC66AA8
:10EE7000F1EE10FA00F318810F2900F06B8192ED8A
:10EE8000766A00F10A01B4EEE66AF1EE10FA00F3D8
:10EE90000D810F292ED0D2ED776A00F10B01F4EE2F
:10EEA000C66AF1EE10FA00F3FF800F2900F05281DC
:10EEB00092ED786A00F10C01B4EEE66AF1EE10FA18
:10EEC00000F3F4800F2915D0D2ED796A00F10D011D
:10EED000F4EEC66AF1EE10FA00F3E6800E2940F077
:10EEE0003981E14A92ED006AB4EEE66AF1EE10FA79
:10EEF00000F3DC8087FE667AC7EE878A94F8BA97BB
:10EF000009F1AC0BB2EE007A0AEB8B02F7EE007A55
:10EF100092ED008AC8FEC78AC8FEA78A17E0F2EE03
:10EF2000008AB7EE007AC7FEE88AC8FE878A94F89E
:10EF3000BA9794ED450A09F1AC0B0AEB8B0393EDFC
:10EF4000008A88EE000A4EF067FFC0B2431C0AEB4D
:10EF5000800207EE900ADBB292ED6C7AF8EEE76A77
:10EF60000F2B27EE077A66EE876A69D80AEB8302D1
:10EF700007EE903A012892ED6C6AF8EEE77A26EEF9
:10EF8000066AE6EE276A37EE067A59D8B5EEC07AF9
:10EF9000B4F80C31F1EE10FA69DD86EE879A94ED43
:10EFA000457A29EE077AB4F8082107EE902AF8EEA0
:10EFB000677AF4EEC77AF1EE10FA05DC07EE903AC4
:10EFC000F8EE677AC7FEC77A94ED477A77EEC87A8B
:10EFD0000AEB8B0A28EE877AA7EE278A8AED008A49
:10EFE00029F09AFE0028B8BF4042C0B214280DD9BB
:10EFF000B4F8343C07EE903AF8EEE77A87FE888A58
:10F00000BCEEC88A18EE103AA4F8343CB9F1000FEF
:10F0100032D10F2D00F0A180112D6AD1934B9FEDBD
:10F02000940AD3ED007A28EE800AFDEEE77A17EE17
:10F03000903A27F8BC3C4EF0EFFE27F8BA0C4AE4B1
:10F040000138C0B20AEB800307EE900A93ED6C6AB8
:10F05000F8EEE77AB4F80C3126EE066A37EE067A57
:10F06000E6EE276AB5EEC07AF1EE10FA95DCB0EE66
:10F07000487A9FED809A96E7102D7FF42EACA6E497
:10F0800094F8BA377C4803EBC302D4ED410A00EB95
:10F090008303D4F8A41100EB820093EDE30AD0F8C7
:10F0A00014A0D0F81890BFE5F0EE466A87FE667AA5
:10F0B000C7EE878A94F8BA9709F1AC0BB2EE007AE2
:10F0C0000AEB8B02F7EE007A92ED008AC8FEC78A3F
:10F0D000C8FEA78A3BE7F0EE477A1846FFF7B8B8B4
:10F0E00036F03CFE801B17F8BF5C27F8B80CFFF722
:10F0F00082B82B2DC0D15D4BD3ED007AFDEEE77ABF
:10F1000017EE903A27F8BA3CFFF7E5BBF0EE667AC7
:10F11000C8B2FFF728B9F0EE477A5FFA8CF0FFF734
:10F1200013B9F0EE667AC8B2FFF742B9F0EE477A4B
:10F130005FFA8CF0FFF72DB9F0EE667AC8B2FFF7F0
:10F1400063B9F0EE477A5FFA8CF0FFF747B9B0EE9B
:10F15000667A2AE6F0EE466ACCE69FED450A29EE8D
:10F16000000A4EF059FE27F8B60CFFF7B6BBAEF119
:10F1700080010EF234630846FFF724BBF7EE008AE5
:10F18000DFF8F8A0D3E636F0E9FD801B17F8BF5C86
:10F1900027F8BA0C57E536F0E1FD801B17F8BF5C85
:10F1A00027F8BA0CF9E41A4601F2844A0020DFED90
:10F1B000317AFFF754B90E2AF0EE477A5FFA8CF0F5
:10F1C00002F102037FF47FA95BE50F2BF0EE477A93
:10F1D000D8B203F101027FF48CA952E50F2AF0EEB8
:10F1E000477AD0B202F101037FF499A949E50F2BC8
:10F1F000F0EE477AD8B203F101027FF4A6A940E508
:10F200000F2AF0EE477AD0B202F101037FF4B3A9DE
:10F2100037E5B7EE007AC8E50F2BF0EE477AD8B2A3
:10F2200003F101027FF4BDA92BE5F7EE006A61E668
:10F230000F2AF0EE477AD0B202F101037FF4C7A99A
:10F240001FE50F2BF0EE477AD8B203F101027FF4ED
:10F25000D4A916E50F2AF0EE477AD0B202F10103E5
:10F260007FF4E1A90DE500BF24080020E808002094
:10F270000000C842000000005C05002038060020A5
:10F280000F2BF0EE477AD8B203F101027FF4E1A927
:10F29000F7E40F2AF0EE477AD0B202F101037FF4CF
:10F2A000EEA9EEE40F2BF0EE477AD8B203F101029B
:10F2B0007FF4FBA9E5E40F2AF0EE477AD0B202F121
:10F2C00001037FF408AADCE40E2BF0EE477AD8B2F3
:10F2D0003FF415AAD5E4F8B5214C1D270E46054686
:10F2E00004F8387C1DF07AFF00201DF01BFF082079
:10F2F0001DF018FF0E201DF015FF38461DF012FFFF
:10F3000004201DF00FFF04201DF00CFF00201DF055
:10F3100009FF30201DF006FF00201DF003FF3046DE
:10F320001DF000FF00201DF0FDFE1DF043FFA4F1C5
:10F3300037001DF04CFE234670B114F8372C62B92B
:10F3400014F8362C302A00D03AB913F8352C22B9EB
:10F3500013F8343C01202B70F8BD0120FCE700BFFE
:10F36000D84C0120104B034410B5044693F8040612
:10F3700015F0EAF90D480A2300EB4404092034F99A
:10F38000241CB1F5FA6FA8BF4FF4FA61B1F57A7F8A
:10F39000B8BF4FF47A71A1F57A71B1FBF3F1BDE812
:10F3A0001040C9B215F0D8B978070608D84C01202A
:10F3B0001C4991F8542F9AB3F0B400260546334601
:10F3C000304637461BB991F8544F2D2C22D02E2AA7
:10F3D00018D0CA1800EB800092F8544F4000A4F1F6
:10F3E0003002092A02D8A0F13002A0180E2B14D83E
:10F3F0000133CA1892F8542F002AE3D106B14042D3
:10F40000F0BC70470133002DF8D0CA182A4482F8A6
:10F41000547FDEE701231E46EBE70020F0BC704777
:10F4200000207047E03B01201FB503AC8DF80C3085
:10F43000002300948DF80D3010F022F804B010BDB8
:10F44000F8B50546262026F0CFF8114C0146D0B974
:10F45000206890F838301E3B012B01D937F0D2FDDF
:10F460000C4F0026AE4207DBA38C0133A3840A4B6A
:10F4700053F8B83C6363F8BD17F8011B01362068E8
:10F4800037F0C0FDEEE7002384F83230EFE700BF2D
:10F49000D84C0120DC4C0120E82A012010B5F9F7F6
:10F4A00097FF044611213AF02BFD20463AF092FED8
:10F4B000C82036F0D1FC2046BDE810403AF090BE9E
:10F4C00008B53E203AF036FD044B986308B12A2374
:10F4D000C3804021BDE808403AF012BDD84C01205D
:10F4E000F8B5684CD4F8DC110B699E0702D5CB68DF
:10F4F0009D074BD40B69580702D5CB685A073DD4FA
:10F500000B691B0702D5CB681F072FD40B69DE06DA
:10F5100002D5CB68DD0621D40B69D80702D5CB68AC
:10F52000DA073FD40B691B0603D5CB681F0600F131
:10F530008E800B69DE0503D5CB681D0600F18B803C
:10F540000B695C0603D5CB68580600F188800B690F
:10F550009A0602D5CB689B0620D4F8BD6FF0100246
:10F5600000230A61CA6984F8F831D5E76FF0080210
:10F5700000230A61CA6984F8F831C7E76FF0040212
:10F5800000230A618A6984F8F831B9E76FF0020252
:10F5900000230A618A6984F8F831ABE76FF0200331
:10F5A0000B61F8BD384B6FF0010299420A61B9D185
:10F5B00041F224033548C558D5F81432002BB1D197
:10F5C000334FFA6B8AB1D0F878C502F03F06624437
:10F5D000C0F87825D0F87825B2F5006F01D1C0F8D1
:10F5E00078350023FB63002E43D0D0F87825D0F87F
:10F5F0007C359A4296D0D0F87825D0F87C359A425E
:10F6000031D9D0F87865C6F50066D0F878C5B6F57A
:10F61000007F204A28BF4FF40076D5F814326244A8
:10F62000C5F81062C5F80822002B7FF47BAF0123D8
:10F6300041F23C01C0F8C46DC5F81432334640585D
:10F64000812105F05BFBD4F8DC11FE636AE76FF003
:10F6500080030B616DE76FF480730B6170E76FF0EF
:10F6600040030B6173E7D0F87C65D0F87835F61A63
:10F67000CBE7D0F87825074BC5F810621344C5F8DE
:10F6800008324FE7E82A012000140040F019012059
:10F69000D84C0120841F012070B5D0F8A852C1EBCE
:10F6A000C1000C46002605EB80001C21C0F8082292
:10F6B000C0F8103280F8FC41C0F8146280F8FD6197
:10F6C0002B6901FB0451012B01F5FE7108BFC0F845
:10F6D0000C22DAB228681CB905F028F8002070BDA9
:10F6E00005F0B0F8002070BD0E4841F22403C35865
:10F6F00010B5A3B190F8A44D00F69450D3F80422AD
:10F7000034B1002440230121FFF7C6FF204610BD7D
:10F710004FF400730121FFF7BFFF204610BD022404
:10F72000204610BDF019012010B50B4CD4F88035DF
:10F7300053B10A49013B0A6CC4F8803512F8014BF9
:10F740000A64047013B10123184610BDFFF7CCFF03
:10F750000123184610BD00BFF0190120D84C01202C
:10F7600013B5064C236C03B9FEE701A8FFF7DCFFD5
:10F770000028F7D09DF8040002B010BDD84C01203D
:10F7800010B50B68054C064AC4F8803510640BB1FF
:10F79000002010BDFFF7A8FF002010BDF0190120C8
:10F7A000D84C012038B5D0F8A84201F00F036268A8
:10F7B00093422BD80A062BD41C25C1EBC102002092
:10F7C00005FB014104EB820201F5FE7182F8FD01A7
:10F7D00001220B708A7094F8BC03904216D084F812
:10F7E000BC234A782068012A09781DD000F53062D0
:10F7F00002EB41121568002D00DBF1B9116841F4EC
:10F80000001111601BB3002384F8BC33002038BD05
:10F810001C21C3EBC302012001FB034104EB820264
:10F820003C3182F83D00D3E700F5106202EB411253
:10F8300015680029E2D0002DE0DB116821F080413D
:10F840001160116841F400111160002BDBD104F547
:10F850007172217C04F03EFFD5E700BF10B504466D
:10F860008021FFF79FFF00212046BDE8104099E767
:10F8700011F0800F01F00F01F0B4D0F8A8424FF062
:10F880001C0042D1C1EBC10500FB0140002604EB86
:10F89000850500F5FE7085F8FD614578017083608F
:10F8A000C27005B1C180022A01D10023037194F80E
:10F8B000BC33012B1AD00122236884F8BC23417881
:10F8C000057891422CD003F5006605F00F0103F591
:10F8D00030638A40F16903EB451341EA0242F26169
:10F8E0001A68120405D5002384F8BC330020F0BC4C
:10F8F000704782681D68C2F30A02C07818492A431B
:10F9000042EA804211431960EDE7C1EBC1050126CF
:10F9100000FB014004EB85053C3085F83D60BCE709
:10F9200005F00F06D3F81CC803F5106203F5006755
:10F93000B14002EB451241EA0C01F9611368190468
:10F94000D1D483681668C3F30A03C07804493343EB
:10F9500043EA804343EA855319431160C3E700BF7C
:10F96000008000102DE9F04F854E83B035686C693A
:10F9700014F0010402D003B0BDE8F08F6A69AB69EE
:10F980001A42F8D06B69AA6913409F0703D56B69C7
:10F9900003F002036B616B69AA691340180379D401
:10F9A00028464369826913405F0300F1D5804269AC
:10F9B00083691A4200F1BA804369826913401905CC
:10F9C00008D5D5F80838DA0700F14783436903F40E
:10F9D000006343614369826913401B0110D5436989
:10F9E00003F00063436196F8F433002B40F0488243
:10F9F000012386F8F433436DC3F38303C6F8F83369
:10FA0000436982691340DF0400F1CD814369826953
:10FA100013409A0400F17081436982691340DB0648
:10FA200012D5836923F0100383612B6AC3F3434229
:10FA300003F00F01022A00F0E582062A00F05E8240
:10FA4000836943F0100383614369826913401F0790
:10FA500000F10B82436982691340DD0200F10082EC
:10FA60004369826913409C0200F1F5814369826910
:10FA70001340590000F1EA814369826913405A0733
:10FA80007FF579AF4468630700F1F18243681C4356
:10FA9000446070E7D5F81878D5F81C381F403F0C43
:10FAA0003FF47EAFDFF8D8A028464FF0000800945E
:10FAB00006E07F0808F101080AF11C0A00F0328212
:10FAC000F907F6D55FFA88F100F5306B0BEB4112C0
:10FAD0009268D0F8143802EA030919F0010F40F0D7
:10FAE000268219F0080F40F0598219F0100F05D046
:10FAF00005F53063102203EB48139A6019F0200FCC
:10FB000009D03169012900F0558305F530632022C1
:10FB100003EB48139A6019F4005FCAD005F530630F
:10FB20004FF4005203EB48139A60C2E7D5F804384B
:10FB300023F00103C5F8043896F8F433012B00F0E4
:10FB4000B681D6F8003493F8752283F8742243699D
:10FB500003F0004343612FE7D0F81838D0F81C2891
:10FB600013409BB2002B3FF422AF05F510620095C5
:10FB7000034F4FF0000A1D469046019409E000BF74
:10FB8000F01901206D080AF1010A07F11C0700F0C5
:10FB9000CB81E907F6D55FFA8AF9D0F81028D0F8BA
:10FBA000344800F5106309F00F0103EB4913CC4012
:10FBB0009B68E401E4B214431C40E20732D54FF0E5
:10FBC000010E009B0AF00F0C08EB4A12D3F8341810
:10FBD0000EFA0CFC21EA0C01D6F810C0F445C3F86B
:10FBE0003418C2F808E003D1D7E911231344BB64E9
:10FBF000D6F800B4B9F1000F40F0E981DBF86C32BF
:10FC0000022B00F0E78233F0040300F01B839BF823
:10FC10007832012B02D100238BF87832BCF1010F2E
:10FC200000F0CD82230703D508EB4A1308229A601F
:10FC3000E10603D508EB4A1310229A60620603D549
:10FC400008EB4A1340229A60A30703D508EB4A1336
:10FC500002229A60240695D5D7E91441A14291D891
:10FC6000621A7B6C00EB4A1C93420CF5106C28BFA7
:10FC70001346DCF81820033392B2B2EB930F2CD367
:10FC800009F10109864600EB09392CB3A14223D2C0
:10FC9000621A7B6C307C9A4228BF1A46BB6C02F118
:10FCA000030B4FEA9B0B70B990B2033080080AD067
:10FCB00003EB800153F8040B8B42C9F80000F9D123
:10FCC000BB6CD7E91441DCF818001344114480B22E
:10FCD000BB6479658345D8D97046A142FFF452AF21
:10FCE0000AF00F010124D0F8342804FA01F122EAC5
:10FCF0000102C0F8342845E7D0F8001900F5006388
:10FD0000BB4A0A40C0F800299A6802F00602042A99
:10FD100000F0D1805A6842F480725A609B6813F0F8
:10FD2000060340F0B081C268F36022F47052C260F2
:10FD3000C36843F41053C3604FF00009D6F8004481
:10FD40004FF0400800220127434620461146FFF7A6
:10FD50008FFD4346002220468021C4F84471C4F838
:10FD60005081FFF785FD0023D4F8A022A761C4F8D5
:10FD7000248084F87472C4F86C326360C4F87C32F6
:10FD8000002A00F0F281D4F88C32204600215B6812
:10FD90009847D6F80034306883F81090436903F42C
:10FDA0000053436138E6D5F804284FF4846105F523
:10FDB000006C904B22F00102CCF80420016101E0BC
:10FDC000013B02D002699106FAD4D6F804E0BEF1F4
:10FDD000000F15D005F510634FF67F31996001349F
:10FDE0001A682033744522F4001243F8202CC3F81B
:10FDF000E811D3F8E02122F40012C3F8E021EDD19C
:10FE0000DCF81C30326B43F00113CCF81C30002AB4
:10FE100040D1DCF8142042F22B031343CCF8143009
:10FE2000DCF8103043F00B03CCF81030D5F8003874
:10FE3000317C23F4FE63704AC5F8003804F04AFCB4
:10FE40003068436903F480534361DFE5436903F09D
:10FE50008043436110E6436903F40013436105E600
:10FE6000436903F480134361FAE5D6F8003493F84C
:10FE70007422032A39D0436903F008034361E9E59A
:10FE8000D6F80034042193F8742283F8741283F8AE
:10FE90007522B5E5DCF8843043F00B03CCF88430F0
:10FEA000DCF8443043F00B03CCF84430BEE70023C9
:10FEB00086F8F4334BE6D0F8002942F00302C0F88C
:10FEC00000295A6842F480725A609B6813F0060356
:10FED00040F0D980C368002223F47053F260C360FD
:10FEE000C36843F41053C36026E7D3F88C22D26969
:10FEF000002AC0D0184690473068BCE7C1EBC1016A
:10FF000005F58055C3F30A1306EB81022C68D2F87D
:10FF10001412C6F8C4430B442968C2F81432C6F858
:10FF2000C8138DE5009C3CE5DDE900543FE505F58F
:10FF300030634FF0010C32690BEB481B03EB4814A4
:10FF40006245C4F808C0D0F840E0DBF8083000F0A3
:10FF500017812A4A964540F0FC801A0440F1F4804B
:10FF60004FF4004219F0080FCBF808203FF4BDAD64
:10FF7000026CDBF80800214B9A4200F0D1801E4948
:10FF8000D6F80004019205F0B1FD1D4B019A9A428A
:10FF900000F2D18008223068A260A6E54FEA48133B
:10FFA0003169026C03F5306B012905F5306183443A
:10FFB00001EB0304DBF80800DDD1114B9A4200F29B
:10FFC000AF800D49D6F8000405F090FDE2E7DBF8BC
:10FFD0008C325B69002B3FF425AE9BF87422032A18
:10FFE0007FF420AE58464946984730681AE600BF6D
:10FFF00000F8FFFF400D0300B41D01200A31544FEB
:020000040801F1
:100000000A30544F47F6F07213423FF419ADC3F370
:100010000A14C1EBC1024FEAC10C2346033406EBBC
:100020008202A408D2F8082208D005F5805502EB18
:1000300084072C6842F8044BBA42FAD1ACEB0102B7
:1000400006EB8202D2F80842D2F814121C440B4488
:10005000C2F80842C2F81432F2E4D6F8003404219F
:1000600093F8742283F8741283F87522AEE4D6F8FC
:1000700000040122D0F88C3280F8742201795B6888
:100080009847306802E523F00403002B3FF422AFC9
:10009000A64A0324A64BD2F8D821A6491344F460FB
:1000A0008B4240F2BF80A44BA44913448B4240F2E0
:1000B000D180A34BA34913448B4240F2EF80A24B63
:1000C000A24913448B42C0F02181A14BA1491344A2
:1000D0008B4240F21E81A04BA04913448B42C0F0DA
:1000E0001B819F4B9F4913448B42C0F01B819E4B49
:1000F0009E4913448B42C0F012819D4B9D4913448D
:100100008B4234BF4FF4E0534FF4C053C2684FF0FA
:10011000010922F47052C260C2681343C3600DE645
:10012000030403D54FF40042CBF808209249D6F8D7
:10013000000405F0DBFC316901297FF42BAF8E4A06
:10014000306804F0C7FA25E79A0602D52023CBF8D9
:100150000830C1EBC103D6F8000406EB8303D3F8E3
:10016000082205F0AFFA3068BBE4D4F89032002BD7
:100170007FF409AED4F89832002B7FF404AE08E681
:100180001A0752D57D4A964505D9190403D54FF46F
:100190000043CBF808307849D6F8000405F0A6FCF7
:1001A000754A0121306804F095FA08233068CBF8CD
:1001B000083096E4704A04F08DFA3068A5E4336D97
:1001C0005AEA03037FF42EAD61466B4A04F082FACB
:1001D000306827E5DBE908239A423ED8DBF81C109B
:1001E000B1FBF3F203FB12120AB98B4259D9DBF8C7
:1001F0008C32DB682BB19BF87422032A01D158465C
:10020000984780215846FFF7CDFA0023052258462B
:100210001946CBF86C221A46FFF73EFAD6F810C002
:100220003068F4E44FF4705370E79A0629D5202221
:10023000CBF8082019F0080F3FF457AC026CDBF83C
:100240000800BAE680215846FFF7ACFAD6F810C08D
:100250003068DCE44FF4605358E7D31A4946B26C77
:10026000DBF8A802CBF820309BB204F047FD4B46E8
:100270004A4649465846FFF70FFAD6F810C030688C
:10028000C5E413F0280FD5D13C4A964517D91B0475
:1002900015D54FF40042CBF80820CBE74FF450536C
:1002A00034E7DBF870329942A1D24B464A464946C0
:1002B000DBF8A80204F022FDCBF87092D7E7DBF858
:1002C0001020C1EBC100DAF80432C2F3120CDAF8E4
:1002D000082206EB80001A44A3EB0C03CAF808229C
:1002E000D0F80822D6F80004CAF8143205F0EAF96A
:1002F000D6F8103258EA03037FF435AF1E4A0121C5
:10030000306804F0E7F93068FFF7EBBB4FF4405377
:10031000FCE64FF43053F9E64FF42053F6E64FF481
:100320000053F3E64FF41053F0E600BFE82A012033
:10033000405327FFFF340C00401E1BFF3F420F00BD
:1003400000DC0BFF7F4F1200808CF9FE20D61300DB
:1003500060B6E5FE5FE3160000D3CEFE40771B00DB
:10036000C05BB3FEC091210000CA91FE2075380029
:10037000E05459FEE09C4100B41D01200A30544F66
:100380002DE9F0414FF0FF35324A002332482C4628
:1003900003E0013310320B2B14D0917A0429F8D1E9
:1003A00003F5B17100EB0111C979CF07F1D4661CD7
:1003B000116801D0A942ECD21C4601330D4610321F
:1003C0000B2BEAD1631C02D10120BDE8F081224D44
:1003D00004F5B17705EB07139988E9B92601DFF831
:1003E0008480AA19D8F8B43541F218601B491E69F7
:1003F0000023105801EB4421194AB047E0B102280C
:1004000017D141F2CC6205EB071701210020AB5850
:10041000B971013BAB50D8E7DFF8488005EB041217
:1004200041F218602601D8F8B4351058DB689847B7
:10043000D7E70020BDE8F08141F2CC62032405EB50
:10044000071741F2D061AB58BC710124013B6C54D9
:10045000AB50BAE7F8650120DC4F0120F44F0120D2
:1004600081040108E03B0120044B41F2E472995CF5
:1004700009B90121995401225A707047DC4F0120BB
:1004800070B50024164D41F2D066164B2046AC558F
:1004900003E0013010330B2814D053F80E4C8C427B
:1004A000F7D11C78032CF4D16AB10F4B03EB402336
:1004B0009A4201D0FFF7D8FF00F5B170012305EB98
:1004C0000010837170BD41F2CC6100F5B17304205E
:1004D0006A5805EB0313013298716A5070BD00BF72
:1004E000DC4F012002660120F44F012038B50020C6
:1004F000114B9C7B14B11D688D4204D00130103328
:100500000B28F6D138BD82B10C4B03EB40239A4245
:1005100001D1022C01D0FFF7A7FF00F5B170084B05
:10052000012203EB0010827138BD00F5B170044B5D
:1005300003EB0010827138BDF4650120F44F0120F7
:10054000DC4F01202DE9F04F83B002F0020C019343
:1005500010B9BCF1000F60D1844C41F638056559E3
:10056000002D61D14FF0FF36814F0025B146B046D6
:10057000B2463B68984200F0BE8097F80EE0BEF1AC
:10058000000F62D0BEF1010F15D105F5B17E04EB6D
:100590000E1E9EF807E01EF0010F0CD11EF07E0F1C
:1005A00009D15FEADE1340F0B080D7F808E0F245E9
:1005B00001D9F246A946013510370B2DD9D1751C4A
:1005C00004D1B8F1FF3F00F0A780464641F2C86869
:1005D00006F5B17704EB061E41F21C6A54F8085088
:1005E0004FEA071941F2186B01354EF80B0044F839
:1005F000085004EB07184EF80A5044F8095000253B
:10060000C8F8045004EB0715AD79042D00F2A98059
:10061000DFE805F02139163955000225FFF724FFE0
:10062000284603B0BDE8F08F04F5C25741F63C06FA
:100630003F68A65907FB0565A84293D3FFF714FF4F
:100640000025284603B0BDE8F08F2E46013510374F
:100650000B2D8ED1B3E712F0010E6FD104EB071012
:10066000019BD51090F80780032B65F3C71880F81D
:10067000078061D94FF6FF70834228BF03469BB2C3
:1006800004EB07108380BCF1000F18D004EB0610B8
:1006900041F218630344987B042810D041F2C86CDF
:1006A00041F2CC654FF0040E54F80C00013044F8D0
:1006B0000C00586083F80EE0635901336351500712
:1006C00005D504EB0710C37943F00103C371D306CA
:1006D00008D504EB0714E379C3F34502013262F352
:1006E0004603E371234B012503EB462628460E60A3
:1006F00003B0BDE8F08F05F5B17704EB07164FEABC
:10070000071EB6796EB92E4660E7A8460135103748
:100710000B2D7FF42EAF52E7B9F1FF3F90D04E463C
:1007200054E741F2C8682E4654F80850013544F8A1
:10073000085044F80E5065E77346A1E70E4A0023BF
:100740000C49D2F8B4C501EB46210C4ADCF808602C
:10075000B04700283FF474AF04EB07140223A371E1
:100760005EE70225FFF780FE5AE700BFDC4F01205D
:10077000F4650120F44F0120E03B0120ED04010865
:10078000F0B5154D83B00E462B78022B0FD14FEAF2
:10079000102CC4B241F630070023012201A9E85908
:1007A0006044FFF7CFFE012806D003B0F0BDC0F3D0
:1007B000D41C00F07F04EDE72B78022B019B04D1C1
:1007C00033F81430336003B0F0BD53F8243023F015
:1007D0007043336003B0F0BDDC4F012010B5144608
:1007E00002070B4610D50B4941F2C472581C8B58B6
:1007F000834204D305D100230120236010BDFFF7FD
:1008000033FE2060012010BD21461846BDE810408F
:10081000B6E700BFDC4F01202DE9F0410D464168ED
:1008200082B00446C1F308032B44B3F5007F58D3CC
:1008300090F91A30591C0AD0304A03F5B173FF21E0
:1008400002EB0313DA796FF30002DA71817694F91F
:100850001B305A1C0FD0294A03F5B173FF2002EB5D
:100860000313DA79C2F34501013921EAE17161F339
:100870004602DA71E0762378022B38D01F4A02F55F
:10088000C2531B68B5EB432F4FEA432825DC41F6E2
:1008900048036768D6583E407242AA421DDCAB1935
:1008A000434512D301AA2169207EFFF797FF012853
:1008B00013D16768A5EB0805206908EB0703019AC7
:1008C000354460619F1B226167602046F8F718F984
:1008D00020B93D440120656000E0002002B0BDE881
:1008E000F08129440120616002B0BDE8F0816168B7
:1008F00001202944616002B0BDE8F081DC4F012095
:1009000070B5154604460E46FFF786FF50B994F8B9
:10091000280028B90223C4E90B5684F8283070BD9A
:10092000022070BD1DB12046A847012070BD0120E6
:1009300070BD00BFD0E9011310B48B4290F91A20AA
:1009400038BF0B46511C83600AD0144B02F5B172BC
:10095000FF2103EB0212D3796FF30003D371817689
:1009600090F91B305A1C0FD00C4A03F5B173FF24C9
:1009700002EB0313DA79C2F34501013921EAE1718F
:1009800061F34602DA71C4760022436A5DF8044BD3
:100990001146426142600361B2E700BFDC4F0120B3
:1009A00070B544220021114841F602044FF0ACFD1D
:1009B0000F4B032141F64C001A784FF6FF761D5875
:1009C00003F5C050022A1E5341F2E87641F60C04AA
:1009D00018BF0A4600F8181941F601011D519A5531
:1009E00010225A54FFF7A6FF012070BDC4670120F2
:1009F000DC4F0120B1F904300F2B2DE9F0410C46FA
:100A000082B01646054633D02846F8F7A1F895F986
:100A10001B800746B8F1FF3F34D02D4B41F21862DE
:100A200003EB08118A58904212D1183303EB482384
:100A3000A1882846013109B203EB4113A18033603C
:100A4000F8F786F803460120236002B0BDE8F08184
:100A5000FFF70AFD2846F8F753F828B100230120D4
:100A6000336002B0BDE8F081002002B0BDE8F08143
:100A70004FF40071FFF7D0FE0028F5D04FF6FF735A
:100A8000A380C1E72846F8F73BF80028E2D10FB968
:100A9000FFF7EAFC38460023112201A9FFF752FDB7
:100AA0000128D7D1019B0B4A9A1A48BF02F2FF12C4
:100AB000B2F5B05F4FEA622106D24FFA81F885F8AD
:100AC0001B80002BB4D1C5E7FFF7CEFC019BF6E7F6
:100AD000DC4F0120F44F012030B50446C06983B0DB
:100AE00010B9012003B030BD0D460023032201A937
:100AF000FFF728FD0128F5D1B4F92030002B03DAE7
:100B0000FFF7B2FC0220EDE7019A012D4FEA4311F5
:100B100002EB431303D0022D12D1E5255554A268F0
:100B2000DA612278032A04D100221A775A779A7759
:100B3000DA77626AC2F30F415A83998203B030BDFB
:100B4000E268DA61EDE700BF10B503780446023BC6
:100B5000012B037E02D913F0060F5AD198063AD41E
:100B600094F91A30591C0AD02D4A03F5B173FF21AC
:100B700002EB0313DA796FF30002DA71A17694F9CC
:100B80001B305A1C0FD0264A03F5B173FF2002EB2D
:100B90000313DA79C2F34501013921EAE17161F306
:100BA0004602DA71E076237E1B070BD51C4841F222
:100BB000C873C35C072B01D0FFF756FC41F2C87322
:100BC0000022C2540023E26A237084F82830FAB16C
:100BD000BDE81040104700231249E0691A018A5805
:100BE000904206D001330B2BBAD01A018A5890429A
:100BF000F8D10B4A03F5B17302EB0313DA79C2F3B0
:100C00004501013921EAE17161F34602DA71A7E792
:100C100010BD0121FFF760FF0128F9D1237E9DE778
:100C2000DC4F0120F4650120B8B138B5027822B15B
:100C300090F828201AB1002038BD012038BD826804
:100C400003244568C162AA4280F8284038BF2A467A
:100C50008260FFF779FF012038BD0120704700BF97
:100C60002DE9F04FDFF84C91174683B08A4699F88A
:100C700000300A68022B7BD1D6B241F630044FF423
:100C80008071A6EB020859F80450B84405EB122510
:100C90008844BA4208F1FF38B8FBF1F864D200F09A
:100CA000010BA844032B06EB0704A8EB05030CBFBC
:100CB00080214FF48071A41A8C4228BF0C460EB9D3
:100CC0008C4235D20B2201A92846FFF73BFC0128B4
:100CD00002D003B0BDE8F08F99F80010DAF80020D8
:100CE000022902F1010325D0A64210D2019A6FF029
:100CF0004040111F304401EB840102EB800242F8B6
:100D0000043F914203F10103F9D1DAF80020A61B58
:100D10003244BA42CAF8002002D1BBF1000F39D1E7
:100D2000BA4205F101051FD299F800300026B9E753
:100D30000A22C8E7A642EAD201996FF0004C881E49
:100D4000B44400EB440001EB4C0121F8023F88421F
:100D500003F10103F9D1DAE76FF00043019A4FF68E
:100D6000FF71234422F81310012003B0BDE8F08F77
:100D700041F6300102F07F06032BC2F3D41559F877
:100D80000140A6EB020814BF4FF480718021B844E3
:100D900025447DE799F80030022BDDD06FF0404309
:100DA000019A4FF0FF31234442F82310DAF8002073
:100DB000B6E700BFDC4F0120F8B590F838300446A4
:100DC000032B4ED8DFE803F0023039442B4B41F2BD
:100DD000A87EC56841F2C47C187803F5C25153F867
:100DE0000C2041F2AC770328096853F80E000CBFC1
:100DF00080264FF48076226101FB06F105EB412548
:100E0000A0EB4120E560951943F80E00D85943F84E
:100E10000C50A0EB4121E06AD951C4E90C2548BB34
:100E20006262012384F8383000211548FFF754FE30
:100E3000012811D1022384F83830626B04F13001AB
:100E40000120FFF70DFF012806D1032384F8383075
:100E500000212046FFF740FE431EDBB2012B01D9E3
:100E6000F8BD022094F82830062BF9D1002384F82D
:100E70002830F8BD921B2263D3E700BFDC4F01206E
:100E80007C6701202DE9F04FDFF82481012887B02D
:100E90000C4698F800608CBF002301231546032EF2
:100EA00002930B6839D0022E62D14FF480724FEA60
:100EB0001329DFB201920138012823D801220392BD
:100EC0009D421AD9384E06F1880A06F11C0B326889
:100ED0001AB1DBF8001099424ED0DAF80000002376
:100EE000092205A94844FFF72DFB01281FD002283D
:100EF0000FD020B123689D42E9D80320256007B0B8
:100F0000BDE8F08F87B1FFF7AFFA022007B0BDE868
:100F1000F08F022007B0BDE8F08F80220192C3F36A
:100F2000D41903F07F07C6E7019A0392C8E7059A30
:100F3000DDF804E0DDE902C198F80030022B14D09E
:100F4000032BE6D152F8273023F07043B3FA83F332
:100F50000F445B096345236823D00B447745236026
:100F6000EAD309F101090027C5E732F81730EDE7A8
:100F70004FF480720192D2E70C49013A096802EB02
:100F800041224902B2FBF1F203991344B3FBF1F29F
:100F900001FB12320AB10B449B1A9D42236096D882
:100FA000ABE7AB42ABD3A8E7846701201C68012004
:100FB000DC4F0120F0B5114D83B00E462B78022B8B
:100FC00017D14FEA102CC4B241F630070023032298
:100FD00001A9E8596044FFF7B5FA012807D12B7839
:100FE000022B019B0CBF23F8146043F8246003B06C
:100FF000F0BDC0F3D41C00F07F04E5E7DC4F012016
:101000002DE9F043002990F83C3083B0044614BF2A
:1010100002210021042B7BD8DFE803F0030C3C47BE
:101020006900FFF759FD012870D1626B002A75D164
:1010300084F83C00404E4FF6F777DFF804813F4DCF
:101040001BE0B94594BF4FF000094FF0010901A919
:10105000B9F1000F48D1FFF793FB0128494652D15F
:10106000206BFFF7A7FF01284DD1019A2B68511E75
:1010700022638B4228BF0B462B603378206B032BF7
:101080001FFA80F9DDD1404594BF4FF000094FF0C1
:101090000109DCE7426B04F130010020FFF7E0FDBD
:1010A000012833D1032384F83C30234B41F2C47030
:1010B000E16A41F2A8771A5803F5C255195041F276
:1010C000AC76511A2A68D85902FB01F2995900EB03
:1010D000422503F5BD5001EB42220021DD519A511A
:1010E000FFF7FAFC012811D1042384F83C3094F86E
:1010F0002830042B02D1002384F82830A36B8BB155
:1011000020469847012003B0BDE8F0830228FAD1B9
:1011100094F82830042B09D00220F4E7022384F845
:101120003C30B8E7012003B0BDE8F0830023022083
:1011300084F82830E7E700BFDC4F01202068012059
:10114000F7FFFF0F38B590F834300446052B42D82E
:10115000DFE803F01E033B0F1868006B4FF0FF3110
:10116000FFF728FF012836D1E06AB0BB032384F8DB
:10117000343000212046FFF7AFFC01282BD1042397
:1011800084F8343094F82830082B2AD0012038BD58
:1011900041F63803244D00F130010120EA580232B3
:1011A000FFF770FE01282AD00238C0B2012812D8F9
:1011B000052384F8343094F82830082B16D041F2F7
:1011C000E57301220220EA5438BDC06A216BFFF7A3
:1011D000F1FE0128CAD0002038BD022384F8343043
:1011E000F4E70023012084F8283038BD00230122D1
:1011F000022084F8283041F2E573EA54E4E705F56B
:10120000C252E368206B41F644011268685003EB58
:101210004223E26AC4E9033002B96062012384F820
:1012200034309BE7004DC6E7DC4F012043682DE9D1
:10123000F04F164683B0C3F30808002A00F0DF80A1
:10124000704B054689464FF0000AA3F1180BC8F50C
:10125000007495F91A702846B44228BF3446791CA8
:101260002ED0F7F775FC41F218620BEB07139B5871
:10127000984205D0FFF7F8F8504603B0BDE8F08F6C
:10128000604B03EB4720224649464044A2444FF0BE
:10129000C9F8002221462846FFF732FB0028EBD090
:1012A0002B7E1B0706D5584B2A691B689A4201D32F
:1012B000FFF7DAF8361BA1444FF00008C7D1DBE78F
:1012C000F7F71EFC002846D12846F7F741FC69686D
:1012D000C1F308031BBB4D4AAB680A4002F500721C
:1012E0009A422CBF062207222B7E03F00C030C2B04
:1012F0001BD0002301A9FFF725F90128BCD10198D3
:10130000404BC31A48BF03F2FF13B3F5B05F4FEA77
:1013100063224CD257B2AF760028B4D1ACE72B7E13
:10132000072203F00C030C2BE3D19BF800C0384BD1
:10133000BCF1030F1B680CBF4FF0800C4FF4807C96
:1013400003FB0CF34FEA432C0CF1FF3C0CEA0101C8
:10135000A3EB5123CEE72B7E1A072CD59BF8002058
:101360002B4B032A95F828201B680CBF80214FF4D3
:101370008071062A03FB01F34FEA43233FF47CAF5D
:1013800024490868834231D891F83D30002B7FF41E
:1013900073AF002A7FF470AF06216B69284685F889
:1013A000382085F82810EB62FFF706FD1AE0FFF7FA
:1013B0005BF80198AFE795F82830002B7FF45CAF1D
:1013C000154B1A78002A7FF457AF082185F834208E
:1013D0006A69284685F82810D3F85F30C5E90B23E1
:1013E000FFF7B0FE01283FF46FAF45E741F2E57328
:1013F000012250460BF8032003B0BDE8F08F92465F
:101400003AE700BFF44F0120A067012000FEFFFF74
:101410001C68012084670120C16701202DE9F04785
:1014200090F8384082B00546032C00F29B80DFE83C
:1014300004F00218620BFFF785FE01280FD0022886
:1014400009D1032385F8383000202B6C022485F85D
:10145000280003B19847204602B0BDE8F08785F820
:1014600038002B78022B52D03F4941F648026B6876
:101470008A5803EA0208C8F34F282846DFF8EC90A0
:10148000F7F766FB0646A8EB0008022201A93046E2
:101490000023FFF757F808EB060701284FF4007206
:1014A000BFB24FF00001044606F10106D3D1019806
:1014B0004FF02AF8EB694FF4007128460BB16B68C6
:1014C0005BB3D9F800305A1E974206D2FFF7A4F951
:1014D0000028DAD1FEF7C8FFD7E7C3EBC35328468D
:1014E000590201F50071FFF797F908B9FEF7BCFF43
:1014F000022385F8383000222B6C85F8282053B160
:10150000012428469847204602B0BDE8F0876B6862
:10151000C3F34F28B1E701249DE7019B4FF0203230
:101520002E244FF0100C1A605A601C70C3F807206C
:10153000D5F824E01A625A62CEF30F4A83F82040AD
:1015400083F82140C3F8272083F80BC0EA6BA3F887
:101550001AE0C2F30F44A3F814A05A879C8683F8BC
:101560002BC0AEE7002476E7DC4F01201C68012089
:101570002DE9F04F90F8303089B00446042B00F28A
:10158000A780DFE813F0A800B10005008900E7009C
:10159000B54D41F61003EB5C002B40F09980B34F42
:1015A00004F11C0901AEB84607F1380BBA463246C1
:1015B00049464046FFF71EFA012840F0168101987F
:1015C000002800F0F98003780BB1E52BEFD1A84A91
:1015D000821A48BF02F2FF12B2F5B05F4FEA6223EF
:1015E00080F03B811B01A34A13449A7B042A0CD050
:1015F00041F2C86641F2CC610427AA590132AA51CE
:101600005A609F736B5801336B5041F60202AB5620
:101610005E1C09D003F5B173FF2105EB0313A95438
:10162000DA796FF30002DA7141F603016B565A1C46
:101630000ED003F5B173FF2605EB0313DA796E5470
:10164000C2F34501013921EAE17161F34602DA7121
:10165000202200214EF058FF2346019A05A853F896
:10166000315F59681560516019899B7A11819372B5
:10167000019B627EDA7241F0B1FFBDF81430002B9D
:1016800040F02E8144F28172019903200A82CB81BD
:101690000A83CB8284F83000237E980600F1A8806C
:1016A0002046FFF747F92369002B00F0AD80237E29
:1016B00003F0F70213F00403227640F0B380122AFD
:1016C00000F0B9800022E36A204684F82820984779
:1016D00009B0BDE8F08F6548FFF72CF94FF6FF72AF
:1016E0000123228484F8303004F11C0801AE5F4FDE
:1016F00004F13109324641463846FFF77BF90128AB
:101700002FD00228E4D1584D41F60202AB56591CA5
:1017100009D003F5B173FF2105EB0313A954DA795E
:101720006FF30002DA7141F603016B565F1C0ED0B5
:1017300003F5B173FF2005EB0313DA796854C2F3A4
:101740004501013921EAE17161F34602DA710423AE
:1017500084F830300020E36A2070984709B0BDE873
:10176000F08F019D0B2249462846002D00F086800F
:101770002B78002B00F0828095F80BA01AF0080F50
:10178000B8D14EF0A7FF0028B4D1637E8AEA0303E4
:10179000DB0640F1C680344D41F60202AB565F1CB9
:1017A000C1D003F5B173FF2105EB0313A954DA7916
:1017B00060F30002DA71B6E73B78092250462E4901
:1017C000022BC4D00B78002BC1D10A708BF80030EB
:1017D0004A6B0B73C1E9053351F8143CC1E901327E
:1017E000FFF71CFE01283FF4E2AE0228AFD06FE7FE
:1017F0000023112205A9E069FEF7A4FE01283FF4A9
:101800004FAF09B0BDE8F08F237E19077FF55AAFBF
:10181000154A41F2C873D15C00297FF459AF072102
:10182000D1544FE70023E26AA168204684F82830AB
:10183000FFF766F84CE7E56A0421626A204684F8FF
:101840003C306363A56384F828106362C4E9023303
:10185000C4E90B22FFF76EF83AE7FEF705FE0198A0
:101860006FF00F03BFE600BFDC4F0120C46701200B
:10187000F44F0120F4650120EC670120474D41F64B
:101880000202AB565E1C09D003F5B173FF2105EBD4
:101890000313A954DA796FF30002DA7141F60301F8
:1018A0006B56581C0ED003F5B173FF2005EB0313E4
:1018B000DA796854C2F34501013921EAE17161F333
:1018C0004602DA71237EDA067FF541AF3448FFF72E
:1018D00031F84FF6FF720223228484F8303058E644
:1018E000304B05A902A8B3F9442041F0CDFE9DF884
:1018F0000C309DF80D00DB029DF80A509DF80B207E
:10190000BDF8081043EA401342EA45129DF80E0064
:10191000A1F2BC7143EA500342EA41229BB292B267
:10192000B2E6A98A6A8B204B42EA01421B686262D6
:101930005A02EB69B3FBF2F102FB1131A36009B16A
:1019400013445B1A154D41F60202E36084F819A0B6
:10195000AB565E1C09D003F5B173FF2105EB0313F1
:10196000A954DA796FF30002DA7141F603016B567C
:10197000581C0ED003F5B173FF2005EB0313DA7981
:101980006854C2F34501013921EAE17161F346026D
:10199000DA71032384F830307EE600BFDC4F01208B
:1019A000C4670120D84C01201C6801202DE9F041BA
:1019B00090F8283084B00446013B082B41D8DFE87A
:1019C00003F048054D525865406A4300394B41F6D3
:1019D000480241689F5803F5C253056B0F401B68CE
:1019E000EA194FEA4328B2EB432F16D258E0216997
:1019F000207EFEF7F3FE012823D1256B6168A5EB5D
:101A0000080522694144039B3D446261C91B23616F
:101A1000A84537466160256342D82046F7F770F83D
:101A200003AA06460028E2D06168A3680020E26AA3
:101A3000994284F8280038BF1946A1600AB12046AF
:101A4000904704B0BDE8F081FFF7E8FC04B0BDE8C2
:101A5000F081FFF78DFD04B0BDE8F081FFF774F869
:101A600004B0BDE8F0810021FFF7CAFA04B0BDE878
:101A7000F0810121FFF7C4FA0128E2D10023216C93
:101A8000204684F82830FFF7CFF8DAE7FFF794F91B
:101A900004B0BDE8F081FFF755FB04B0BDE8F0816C
:101AA00020460191F7F72CF801990028BDD129446F
:101AB0006160BAE7DC4F01202DE9F0470D46904602
:101AC0000021442204461E46089F4EF01DFD0123BE
:101AD0004FF6FF722676628384F828302B782E2BFF
:101AE00042D004F1310A04F139092E46327820231C
:101AF00010462AB12E2A03D03EF05EFA0136C3B258
:101B00000AF8013BCA45F1D130782E2801D170780E
:101B1000013604F1380904F13B0A202318B13EF0E4
:101B20004BFA0136C3B209F8013FD14507D03078EE
:101B300020230028F3D109F8013FD145F7D118F04F
:101B4000100F84F81980E76214BF03230123237068
:101B50002B782E2B24D00023204684F83030FFF73A
:101B600007FD2046BDE8F0876B78002BB9D1124BFA
:101B700041F60C0041F2F47141F2F0721E589A588D
:101B8000585841F601016662C4E9022041F2E87248
:101B9000595C61769B5CE76223702B782E2BDAD13F
:101BA0006B78002BD7D10323204684F83030FFF721
:101BB000DFFC2046BDE8F087DC4F01200121032037
:101BC00008B546F0FFFF72B644F0A8FE2DE9F04FCD
:101BD000CD4C8DB04FF00008DFF84093CB4D009016
:101BE00054F80B0C002800F0FE8035F007FA06468A
:101BF000002800F0D78159F8B83CE026A4F10B0B7F
:101C0000C34F44F8073C002306FB08F604F8033CE6
:101C100054F80B0C35F0F2F9002800F0E48054F889
:101C20000B0C35F0E3F914F8023C82465A1E0B2ADD
:101C30000DD8DFE812F01F003A0046005300830081
:101C40009B00E200150134013F0175018C0124283D
:101C50000CD0009A3AB915F87A2C824240F07D8176
:101C6000012204F8032C0D2BD2D186E0012304F8C5
:101C7000023CCDE700234D28C4F8C53084F8CD30B0
:101C800084F8CE3004D0582808D004F8023CBFE7CE
:101C9000022284F8C43004F8022CB9E7032304F8C4
:101CA000023C022384F8C430B2E704233C2804F841
:101CB000023C0BD0BAF13E0F0CD0002304F8023CDA
:101CC000A6E70A233C2804F8023CF3D1002304F8D9
:101CD000013C9DE7012304F8013C99E7D4F8C500D5
:101CE000BB19421C0344C4F8C520022A83F81FA66E
:101CF00094F8CD008AEA000184F8CD1088D12378C9
:101D0000C02BDAD86278FF2A08D1052BD5D9012358
:101D100084F8C430072304F8023C79E7A4F8C12012
:101D20000022C4F8C930934284F8C320C4F8C52007
:101D300014BF0523062304F8023C69E7D4F8C50064
:101D4000BB19421C0344C4F8C52083F81FA694F8AD
:101D5000CD00D4F8C9308AEA00019A4284F8CD1047
:101D60007FF456AF062304F8023C51E794F8CD30D7
:101D70008342A2D10D2304F8023C14F8017C002F09
:101D800040F0F280634B04AE0894ADF82C700397DA
:101D90000FCB86E80F00D4F8C930324608A9D4F832
:101DA000D10023440993B4F8C130ADF8283094F839
:101DB000C3308DF82A3001238DF82E3003AB2EF07E
:101DC000B1FB48B1049B314694F8C42058460593B2
:101DD000514B04932BF0D0FB0023039E04F8023CEC
:101DE000002E40F0D78008F10108E034B8F1030F6D
:101DF0007FF4F6AE0DB0BDE8F08FD4F8C500BA1987
:101E00005146431C0244C4F8C53082F81FA694F81A
:101E1000CD2094F8CE008AEA0202019384F8CD2006
:101E200041F08EFE019B84F8CE00072B7FF4F0AECC
:101E3000B4F80530C02B3FF640AFB4F80320C4F827
:101E4000C930A4F8C120A27884F8C32000229342AC
:101E5000C4F8C52014BF0823092304F8023CD7E6C0
:101E6000014694F8CE0041F06BFE94F8CD3084F832
:101E7000CE008AEA0303D4F8C50084F8CD30BB193C
:101E8000421C0344C4F8C52083F81FA6D4F8C93007
:101E90009A427FF4BDAE092304F8023CB8E694F8F8
:101EA000CD30434084F8CD3094F8CE3083427FF477
:101EB00004AF57E7D4F8C500BA195146431C024491
:101EC000C4F8C53082F81FA694F8CE00019341F003
:101ED00037FE019B84F8CE00052B7FF499AEB4F851
:101EE0000120B4F80330A4F8C1202278C4F8C93026
:101EF00084F8C32000229342C4F8C52014BF0B23EA
:101F00000C2304F8023C83E6FF410120D84C012059
:101F1000E03B0120940D060868DB0120E82A01203F
:101F2000014694F8CE0041F00BFEBB1984F8CE00B8
:101F3000D4F8C500421C0344C4F8C52083F81FA68A
:101F4000D4F8C9309A427FF463AE0C239DE694F82E
:101F5000CE3083427FF4B1AE0CE723287FF483AE0A
:101F6000022204F8032C7EE6012F4FF0000602D077
:101F700004F8026C37E7D4F8C93008A80894234461
:101F80000993B4F8C130CDE90A66ADF828302AF0DB
:101F900001FDEDE754F80B0C2BF02EFD54F80B0C63
:101FA000B04720E714F8033C002B3FF41CAF59F86E
:101FB000B82C54F8071C521A632A7FF614AF012B71
:101FC0002ED0022B7FF40FAF54F80B3C012285F882
:101FD000590085F846206B65124A13482A65134A52
:101FE000C5E912334023C5F89C2085F85830104BC2
:101FF000C3F8642F93F8CF380E4A003B18BF012373
:1020000082F8383C3AF07EFB4FF400502EF056F93F
:1020100009483AF06DFB85F8A06085F8A160E2E61A
:10202000FFF7CCFDE93704080D970608284D01207D
:10203000E03B012014000020439706080000000048
:10204000034B93F82400003818BF0120704700BFED
:10205000F41E012003460A2201481A80704700BF7F
:102060003C0301200346202201481A80704700BF2C
:10207000480301200346202201481A80704700BF10
:10208000680301200346202201481A80704700BFE0
:102090008803012003460A2201481A80704700BFC6
:1020A000A80301200023D0F8982218461373704724
:1020B0000346222201481A80704700BFB403012062
:1020C0000346222201481A80704700BFD80301202E
:1020D0000346222201481A80704700BFFC030120FA
:1020E00003460A2201481A80704700BF20040120DD
:1020F0000346432201481A80704700BF2C04012088
:102100000346432201481A80704700BF7004012033
:102110000346432201481A80704700BFB4040120DF
:10212000D0F8943283B110B5D0F8904294F8000200
:10213000FF2807D09B68214694F801229847FF2387
:1021400084F80032002010BD0020704701F00F011C
:10215000D0F8A822C1EBC10102EB810238B5D0F85A
:102160009032D0F89452D2F8144203F50371EA6821
:10217000D3F80402C3F80C429047002038BD00BFDA
:1021800008B5D0F88C325B689847002008BD00BFC6
:1021900008B5D0F88C321BB11B68984700B908BD50
:1021A000022008BD836B40221A645A6C42F004027C
:1021B0005A647047704700BF836B1A6C12F0500F5F
:1021C0001A6C20D142F4007219681A648A6812F0FD
:1021D000405F1AD19A69C2B9CA6A12F4700F02D06C
:1021E0008A68500511D44A6822F020024A601A6CAD
:1021F00022F480721A641A6CD10406D41A6C42F06C
:1022000001021A647047D20600D570479B6BDB6CE5
:10221000184700BF0022836BA3F85A20A3F852206E
:10222000704700BF836B1A6810B45C6F986F916839
:10223000090601D5212C1AD09168490601D522281A
:1022400006D0DA6F5DF8044B42F01002DA6770478F
:1022500000202024A3F85A00116821F49071116025
:10226000916821F00101916018669C67E9E70021FF
:102270002024A3F85210116821F0C00111605C679E
:10228000DAE700BF704700BF704700BFC369B3F50E
:10229000807F12D0826B002120201368A2F85A1090
:1022A000196821F480711960996821F00101996021
:1022B000996821F04001996090677047C369B3F550
:1022C000807F0CD0826B00211368A2F852109A68AC
:1022D00022F080029A601A6842F040021A60704749
:1022E000836B0121002283F83D101A77704700BFED
:1022F0000122836B83F83D20704700BF90F8BC3308
:10230000012B29D0012380F8BC330B060ED40268C0
:102310001021124B116101E0013B02D01169C90685
:10232000FAD4002380F8BC331846704701F00F013F
:102330000A4B890110B441F020010468216101E0D9
:10234000013B02D022699206FAD4002380F8BC3304
:1023500018465DF8044B704702207047400D03009B
:1023600011F0800F4FF01C0301F00F0170B432D157
:1023700003FB0103C1EBC102002400EB820203F561
:10238000FE7382F8FD41197090F8BC23012A31D008
:102390000121026880F8BC135C781D7802F50063A7
:1023A0008C422AD005F00F04DE6B02F53062A140AA
:1023B0001C4C02EB451226EA0146DE63DD6925EA84
:1023C0000141D96113681C401460002380F8BC33BC
:1023D000184670BC704703FB0103C1EBC102012426
:1023E00000EB82023C3382F83D40197090F8BC2328
:1023F000012ACDD1022070BC704705F00F01DE6BC1
:1024000002F510628C40084902EB451226EA0406E8
:10241000DE63DD6925EA0404DC611368194011609C
:10242000D3E700BF0078F3EF007833EC11F001033D
:1024300007D090F8413003F02803282B0CBF42232B
:10244000F2238A0709D590F8412002F02802282AB1
:102450000CBF43F0440343F0F4034A07016848BF4C
:1024600043F0B8030A6822EA03030B60704700BF19
:10247000C16838B5022903689A699C699A68DD6861
:102480000DD1C2F3C21282EA144212F0060206D142
:10249000816C01318164816C022907D038BD04212F
:1024A000FFF7C4FF002380F8403038BD0821826464
:1024B000D96180F8402038BD836B0022D3E90E013A
:1024C00002650A6593F84120602A02D1202283F830
:1024D000412070470023202210B5134C4363C4628F
:1024E000036380F8412080F842304B0712D5026820
:1024F000436A526A1A70436A028D013343624AB1D9
:10250000438D013A013B02859BB24385436C43F006
:10251000040343640721FFF789FF102102680023A9
:10252000D16180F8403010BD0000FFFF38B50025B4
:1025300080F8425090F84130292B04D090F8413077
:102540002A2B0BD038BD28222123012180F84120DD
:102550000363FFF76BFF80F8405038BD2822222329
:10256000022180F841200363FFF760FF80F84050AC
:1025700038BD00BF38B50025202280F8425090F8C1
:102580004130212B0AD0122380F8412002214563DB
:102590000363FFF74BFF80F8405038BD112380F8EC
:1025A0004120012145630363FFF740FF80F840505D
:1025B00038BD00207047704730B1044B93F90000DC
:1025C0000028D4BF00200120704700BF30680120E0
:1025D00008B5FFF7F1FF50B1054A537892785B00D8
:1025E00003F00203002A18BF43F001030B6008BD8B
:1025F0003068012008B5FFF7DFFF10B1014B5B68C1
:102600000B8008BD3068012070B5FFF7D5FF78B1A9
:10261000084A158965B1D6680023B3421C4607DA1B
:1026200002EB44040133248ADBB2AC42F5D30B70D5
:1026300070BD00BF3068012008B5FFF7BDFF10B1C5
:1026400000230B70137008BD0420704728B1034BA2
:1026500093F9BC01003818BF012070473C030120EA
:1026600008B5FFF7F3FF48B1064B93F9BC21012AE7
:1026700005DD93F8BF31C3F340030B6008BD0020B4
:10268000FCE700BF3C03012008B5FFF7DFFF18B1EE
:10269000024B93F8BE310B7008BD00BF3C03012014
:1026A00070B5FFF7D3FF38B10E4C94F8BF31DB079C
:1026B00003D500230B70137070BD0B4D94F9BD3121
:1026C00095F8206093FBF6F301330B7094F9BD414C
:1026D00095F8201094FBF1F301FB134301331370C1
:1026E000EAE700BF3C030120306801200320704767
:1026F0000A4A70B592F8243006255E1CB6FBF5F444
:1027000005FB146492F82550AC4205D002EBC303DC
:1027100082F82440C3E90A0170BD00BF306801207F
:10272000002230B504461046914200DC30BDA35C67
:102730000825584010F0800F4FEA400318BF83F07F
:10274000D503013DD8B2F5D10132EDE710B5D9B1CD
:102750000E4B986D814217DCB2B11B6A9A4213DCB2
:10276000013A01390A4C03FB012104F5E37084F8B6
:10277000CA110521FFF7D4FF062184F8CB0104F527
:10278000E370BDE81040B3E710BD00BF3068012022
:102790003C0301200023038083708380C380037285
:1027A000704700BF074A084992F85C300978013346
:1027B000DBB2994282F85C3002D1002382F85C30AF
:1027C000704700BF30680120800A0020F8B5784CBF
:1027D000236E83B1774B1B6893F82E305BB1764B39
:1027E00094F86420A3FB0013012A4FEA93132FD01F
:1027F000022A08D002B1F8BD704B9842FBD90123E0
:1028000084F86430F8BDA26E64329A423DD894F8E0
:102810005C3004EB031393F87C20FF2A06D00132CE
:102820006749012083F87C2081F8CC01FFF7BAFFCB
:10283000644B01221B7884F86420092BDBD1B4F8A7
:10284000FE30614A01339BB2A4F8FE305380F8BDDC
:1028500094F85C1004F170055C48002701EB8106D8
:10286000A366E566022500EB461356480A2684F85F
:102870007A7000789A70092884F87B6084F8645034
:10288000B9D10131504B1980F8BD94F87A2094F8F1
:102890007B309A42AFD104F16F0004F17805002338
:1028A00010F8011F08224B4002E0013ACBB209D0D8
:1028B00013F0800F4FEA4301F7D081F00703013A8C
:1028C000DBB2F5D18542EBD194F87910994238D139
:1028D000B4F87360012794F85C5076BA94F877C026
:1028E00004EB0511B4F87500B6B294F8783040BA2C
:1028F00081F87C2043EA0C23C1F8806094F871C011
:1029000080B294F872601BB2C1F88400032D46EACD
:102910000C2294F97000A1F88830A1F87E20284A92
:1029200081F87D0082F8CC7108D8264A12780C2AEA
:1029300029D00D2A02D1244B23F81500FFF732FFCE
:102940005DE794F85C3004EB031393F87C20FF2AD6
:1029500006D001321A49012083F87C2081F8CC018D
:10296000FFF720FF174B01221B7884F86420092B06
:102970007FF441AFB4F8FC30134A01339BB2A4F8A2
:10298000FC309380F8BD03EB83031149114A03EB3C
:102990008303897E0C48F9409B0093FBF1F382FB93
:1029A0000312DB17C3EBA20320F81530C6E700BF04
:1029B000306801206C090020D34D62103F4B4C0061
:1029C0003C030120213B0120243B0120500C00202E
:1029D000382A0120676666660A4B93F87A1093F8E6
:1029E0007B2091420DD0C0B210B493F87A20DC6EF7
:1029F000511CD2B2C9B283F87A10A0545DF8044BCE
:102A000070477047306801200E4B0F4AD3F80031F1
:102A1000B2F900055B0707D400EB8000400080B2EC
:102A200000F5C87080B27047084B094ADB6B32333F
:102A300082FB0312D817C0EBA20080B200F5C87069
:102A400080B2704730680120500C0020DC4001202B
:102A50006766666680F08003042B70B520D9412834
:102A60001ED0FD2806D0F0281DD0EF281FD002244C
:102A7000204670BD0B2004260F4D2E440024013546
:102A8000FFF7E8FF2044AE42C4B2F1D015F8010BC5
:102A9000FFF7E0FF2044AE42C4B2F7D1204670BD3C
:102AA0000424204670BD03200526044DE5E70C20D4
:102AB0000626034DE1E700BFCC120608D012060837
:102AC000C41206080C4AD2F81831F0B41C6800276A
:102AD000D2F810614FF6F6751981611C9F81C3E928
:102AE00000162070D2F81831D2F810111A689D81A2
:102AF000C3E90012F0BC70473068012070B5D0F80F
:102B0000A052044695F8183213B9D5F814323BB9DF
:102B100081212046FCF746FE6B7A022B07D070BD60
:102B20006B7A002BF4D10121FCF73CFEF0E705F5B0
:102B3000037220461F230121BDE87040FCF7ACBDA5
:102B400038B5044600250121D0F8A802FFF708FC9B
:102B50008121D4F8A802C4F85851FFF701FCD4F839
:102B6000A002E5624DF0A0FC2846C4F8A05238BD92
:102B700038B504468321D0F8A8020025FFF7F0FB02
:102B8000D4F89802656518B14DF08EFCC4F89852DF
:102B9000002038BD38B5044600258121D0F8A802B0
:102BA000FFF7DEFB0121D4F8A802E562FFF7D8FBAE
:102BB000D4F8A8028221C4F85851FFF7D1FBD4F809
:102BC000903225644BB1D4F894325B689847D4F8BE
:102BD00090024DF069FCC4F89052002038BD00BF4F
:102BE00070B5037C044601259BBB4FF400730222A1
:102BF0002946FCF73DFE4FF40073C4F858510222F9
:102C000081212046FCF734FEE5624FF41B704DF045
:102C100043FC0546C4F8A00220B30026D4F8A43231
:102C200006813046A5F85C621B6898470121D4F8FC
:102C3000A802FFF763FB8121D4F8A802FFF75EFB2F
:102C400005F5037220461F230121FCF725FD3046C0
:102C500070BD402302222946FCF70AFE4023C4F837
:102C60005851CCE7022070BD10B508230322832100
:102C70000446FCF7FDFD0123102063654DF00CFCBC
:102C8000C4F8980218B103460020187310BD022042
:102C900010BD00BF2DE9F041037C04460125BBBBFC
:102CA0004FF4007302228121FCF7E2FD29464FF424
:102CB000007302222046E562FCF7DAFDC4F85851A1
:102CC0004FF001080823032282212046FCF7D0FDA3
:102CD0004FF40770C4F840804DF0DEFB0546C4F8A1
:102CE000900258B3D4F8943200271B689847267C8A
:102CF000C5F814724146D5F804222046C5F818726A
:102D0000AEB140233E46FCF7C7FC3046BDE8F0813B
:102D1000402302228121FCF7ABFD294640230222F9
:102D20002046E562FCF7A4FDC4F85851C8E74FF40B
:102D30000073FCF7B1FC3046BDE8F0814646E4E79D
:102D4000134B002210B483F81E11090A0F2483F8D4
:102D50001D0183F81F1103F58E700121C3F8202196
:102D6000C3F82421C3F8282183F81C4110F8014F2F
:102D7000013122440E29D2B2F8D183F82A2110223F
:102D80000449D3F82C015DF8044B34F007B900BFB7
:102D9000306801204C690120054B002183F8301177
:102DA000C3F83411D3F82C3103B1C9E7704700BF21
:102DB0003068012013B50446FFF748FCF8B1002342
:102DC0000DF106022046ADF8063010F0F9FEB0B164
:102DD0000C4C9DF8062094F9BC1184F8D1210329EC
:102DE00003D162F07F0284F8D12105210648FFF764
:102DF00097FC062184F8D2010348FFF779FC02B062
:102E000010BD00BF3C030120090501202DE9F84F4A
:102E10001B4C05461E2094F838A194F839B194F85B
:102E20003A61B4F83C91B4F83E8194F8407122F0D4
:102E3000DBFB30B1B8F1000F03D0C14601264FF0E3
:102E4000000A94F84231DA070AD494F847213AB9D3
:102E5000012F12D0022F03D113F0020F08BF012659
:102E6000284685F800A085F801B0AE70A5F804905A
:102E7000A5F806802F72BDE8F88F3E46F0E700BF48
:102E8000306801202DE9F84F2DED028BFFF7DEFBB6
:102E9000002844D0264B93F9BC0101283FDD93F86C
:102EA000D3411546DFF890808E1E02EB44099FED5A
:102EB000218A0FF2740BDBE900AB4D4504D12046AB
:102EC000BDEC028BBDE8F88F38F8027B07EE907AF4
:102ED00026F8027FF8EEE77A67EE887A17EE900A16
:102EE00049F0CCFA52465B4649F020FB41EC100B0E
:102EF0004DF02AF851EC100B49F040FE0E2F80B235
:102F00000AD919303223B0FBF3F080B200EB800015
:102F100000EB8000400080B225F8020BCDE70024D2
:102F2000CDE700BFAFF300801655B5BBB16B0240D3
:102F30003C030120CDCCCC3D9C69012038B50D4629
:102F4000FFF784FB044638B10C4890F8BF31DB072B
:102F500004D5B0F8C0012880204638BD084A00F5E5
:102F6000EA7010F9173C92F8202093FBF2F102FB73
:102F700011320131013210F037FEECE73C03012041
:102F80003068012038B5134C94F8253094F824208B
:102F90009A4219D004EBC3030F49D3E90A20002356
:102FA000984212DC93780D4A5B08C4F87C011370D8
:102FB000FCF746FA94F8253006210133B3FBF1F211
:102FC00001FB123384F8253038BDD55C013301F89C
:102FD000015BE5E730680120DC4C01200A4D01204F
:102FE000A94B1B782DE9F04F81468BB0002B40F0A8
:102FF000B380A64DD5F88061002E00F0AD80A44AC4
:10300000D2F8D84104F0F021B1F1E02F6DD1C2F82F
:10301000D831D5F88421944267D004930DF110087B
:10302000C8F80430A8F80830B5F83C3195F838E114
:10303000ADF8143095F839C195F8403195F83AA1BA
:103040008DF8183007AB8DF810E08DF811C08DF8B1
:1030500012A0904FC5F8844198E8070003C31A8076
:10306000C4F34253C4F303423B440132597C8E45BE
:1030700001D1944508D030468DF81C108DF81D20E4
:1030800010F0B2FDADF82000304604F0070B10F050
:10309000E1FF032834D0042835D000239A4501A944
:1030A000304618BF8DF81E3010F018FE48B1019B55
:1030B000C4F3001103F001038B4202D0304610F03C
:1030C000BBFE0A2207A940464DF0F6F968B19DF80B
:1030D0001E30BDF81C2085F83A31BDF82030A5F827
:1030E0003821A5F83C313CF025FA95F888A104AFC9
:1030F00095F88831032B79D8DFE803F0083174A103
:103100005F44BB7DCAE75F44BB7FC7E739463046B3
:1031100010F0EAFD044658B107A8FFF777FE9DF8C6
:103120001E109DF810308B4260D0304610F0FAFE31
:1031300095F88831013303F0030385F888310CB921
:103140009A45D5D195F84231DB0700D524B13368D3
:10315000494630461B6898470BB0BDE8F08F01A880
:10316000FFF754FE95F842819DF8044008F00108ED
:10317000ECB1B8F1000F39D13A460DF103013046F8
:1031800010F0B5FD044688B307A8FFF73FFE9DF891
:103190001C109DF803309DF81D208B4203D19DF833
:1031A0001030934222D0304610F0C6FEC0E7B8F18E
:1031B000000FBDD13946304610F093FD0446A8B14A
:1031C00007A8FFF723FEBDF82010BDF810308B4292
:1031D0000CD085F88981304685F88A8133689B69EF
:1031E0009847A5E795F84231D80701D500249FE715
:1031F00007A9304610F072FD04460028F6D01E20C4
:1032000022F0F2F995F88B3180468342EED085F8B2
:103210008B0160B1B5F83E31002BE7D1079BD90790
:10322000E4D401213046444610F006FE80E7079BB7
:10323000DA07DBD50146304610F0FEFD78E7384668
:10324000FFF7E4FD07AB97E8070003C31A809DF87A
:1032500010309BB10DF11D0207A9304610F047FD5B
:103260000DF11E01304610F03FFD0A2207A9384635
:103270004DF022F9041E18BF012459E708A9304671
:1032800010F02FFDECE700BF1E4D0120306801203B
:103290003C030120C4120608FD292DE9F041044633
:1032A00084B000F0D980F02900F0BD80EF2900F053
:1032B0002B814AB10346861803AD002003F8010BA9
:1032C000B34205F8010BF9D19A4B0B2003F1090524
:1032D00001E013F8010F814200F0C380AB42F8D146
:1032E0004B1E832B00F29380DFE813F01D013201A7
:1032F0003C014701B401840051015C016801910067
:1033000091006E016E016E018401840184016801E7
:10331000910091008E019601910091009100910021
:103320009100910091009100910091009100910015
:103330009100910091009100910091009100910005
:1033400091009100910091009100910091009100F5
:1033500091009100910091009100910091009100E5
:10336000910091009100910091009100AA019100BB
:1033700091009100910091009100910091009100C5
:1033800091009100910091009100910091009100B5
:1033900091009100910091009100910091009100A5
:1033A0009100910091009100910091009100910095
:1033B0009100910091009100910091009100910085
:1033C0009100910091009100910091009100910075
:1033D0009100910091009100910091009100910065
:1033E0009100910091009100910091009100910055
:1033F00019011901504BB3F8DC11002900F05C8170
:10340000019229F051FE019A80B2ADF80C003AB158
:1034100003AB224413F8011B04F8011BA242F9D1AB
:1034200004B0BDE8F08103214FF00508434FB844D4
:103430000025013701E017F8011B0846FFF70AFBDA
:10344000064660193246FFF727FF7019B845C5B226
:10345000F1D104B0BDE8F0810B214FF00408384FE2
:10346000E5E7354BD3F8000180060CD4002AD7D00D
:1034700003AB224413F8011B04F8011B9442F9D159
:1034800004B0BDE8F08193F88C01870741D52D4D3C
:10349000287D052834BF02260326142916D97C3935
:1034A000C8B20628E2D80629E0D801A050F821F0D9
:1034B000A3360108A33601088D3601086D340108D2
:1034C00079360108733601087F3601080929CDD9FC
:1034D0000A390A29CAD801A757F821F0613601082C
:1034E000AD3601086D3401086D3401086D340108F2
:1034F0006D3401086D3401086D3401086D34010824
:1035000085360108A33601080C214FF006080E4F3E
:103510008DE70C4B0B29187DA8D10126C7E00B4B7A
:103520009B6B039373E70192FFF76EFA019AADF874
:103530000C006CE7EC12060830680120D012060877
:10354000CC120608F04B0120C4120608DC40012012
:103550006A4BD3ED737AFDEEE77A17EE903AADF849
:103560000C3054E7654B93F8A301B3F89011002891
:1035700040F0AA80ADF80C1049E76049B1F89031ED
:1035800091F8BC11B3FBF1F3ADF80C303FE75B4DA4
:1035900095F84231DE0700F19C80B5F8DC31ADF8DA
:1035A0000C3034E7564B5749B3F9043081FB030123
:1035B000DB17C3EBA103ADF80C3028E74F4BB3F892
:1035C000F831ADF80C3022E70C394F4B9FED4F7AB4
:1035D000C9B2D3ED007A03EB810367EE877A93EDEE
:1035E000157A67EE877AFDEEE77A17EE903AADF836
:1035F0000C300CE70F39424B33F8113003EB8303E7
:103600005B00ADF80C3002E73C4B93F8423103F01D
:103610000103ADF80C30FAE63D4B1988CD0551D4C5
:10362000CB4303F0010311F0440F18BF042311F042
:10363000020F18BF072311F4806F18BF0923AEE7EC
:103640000192FFF7E1F9334B019A1B6C43EAC0404A
:103650000390DCE6294BD3F8EC31ADF80C30D6E61C
:103660002B8A03EB830303EB83039B00ADF80C3041
:10367000FCE66B680393F9E62B680393F6E6AB6808
:103680000393F3E6EB89ADF80C30EFE6EB892249C2
:1036900003EBC3039B00A1FB03135B09ADF80C30E4
:1036A000E4E6B3F88E31ADF80C30DFE6F6B28DF813
:1036B0000C608DF80D00D9E6D3F8F40180F310000A
:1036C00080B2A2E60323AEE793F8BC31B1FBF3F17D
:1036D00050E7019223F09CFBD5ED737A019AFCEE42
:1036E000E77A17EE903A9BB200287FF458AF0B4967
:1036F000096811F0100F18BF002350E7306801204F
:10370000644C0120676666665411002000007A440C
:10371000884C0120DC4001201F85EB51244B012007
:1037200030B5952383B008240A0E05468DF8053080
:1037300040F040000B0C8DF80410E1408DF80000C3
:103740008DF801208DF802308DF80310F9F7CEFBCB
:10375000FF2802D0013CF9D16DB9084906230022A7
:103760000924C86D694645F097FDF9F7BFFBFF28AE
:1037700002D1013CF9D1FF2003B030BDF41E01207D
:1037800010B5084CE26D936813F4C05FFBD19368E9
:103790001B06F8D40A2032F043FA606EBDE81040F0
:1037A00036F01EBDF41E0120014B1B681B6A184732
:1037B00094410120024B186808B18369184770478B
:1037C00094410120024B186808B1436918477047BB
:1037D0009441012010B5074C606D40B137F0D0FA2C
:1037E00094F8513013B180F00100C0B210BD012037
:1037F00010BD00BFF41E012010B5FFF7EBFF0E4C0B
:1038000048B194F82430032B10D8237E0133DBB267
:10381000072B237603D9002384F8243010BD074BEF
:1038200001221B6884F82420636110BD4FF480716D
:10383000E06D43F06BFAE8E7F41E0120302A012026
:10384000002807DB00F01F0101234009024A8B40DA
:1038500042F82030704700BF00E100E0B1F5805F22
:10386000F0B400F0D4802AD8102900F0F580B1F52A
:10387000807F4ED1046A166924F4807457689A4B8D
:103880000462016A446821F40071C56941EA0621B5
:10389000964E2B40156821F48071B04245EA03052D
:1038A00041EA072173D0924B984270D0D26800232E
:1038B0004460C561C26301621846F0BC7047B1F54F
:1038C000803F00F08180B1F5801F48D1046A1569FE
:1038D00024F480145668874B0462016A446D21F415
:1038E00000112340146841EA0551804D43EA042445
:1038F00021F48011A84241EA06515DD07C4B9842E8
:103900005AD0D26800234465C26501621846F0BCF3
:103910007047012923D1046A166924F0010457680D
:10392000714B0462016A446821F0020185693143E8
:103930006E4E2B40156821F00101B04245EA0305A7
:1039400041EA07010FD06A4B98420CD0D26800239D
:1039500044608561426301621846F0BC70470123F0
:10396000F0BC18467047D2E9056321F0080124F441
:10397000807441EA86011C439668D36921F00401F2
:1039800024F4007441EA860144EA4304DEE7D2E904
:10399000056321F4006124F4805441EA862196688D
:1039A00044EA0314D36921F4806124F4005441EA09
:1039B000862144EA431479E74368956923F4802318
:1039C00043EA852343609CE7046A156924F4803444
:1039D0005668494B0462016A446D21F4003123406A
:1039E000146841EA0541414D1C4321F48031A8424D
:1039F00041EA064155D03E4B984252D0D26800234E
:103A00004465846D826501621846F0BC7047046AA3
:103A1000166924F480545768384B0462016A45687B
:103A200021F40051C46941EA0631304E2340146844
:103A300021F48051B04243EA042441EA073138D0EE
:103A40002B4B984235D0D26800234560C461026494
:103A500001621846F0BC7047046A166924F010042D
:103A60005768264B0462016A446821F02001856989
:103A700041EA06111D4E2B40156821F01001B0429D
:103A800043EA052541EA071119D0194B984216D08F
:103A9000D268002344608561826301621846F0BCED
:103AA00070474368956923F4803343EA05234360F4
:103AB000A4E725F48045936945EA8315C3E7D2E975
:103AC000056321F0800124F4806441EA8611966840
:103AD00044EA8304D36921F0400124F4006441EAFC
:103AE000861144EAC304D3E78CFFFEFF00000140C7
:103AF00000040140FF8FFFFE8FFFFEFFFF8CFFFEE3
:103B000070B4344CB0F1804F0368A0EB0404B4FAF5
:103B100084F44FEA541406D02CB92F4D2F4A90420A
:103B200018BFA8421DD12E4A23F070034D68821A97
:103B30002B43B2FA82F2520923F44073D1E90265B1
:103B40002B430D880360C66285623CB932B9436974
:103B500043F0010370BC4361002070470B7C03639A
:103B6000F5E702F58062904220D002F5784290425B
:103B70001CD01C4A1C4DA84218BF90420CBF012209
:103B8000002224D0194EA5F59635A84218BFB042A0
:103B9000D2D0174A90421AD002F58062904216D0D5
:103BA0008C680A880360C4628262D0E70C4A23F002
:103BB0007003104D821A4E68A842B2FA82F243EAAC
:103BC00006034FEA5212B7D0002AB5D1D1E700223E
:103BD000B2E700BF000001400004004000080040C0
:103BE0000004014000400140004401400048014001
:103BF000001C0040000C00402DE9F04F002383B072
:103C0000DFF810820D68DFF810E203E00133102BBB
:103C100000F0B88001229A4032EA050405EA020C5D
:103C2000F4D14C6824F01007022F40F0AE80DF087A
:103C300003F0070A4FF00F0B0E6900EB87074FEAFE
:103C40008A0AD7F820900BFA0AFB06FA0AF64FEA1E
:103C5000430A29EA0B094FF0030B46EA09090BFA5C
:103C60000AF604EA0B0BC7F820906FEA060907680A
:103C70000BFA0AFB27EA06064BEA06060660876887
:103C8000C4F3001607EA090BCF689E4007FA0AF74B
:103C900047EA0B078760476827EA02021643466037
:103CA000C668E7008A6806EA090902FA0AF242EAE7
:103CB0000902C260AAD5D8F8447023F0030903F0C2
:103CC00003020F2647F4804709F180499200C8F8A3
:103CD000447009F59C39D8F8447006FA02FA07F4E2
:103CE00080470197444F019EB842D9F8086026EA00
:103CF0000A061AD007F58067B8425ED03F4FB84237
:103D000060D03F4FB84262D03E4FB84264D03E4F81
:103D1000B84266D03D4FB84268D03D4FB8420CBF64
:103D20000727082707FA02F21643C9F808606FEA66
:103D30000C07DEF80020E60303F1010354BF3A400C
:103D40004CEA0202CEF80020A203DEF8046054BF61
:103D50003E404CEA0606E202CEF80460DEF8086057
:103D600054BF3E404CEA0606A402CEF80860DEF8D6
:103D70000C2054BF3A404CEA0202102BCEF80C2023
:103D80007FF448AF03B0BDE8F08F4FEA430A4FF02D
:103D90000309D0F800B0013F04EA090609FA0AF95C
:103DA000012F2BEA090B06FA0AF66FEA090946EA1F
:103DB0000B0606603FF674AF61E7012707FA02F2CF
:103DC0001643B2E7022707FA02F21643ADE70327CC
:103DD00007FA02F21643A8E7042707FA02F216438D
:103DE000A3E7052707FA02F216439EE7062707FA1C
:103DF00002F2164399E700BF0000024000080240AB
:103E0000000C024000100240001402400018024062
:103E1000001C024000380240003C014030B4002346
:103E2000154C0168C36725680B681B0709D400227D
:103E300020231446436780F870208367204630BCF7
:103E40007047CB6913F40013F1D12268521BB2F111
:103E5000007FF6D30A682025032422F4D0720A607A
:103E60008A6822F001028A60456780F870308567B1
:103E7000204630BC704700BF4C350120436ADA074A
:103E800010B406D50168846A4A6822F400322243DD
:103E90004A609C0706D50168C46A4A6822F48032E9
:103EA00022434A60590706D50168046B4A6822F428
:103EB000802222434A601A0706D50168446B4A688B
:103EC00022F4004222434A60DC0606D50168846B76
:103ED0008A6822F4805222438A60990606D50168D6
:103EE000C46B8A6822F4005222438A605A060AD5BB
:103EF0000168046C4A68B4F5801F22F4801242EA1B
:103F000004024A600BD01B0606D50268816C536818
:103F100023F400230B4353605DF8044B70474A6859
:103F2000446C22F4C00222434A60ECE71F4BF0B419
:103F3000595C0446D2E90236451810693343566984
:103F40006758034390693343D6690343906A334308
:103F5000174E03433E40D06A3343635090B16E69BD
:103F6000176B26F00706536B3843976B3043686135
:103F7000605820F0C07018436050635823F4C003A9
:103F80003B436350566800201368EE60AB60094EF7
:103F90006B681E40D2E908321E436E60635823F0FE
:103FA000F05313436350F0BC704700BFA40D0608E4
:103FB0001F80FCFF0000FFFF30B4614C0346614AE4
:103FC000655C0C1E18BF0124821A405918BF0122DB
:103FD00020F00100585192B98CB95B4A0021212090
:103FE000116051609160D160116150615A5922F0A5
:103FF000F0525A513F2200209A6030BC704753481B
:10400000181A18BF012014B908B9514AE6E74C1E26
:1040100018BF01241ABB14BB4E4A00202124106093
:1040200050609060D060106154615A5922F0F05293
:104030005A5101290DD0022915D0032924D0042971
:1040400027D0052914D006292BD0072935D00120E7
:10405000D3E74FF47462002030BC9A60704760B9B7
:104060005CB93D4AD9E74FF47C1200209A60C4E75E
:104070004FF474620020DA60BFE78C1E18BF012481
:104080005AB954B9354AC8E74FF0746200209A60B3
:10409000B3E73F220020DA60AFE738B934B9304ADD
:1040A000BBE74FF47C120020DA60A6E7CC1E18BFF5
:1040B00001243AB934B92B4AAFE74FF074620020BB
:1040C000DA609AE710B90CB9274AA6E70C1F18BFA7
:1040D000012412B90CB9254A9FE710B90CB9244A3A
:1040E0009BE74C1F18BF012412B90CB9214A94E771
:1040F00010B90CB9204A90E78C1F18BF012412B9DF
:104100000CB91E4A89E710B90CB91D4A85E70D4A5A
:10411000934203D1072901D11A4A7EE71A4A0020A7
:104120002124106050609060D060106154615A5931
:1041300022F0F0525A5100297FF47BAF5AE700BFBA
:10414000A40D0608006002401060024000640240B6
:10415000106402402860024028640240406002402F
:10416000406402405860024058640240706002405F
:10417000706402408860024088640240A06002408F
:10418000A0640240B8600240B8640240034A0130B3
:10419000116813685B1A8342FBD370474C350120CA
:1041A00003682DE9F04F13F0010785B000F0F080AF
:1041B000C44A13F40025916821F400019160C46A97
:1041C0009168B4FA84FE41EA04014FEA5E1E9160F0
:1041D00000F0E380BB49446BD1F88C20B4F5801F1C
:1041E00022F4401242EA0402C1F88C2000F0B681A9
:1041F000B4FA84F413F480124FEA5414019240F09C
:10420000D280990600F1E480DE060CD5AD49D1F8E4
:104210008C2022F08072C1F88C20D1F88C20066BA3
:104220003243C1F88C20590408D5A649C66DD1F88F
:10423000902022F440323243C1F890201A0408D56D
:10424000A049066ED1F8902022F440223243C1F8F2
:104250009020DE0308D59B49466ED1F8902022F4C9
:1042600040123243C1F89020590608D59549C66BD3
:10427000D1F8902022F003023243C1F890201A06B0
:1042800008D59049066CD1F8902022F00C023243F8
:10429000C1F89020DE0508D58A49466CD1F89020F7
:1042A00022F030023243C1F89020990508D58549A3
:1042B000866CD1F8902022F0C0023243C1F89020E1
:1042C0005A0508D57F49C66CD1F8902022F4407277
:1042D0003243C1F890201E0508D57A49066DD1F801
:1042E000902022F440623243C1F89020D90408D5CE
:1042F0007449466DD1F8902022F440523243C1F8FF
:1043000090209A0408D56F49866DD1F8902022F448
:1043100040423243C1F8902013F4001C0ED069498A
:10432000D0F87480D1F89020B8F1006F22F00062CC
:1043300008BF012442EA0802C1F890205E0309D5B3
:10434000DFF88081C26ED8F8901021F040710A43E6
:10435000C8F89020190209D5DFF86881826FD8F873
:10436000901021F080510A43C8F890205A0100F1C2
:104370008E80B3F1007F00F09980BEF1000F40F015
:104380009580012C00F0F180002005B0BDE8F08F91
:1043900013F40025BE467FF41DAF2C4613F48012A3
:1043A00001923FF42EAFDFF81CC1816BDCF88C204A
:1043B000B1F5800F22F4400242EA0102CCF88C20D1
:1043C00000F0D080002908BF012499067FF51CAFBA
:1043D000DFF8F0803C4AD8F840903C49944649F0D8
:1043E0008059C8F84090D8F8408008F08058CDF83F
:1043F0000C80DDF80C80D2F8008048F48078C2F898
:104400000080D1F8008005E00A68A2EB0802642A67
:1044100000F2A080DCF80020D205F5D5DFF8A480FA
:10442000D8F8702012F4407C826A02F4407919D0E6
:10443000E14517D0D8F870C0D8F870A02CF4407CB3
:104440004AF4803AC8F870A0D8F870A02AF4803AEC
:10445000C8F870A0C8F870C0D8F870C01CF0010F80
:1044600040F00581B9F5407F00F0EE80DFF854C0E0
:10447000DCF8081021F4F811CCF808101149C2F347
:104480000B02D1F870C042EA0C020A67BCE6DFF802
:104490003480B3F1007FC26FD8F8901021F0005142
:1044A00042EA0102C8F890207FF467AF054A074945
:1044B000D2F80080964628F08068C2F80080D1F8D3
:1044C00000800AE000380240007000404C350120B6
:1044D0000A68A2EB0802642A3CD8DEF80020160124
:1044E000F6D46FB1C26A5AB98268DEF88470466841
:1044F000120707F0706742EA86123A43CEF884202A
:10450000002D40F08380019A22B1826BB2F5800FBA
:1045100000F081809A010AD5C36842681B0687684B
:1045200043EA82135B4A43EA0773C2F88430594B6B
:104530001F681A4647F080671F600F6803E00B682A
:10454000DB1B642B06D813681B01F8D5012C7FF404
:104550001BAF0AE0032005B0BDE8F08F00244FF048
:10456000010E1BE74FF0010E4BE64A4B4A491C680F
:104570001A4624F080541C600C6803E00B681B1B77
:10458000642BE7D813689E00F8D4002D6BD1019BF3
:10459000C3B1836BB3B93F4A4369D2F88840056918
:1045A0001B0604F4403443EA85132343C2F88830E1
:1045B000D2F88C30046A23F4F853013C43EA042314
:1045C000C2F88C30BCF1000F10D0436FB3F1006F14
:1045D0000CD183692F4C00691B04D4F8882043EA6E
:1045E000801302F070621343C4F88830294B1868B6
:1045F0001A4640F080501860086803E00B681B1AE8
:10460000642BA7D813689B00F8D5BDE6426BB2F5C2
:10461000801F7FF478AFDFF87CE0C268DEF884703A
:104620004668120607F0E04842EA861242EA0802AB
:10463000CEF88420DEF88C70C26927F01F07013A9B
:104640003A43CEF88C2065E7DFF84880DFF84CC0AD
:10465000D8F8081002EA0C0C21F4F81141EA0C0118
:10466000C8F808100AE7436B002B94D08FE7D1F805
:1046700000B041F2883A06E0D1F800C0ACEB0B0C78
:10468000D4453FF667AFD8F870C01CF0020FF3D0E6
:10469000E8E600BF003802404C350120FFFCFF0F68
:1046A0000B4B01E0013B10D00269002AFADA0369E2
:1046B000074A43F00103036101E0013A05D00369B1
:1046C00013F00103F9D1184670470320704700BF6B
:1046D000400D0300144B10B4046C9C421AD800F532
:1046E0003060002301290361036943F4002303615F
:1046F000036943F018030361036943F0C043036196
:1047000004D14261036843F08023036000205DF818
:10471000044B7047D0F8003B00F53060002BE0DA26
:1047200000205DF8044B70470A30544F4B78012B42
:10473000F0B50D7826D000F53060404C404B00EBD2
:1047400045104D69066934400461046923400361E2
:104750008B6805B14B610469C3F31203012A44F469
:1047600000240461046943EA0403036105D003687B
:1047700043F0044303600020F0BDCB68002BF6D06B
:104780004361F4E74B6993B300F510642B4FD1F804
:1047900008C004EB45142A4E6345D4F810E00EEA35
:1047A00007072761276906EA07062661266938D9BF
:1047B00046F40026C1F814C0CCF31203012A266186
:1047C000266943EA0603236126D0BCF1000F08D016
:1047D00005F00F020125D0F8343895401D43C0F88C
:1047E00034582368002043F004432360F0BD00F5F3
:1047F0001060134EA3F50023012A00EB4514206935
:1048000006EA00062661206940F400202061206944
:1048100003EA00032361E4D10B69002BE1D063615B
:10482000DFE746F40026C3F31203012A2661266956
:1048300043EA06032361CBD1EEE700BF0000F8FF97
:10484000FFFF07E02DE9F0434D780F78012D4DD0A3
:1048500000F530636F4E4C6903EB47136E4D1F69D3
:104860003E401E611E6935401D616CB38D68012A92
:104870006A4E2C441F6904F1FF34B4FBF5F41FFAAF
:1048800084FC06EAC44405FB0CF544EA0704C5F3BE
:1048900012051C611C6945EA04051D6121D0CA7816
:1048A000012A0AD1D0F8082812F4807F1A680CBFB8
:1048B00042F0005242F080521A601A6842F00442FC
:1048C0001A600020BDE8F0838C68012A1D69C4F3DA
:1048D000120444EA05041C611C6944F400241C61B0
:1048E000DDD1CA68002ADAD05A61D8E74B6900F5F1
:1048F0001064002B37D104EB4714474E454D012A75
:10490000D4F810C00CEA06062661266946F4002693
:104910002661266905EA06052561CE7872D0012E4A
:1049200059D1D0F8085815F4807F25680CBF45F0A0
:10493000005545F080552560256845F00445256003
:10494000002ABED19BB203339C08BAD0CA6800F5D6
:10495000805302EB840403EB073352F8041BA2429A
:104960001960FAD1ADE704EB4714D1F808E0DFF89D
:10497000A490C3F31206D4F8108003EB0E0C08EADF
:1049800009090CF1FF3CDFF89080C4F81090D4F8CE
:104990001090BCFBFEFE09EA0808DFF880C0C4F8EE
:1049A00010800CEACE4CD4F810E04CEA0E0CC4F89F
:1049B00010C0D4F810C046EA0C062661CE78012E4D
:1049C00010D0012A22D007F00F03D0F834789D4090
:1049D0003D43C0F834582368002043F0044323606B
:1049E000BDE8F0832569012A25F0C04525612569C8
:1049F00045F00055256194D10D69002D91D01646E2
:104A000065618CE70D69002D89D0F9E70D69002DEE
:104A1000F6D1E0E70000F8FFFFFF07E00000F81F15
:104A200001F01F01036A10B401248A408C4023EA7C
:104A300004035DF8044B0362016A0A430262704793
:104A4000034690F83C00012800F0C6800220F0B434
:104A5000012483F83D0083F83C40002A31D0042A29
:104A600073D0082A1A6800F09580166AC86826F480
:104A700080560D684F688C68010316622D03D0695B
:104A800089B2166A05F4204520F4407026F42046C9
:104A900040EA0720354320F470400143D16115629C
:104AA000D06920F44060D061D16941EA0421D1612C
:104AB00000220121104683F83D1083F83C20F0BC11
:104AC00070471A68DFF814C1166A62450C6826F050
:104AD00001064D68C86816629769166A1DD0B2F162
:104AE000804F1AD0ACF57C4C624516D00CF5806C2A
:104AF000624512D00CF5806C62450ED00CF5784CF6
:104B000062450AD00CF5705C624506D0ACF5943C69
:104B1000624502D047F0010502E027F003073D435C
:104B2000000125F0F00526F00A0604F00A04C0B2E0
:104B30008F683443284390611462906920F00C0020
:104B40009061916939439161B2E71A68C868166A41
:104B50000D6826F010064F688C68010316622D015F
:104B6000906989B2166A05F0A00520F4407026F01D
:104B7000A00640EA0720354320F4704001439161CC
:104B80001562906920F440609061916941EA0421C6
:104B900091618DE7176AC86827F480770E684C68C2
:104BA0008D68010117623602D069C9B2176A06F42E
:104BB000206620F0030027F4206720433E4320F0C6
:104BC000F0000143D1611662D06920F00C00D06181
:104BD000D1692943D1616BE7022070470000014091
:104BE000F0B490F83D30002B66D0026802233B49B8
:104BF000B2F1804F80F83D30A2EB01011368B1FAA9
:104C000081F14FEA51113BD0002939D1344D354C57
:104C1000A24218BFAA4233D0334F05F50065D71B17
:104C2000AA42B7FA87F74FEA57174AD0002F48D160
:104C30002E4F2F4CA24218BFBA420CBF01270027AB
:104C40004AD02C4DA4F59634A24218BFAA4220D0D7
:104C500004F58064A2423FD004F58064A2423BD0B8
:104C6000816923F08003C4680B4341681360D462F8
:104C700091620123536180F83D300020F0BC704701
:104C8000194F23F070038568D71B2B43B7FA87F7BA
:104C90007F09046923F4407385692343C668446827
:104CA00023F080032B431360D662946209B9002F6E
:104CB000DFD043691363DCE703F0FF0280F83C2098
:104CC00093E70D4C23F070038568A24243EA050385
:104CD000DFD0002FDDD1ABE70027DAE7000001408D
:104CE0000004004000080040000401400040014072
:104CF0000044014000480140000C0040F8B501F0BC
:104D00000F05012600271C21C5EBC50401FB050189
:104D100000EB84043C31A264236584F83C50676551
:104D200084F83D600369B34208BFE264DAB2006808
:104D30001DB9FFF7FBFC0020F8BDFFF783FD002045
:104D4000F8BD00BF2DE9F0410A46D0F8A052002777
:104D50000B4E044685F838222F7205F50B720D2391
:104D60008121C5F82C62D0F8A802FFF7C7FF05F52E
:104D7000037220461F230121BDE8F041FAF78CBCE5
:104D8000555342532DE9F047137882B091460446BB
:104D90008A465A2B5CD8DFE813F0CE005B005B003C
:104DA0007D005B005B005B005B005B005B005B0009
:104DB0005B005B005B005B005B005B005B00B200C4
:104DC0005B005B005B005B005B005B005B00A901BC
:104DD00074005B005B0074005B005B005B005B00C9
:104DE000CD015B00F7015B005B003B015B00E00075
:104DF0005B005B005B005B0028015B005B005B000D
:104E00005B005B005B005B005B005B005B005B00CA
:104E10005B005B005B005B005B005B005B005B00BA
:104E20005B005B005B005B005B005B005B005B00AA
:104E30005B005B005B005B005B005B005B005B009A
:104E40005B005B005B005B005B005B005B001802CB
:104E5000D0F8A0120524002091F85D325A1C01EB15
:104E6000C303D2B283F83C4283F84002042A00F024
:104E700003824FF0FF3581F85D22284602B0BDE87D
:104E8000F087D0F8A032002005465881284602B0AD
:104E9000BDE8F087D0F8A042002104F10B0304F133
:104EA0001D0003F8011F8342FBD1702094F85C328F
:104EB0000C25207394F85D02E574984213D004EB3E
:104EC000C300013390F83C52DBB2A573042B90F879
:104ED0004152257690F8400218BF84F85C32607623
:104EE00008BF84F85C121223638199F80430122BF6
:104EF00098BF63810025284602B0BDE8F08799F885
:104F00000130D0F8A002DB0740F18381072100F1D6
:104F1000120300F10B0583224181C3F10604D54938
:104F200001E092F8342003F80129E218AB4211FAAB
:104F300082F2F6D1DEE7D0F8A062D6F81472002F24
:104F400040F02D82D0F8A43208469B689847054669
:104F5000002840F06D8270818FE7D0F8A062357A2A
:104F6000002D40F0908196F91832002BC0F270812C
:104F7000D0F8A43208469B6898470746002840F0BE
:104F80007182D4F8A4325046DB6898470546002861
:104F900040F08D82D9F80210D4F8A00209BAD0F8F6
:104FA0006072C6F86412B9F807305BBA9BB2194454
:104FB000C6F86832B94200F26882B6F85E12D6F8D6
:104FC000142203FB01F3934240F09E81B3F5007F6E
:104FD0004FF00101204606F10C0228BF4FF4007388
:104FE00031729BB2FAF758FB47E799F80150D0F8B5
:104FF000A03215F0020040F0F781D3F86012D3E937
:10500000992422448A4200F201820546588134E7FD
:10501000D0F8A08298F80860002E40F0328198F90C
:105020001832002B80F2CE81D0F8A43208469B685B
:1050300098470546002840F04E82D9F80200D4F87F
:10504000A06200BAD6F86072C8F86402B9F80730F6
:105050005BBA9BB21844C8F86832B84200F2F880D4
:10506000B8F85E22022003FB02F3D8F8142288F875
:1050700008009A4240F0EC80B6F85E324FF4007CB3
:10508000D6F8687206F10C05D4F8A422504607FB46
:1050900003F72946A8F80AC06745D2F81080D6F869
:1050A000642228BF6746B7FBF3F39BB2C0470028D2
:1050B000C0F25F812A463B46D4F8A8028121FFF75F
:1050C0001DFEB6F85E52D6F83432B7FBF5F5D6E9D8
:1050D0009920DF1B2A44451BC6F83472C6E999257E
:1050E000002D7FF407AF03233372C6E6D0F8A07219
:1050F000082000225F4E07F11303788107F10B05AA
:10510000C3F1070001E092F83C2003F80129C2181E
:105110009D4216FA82F2F6D1D4F8A4325046DB68EA
:10512000984700283FF4E6AEBB7B002563F07F0381
:10513000BB73A2E6D0F8A062002506F10B0306F1CE
:10514000170203F8015F9342FBD1D4F8A432504612
:105150000DF1020201A95B689847002840F0F78032
:10516000019B0821BDF802200220013BF17352BAD5
:105170000C211C0EF374F2821A0C1B0A3474727424
:10518000B374B0827181B5E6D0F8A0620846D4F855
:10519000A43206F25E2206F518715B689847054650
:1051A000002840F0C180D6F860320821B6F85E22AF
:1051B000013B308252BA7181180EF373190C72825E
:1051C0001B0A30737173B37357E6D0F8A0720820CE
:1051D0000022284E07F11303788107F10B05C3F174
:1051E000070001E092F8442003F80129C218AB42FD
:1051F00016FA82F2F6D1D4F8A4325046DB6898470A
:1052000000283FF477AEFB7B002563F07F03FB7340
:1052100033E6D4F8A44201EBC10199F80430E46903
:1052200004EB810422790532934228BF134643815F
:10523000002B3FF45FAE013B9AB2531C0C32234467
:10524000024413F8011D9C4202F80119F9D151E6FC
:1052500096F85D3205211A460133DBB206EBC20235
:10526000042B82F8405282F83C1200F0A88086F8A5
:105270005D323FE6C41206084FF0FF3581F85D024B
:10528000FBE54646F8E6B6F85E5206F10C08D6F89D
:1052900068720846D4F8A432414607FB05F7D6F8F1
:1052A0006422D3F81490B7F5007F28BF4FF400773D
:1052B000B7FBF5F39BB2C8470028C0F22781B6F8C8
:1052C0005E02D6F83432B7FBF0F1D6E99925DB1B44
:1052D0000A446D1AC6F83432C6E9992525B9204624
:1052E0002946FFF72FFDC8E505FB00F3424620469F
:1052F0000121B3F5007F4FF0000528BF4FF4007384
:105300009BB2FAF7C9F9B8E590F85D3205215A1C4D
:1053100000EBC303D2B283F8405283F83C12042A54
:105320003AD080F85D22E5E5D4F8A02202200025DD
:1053300092F85D32591C02EBC303C9B283F83C02F8
:1053400083F84052042924D082F85D12D2E5D4F8C3
:10535000A022022092F85D32591C02EBC303C9B2AD
:1053600083F8405283F83C020429EDD182F85D5263
:10537000C0E5D4F8A0220420002592F85D32591C23
:1053800002EBC303C9B283F83C0283F84052814266
:10539000DAD182F85D5270E580F85D526DE596F8DD
:1053A0005D32052100251A460133DBB206EBC2024D
:1053B000042B82F83C1282F840527FF458AF86F8F2
:1053C0005D525AE598F85D3205211A460133DBB289
:1053D00008EBC202042B82F8406282F83C1200F013
:1053E000918088F85D3285E593F85D2205200025DF
:1053F00011460132D2B203EBC101042A81F83C020A
:1054000081F840527BD083F85D2273E593F85D22EA
:10541000052411460132D2B203EBC101042A81F8FE
:10542000400281F83C42EED1054683F85D0224E556
:10543000D4F8A0220220002592F85D3219460133EB
:10544000DBB202EBC101042B81F8407281F83C020F
:1054500018BF82F85D324FF0050308BF82F85D7215
:1054600033720AE5D4F8A022022092F85D32194680
:105470000133DBB202EBC101042B81F8405281F809
:105480003C0286D082F85D3234E590F85D32052129
:105490001A460133DBB200EBC202042B82F8405201
:1054A00082F83C123FF478AF80F85D3222E5D4F800
:1054B000A022022092F85D3219460133DBB202EBE2
:1054C000C101042B81F8407281F83C02DAD13D46DB
:1054D00082F85D72D1E4D4F8A022022092F85D3205
:1054E00019460133DBB202EBC101042B81F84062A3
:1054F00081F83C02C6D1354682F85D62BDE483F88E
:105500005D52BAE4354688F85D62B6E4D4F8A0226C
:105510000420002592F85D3219460133DBB202EB1C
:10552000C101834281F83C0281F84052AAD130E7A0
:10553000D0F8A01210B50B7A022B07D0033B012B39
:1055400002D80021FFF7FEFB002010BD01F21B2254
:1055500091F819120446FFF715FC0028F4DA2046EA
:105560000121FFF7EFFBEFE7F8B5D0F8A0420546C1
:10557000267A5EB1012E07D104F21B2294F819128B
:10558000FFF700FC00282FDB0020F8BDD0F8A83280
:10559000D4F81012D3F83032D4F814221F2BC4E9F7
:1055A0008C1208D12D4BD4F80C229A4203D194F8D6
:1055B000191201291DD994F85D32002105205A1CC9
:1055C00004EBC303D2B283F83C0283F840120223F7
:1055D000042A2846637214BF84F85D2284F85D12A1
:1055E000FDF78CFA0020F8BD28460121FFF7AAFB41
:1055F000CAE794F81A32013B0F2BDCD804F21B22C5
:10560000FFF7C0FB0028237A1DDB013B022BBBD92F
:105610006189F1B1D5F8A07204F10C020420D7F829
:105620003432D7F814425B1A87F83862A1423872D4
:10563000D5F8A802C7F834320B4628BF234681218B
:10564000FFF75CFBA0E7052BCED02846FDF756FA06
:105650009AE72846FFF776FB96E700BF555342438B
:1056600070B5D0F89062E6B101EB810500EB8505DD
:10567000EB695BB1D0F8A802C1EBC10400EB840474
:10568000626CB3FBF2F402FB14341CB10020C6F8C8
:10569000140270BD23462246EC61FFF72FFB204623
:1056A00070BD022070BD00BF002310B504241A464F
:1056B0001946C0F86C42D0F8A802FFF71FFB002083
:1056C00010BD00BF70B5054641B9D0F86C320C462C
:1056D000032B10D0052B1FD0002070BDD0F88C32CA
:1056E0009B6933B190F87422032A02D198470020B5
:1056F00070BD022070BDD0E953639E4212D8D0F82D
:105700008C321B6923B190F87422032A00D1984788
:105710002846FFF7C9FFDFE7C5F86C12FAF742F831
:10572000204670BDF61AB342C0F84C6128BF33461C
:105730009BB2F9F7B1FF204670BD00BF10B513460C
:1057400002240A460021C0F86C42C0E90733D0F8B1
:10575000A802FFF7D3FA002010BD00BFF0B5002368
:1057600083B00E460446ADF806300B78D0F8A07230
:1057700013F0600522D0202D19D14A78FE2A11D0CD
:10578000FF2A14D14A8892B9CD8885B91B060ED458
:105790004FF4807107F503721F2339810121F9F756
:1057A0007BFF08E04D8815B9CE88012E73D02046C6
:1057B0000225FAF753F8284603B0F0BD4B780B2BBF
:1057C000F5D801A252F823F0075801082F58010814
:1057D000AF570108AF570108AF570108AF5701088D
:1057E000AF570108AF570108AF570108AF5701087D
:1057F0001D580108F957010890F87432032BD6D1CF
:105800008B787B60D7E790F87422032ACFD10222ED
:105810000DF106011D46FFF791FFCCE790F87432B9
:10582000032BC4D1391D0122FFF788FFC3E7097993
:10583000D0F8A802FCF762FD3179D4F8A802FCF791
:105840008FFDB38896F9042003F00F03002A4FF070
:10585000000203EB830304EB83032ADBC3F8442138
:10586000237C9BBB4FF40073022201212046F9F7F1
:10587000FFFF0123C4F85831D4F8A0727B7A022BC1
:1058800032D03279D20996D0012B94D02046012112
:10589000FFF758FA8FE71A0689D5D0F8A4329B692A
:1058A000984703463246204639463B60FFF746FF9D
:1058B00081E79A61237C83B94FF40073022281212E
:1058C0002046F9F7D5FF0123E362D5E74023022202
:1058D00001212046F9F7CCFFCBE7402302228121AA
:1058E0002046F9F7C5FFEEE720468121F9F75AFF78
:1058F00000237B725FE700BF10B50C7882B00023F5
:10590000D0F8982214F06004ADF8063016D0202CA0
:105910000ED14B78023B092B0AD8DFE803F033396C
:105920000909090909093F2F90F87432032B5AD04D
:105930000224F9F793FF204602B010BD4B780B2BE1
:10594000F6D80FF2080C5CF823F000BFD15901081B
:1059500031590108315901083159010831590108FB
:1059600031590108A7590108315901083159010875
:105970003159010829590108C35901088B780024BD
:105980001360D8E7111D01220024FFF7D7FED2E7EC
:10599000114601220024FFF7D1FECCE74B880024FA
:1059A0001B0A5360C7E74B881B0A222B1FD0212BF1
:1059B000BED1CA881149092A28BF0922FFF7BEFEB5
:1059C000B9E790F87432032BB2D18B789360B2E7C9
:1059D00090F87422032AABD102220DF106011C4675
:1059E000FFF7ACFEA7E702F108010122E6E7CA884B
:1059F0000349362A28BF3622E0E700BF50050120C0
:105A0000180501202DE9F0410A7884B000270D46E1
:105A100012F060060446D0F890328DF80D70ADF8A3
:105A20000E7016D0202E1AD1CE8806B3120643D59A
:105A300019460193D4F89432324668783E46D3F83A
:105A40000880C047019BEA8820461946FFF776FE8A
:105A500009E04B780A2B20D00B2B28D08BB12046A5
:105A60000226F9F7FBFE304604B0BDE8F081D0F81D
:105A70009432324648789B689847304604B0BDE877
:105A8000F08190F87432032B29D002262046F9F7D2
:105A9000E5FE304604B0BDE8F08190F87432032B87
:105AA000F3D101220DF10D01FFF748FEDBE790F87D
:105AB0007432032BD7D0E8E74A78032583F80162D4
:105AC000394683F800221A46C0F848613346C0F8C8
:105AD0004C613E46C0F86C52F9F7DEFDC3E7022286
:105AE0000DF10E01FFF72AFEBDE700BF2DE9F043DF
:105AF0000D784FF0010883B0044680F8805205F01D
:105B00001F0C4F7800F5207EC44580F88172CB7859
:105B10008E7806EB0326B6B2A0F882624A790B793A
:105B200003EB02239BB2A0F8843291F807908A79A4
:105B3000C0F86C8202EB092292B2A0F88622C0F86B
:105B400070220DD0BCF1020F3ED0BCF1000F19D075
:105B500005F08001F9F726FE002003B0BDE8F083D0
:105B600005F06002402A67D06A0665D5802120468C
:105B7000F9F718FE20460021F9F714FE002003B0C3
:105B8000BDE8F08305F06005202D6FD0402D6DD06D
:105B9000002DEBD1092FE9D801A151F827F000BF62
:105BA000B95C0108E75C01086D5B0108055D01084F
:105BB0006D5B0108155D0108755D01086D5B0108ED
:105BC000A15D0108815C010805F06005202D4DD024
:105BD000402D4BD0002DC9D1012FD9B200F0048146
:105BE000032F00F0EF80002FC0D190F87422022A1A
:105BF00000F0CC81032AB9D113F0800F01F00F031C
:105C000003EB830300EB830340F0D881D3F84431E6
:105C1000002BABD001F07F03142202FB030202F53C
:105C2000A072002B40F00D82002313601146204625
:105C30000222FFF783FD8FE794F87422013A022ACB
:105C400094D8DBB2032B91D8D4F88C32714620461D
:105C50009B689847B4F88632002B7FF47DAF00280C
:105C60007FF47AAF2046FFF71FFD75E7D4F88C323A
:105C7000714620469B689847002003B0BDE8F0833A
:105C8000F1B2C14D012985F8FA113FF66FAF90F8D6
:105C90007432022B00F0BE81032B00F0A981802119
:105CA000F9F780FD00212046F9F77CFD95F8FA11FF
:105CB0002046FCF765FA4FE790F87432013B022B5F
:105CC0003FF654AF022A7FF451AF0122D0F87C3264
:105CD000C2600BB10323C360022204F10C01204611
:105CE000FFF72CFD38E790F87432013B022B3FF6AA
:105CF0003DAF012E7FF430AF0023C0F87C32FFF7B8
:105D0000D3FC29E7012E7FF427AFC0F87C62FFF7B0
:105D1000CBFC21E713437FF429AF7F2E3FF626AF5C
:105D200090F87432032B3FF421AFF1B2D0F8A832CF
:105D300080F8761293F8BC23012A11D01A6800204B
:105D400083F83810D2F8001821F4FE61C2F8001868
:105D5000D2F8001841EA0611C2F8001883F8BC0313
:105D60002046FFF7A1FC002E00F07C81022384F87E
:105D70007432F1E6330A013B062B3FF6F7AE01A27F
:105D800052F823F0055F0108EB5E0108D95E0108B7
:105D90006D5B01086D5B0108C35E01087D5E010853
:105DA000012A7FF4E3AE90F87432022B00F2FF80F8
:105DB000002B3FF4DBAE0023014641F8083FFFF71C
:105DC000BDFCC9E690F87432022B00F0D380032B9F
:105DD0007FF4CCAE4F063FF445AF56EA02037FF4A2
:105DE00041AFF9F7DFFC3DE790F87422022A00F09A
:105DF000C180032A7FF4BAAE002E7FF4ADAE480610
:105E00003FF430AFD4F8A80201F00F01426891428C
:105E10003FF628AF13F0800F4FF01C0340F02681AF
:105E200003FB01020025134602F5FE7283F8FD51C3
:105E300000231170937090F8BC33012B3FF412AF24
:105E40000121036880F8BC1355781178012D0CBF2F
:105E500003F5106303F5306303EB4113196821F474
:105E600000111960D278023A012A03D81A6842F068
:105E700080521A60002380F8BC33F3E6037C002BC9
:105E80007FF474AED0F88C320DF106001B6B98478E
:105E900007234370BDF806306BB1B4F88622002AA0
:105EA0003FF4E0AE9A420146204628BF1A46ADF8BC
:105EB0000620FFF743FCB4F88632002B7FF44CAE8B
:105EC000D0E6037C002B7FF451AED0F88C320DF17C
:105ED00006005B6B9847DDE7F6B2052E3FF646AE4F
:105EE000DFE806F0302820184038037C002B40F013
:105EF0009F80D0F88C320DF106009B6A98470223F0
:105F00004370C7E7D0F888320DF10601007C1B68AA
:105F10009847BFE7D0F888320DF10601007C1B6975
:105F20009847B7E7D0F888320DF10601007CDB68AE
:105F30009847AFE7D0F888320DF10601007C9B68E6
:105F40009847A7E7D0F888320DF10601007C5B681E
:105F500098479FE7D0F888320DF10601007C9B69D5
:105F6000984797E7D0F888320DF10601007C5B690D
:105F700098478FE74D063FF4F9ADF9F713FC20463B
:105F80008021F9F70FFCE7E5306801204A067FF42D
:105F9000EDAD1B064FF000034FF002024CBF00F1C5
:105FA000140100F5A0710B60FFF7C8FBD4E5032BCB
:105FB0007FF4DCAD011DFFF7C1FBCDE59B69002B34
:105FC0003FF4D4AD01F07F035A1C02EB820200EBD8
:105FD0008202002B3FF428AED0F8A8121C2000FB50
:105FE000031393F83E30002B3AD0012313601DE6D3
:105FF00079B3416801293FF435AEC9B2FCF7C0F866
:1060000095F8FA1120466160FCF7C2F802287FF487
:1060100029AEABE500293FF425AE01210323416001
:1060200080F87432FCF7B4F802287FF41BAE9DE5CB
:10603000D0F88C320DF10600DB6A984702234370DA
:1060400028E7D0F8A8321C2000FB013393F8FE317A
:10605000C9E70223416080F87432FCF791F801E649
:106060001360E3E5012384F8743275E503FB010254
:10607000012513463C3283F83D50D9E6054A064BCC
:1060800092680649C2F382220868134493F84C30A0
:10609000D840704700380240C4120608C02C0120C6
:1060A000164908B58B6803F00C03042B1BD0082B92
:1060B00017D14A684B6802F03F02496813F4800325
:1060C00013D10F48C1F38811A1FB000146F0C6FDB2
:1060D0000A4B5B68C3F3014301335B00B0FBF3F091
:1060E00008BD074808BD074808BD0648C1F3881128
:1060F0000023A1FB000146F0B1FDE9E700380240B2
:106100000024F40000127A00F8B504468368B84908
:10611000E669E768B74DD0E904201A4323680243D3
:106120001868AB4201EA000142EA060242EA0102B3
:10613000A1691A605868226A20F4405042EA0102BC
:1061400040EA07005860996821F4306142EA010290
:106150009A605FD0A84A93421CD0A84A934200F0AC
:106160000881A74A934200F01281A64A934200F0A8
:106170008B80A54A934200F0A380A44A934200F08A
:106180005381A34A934200F0208100230120C4E9F7
:106190001833F8BD9F4BA04AD3F8903003F00C039E
:1061A000134493F85830B6F5004F17D0082BECD8AD
:1061B00001A151F823F000BFF1620108316201082A
:1061C000D76201088B610108AB6201088B6101088D
:1061D0008B6101088B61010861620108082B06D8F8
:1061E000DFE803F0BBA79E059205050589000120A5
:1061F0000023A3F110014FF6EF729142C5D823F0AE
:106200000F02C3F3420321681343CB600023C4E9A8
:106210001833F8BD7F4B804AD3F8903003F0030366
:10622000013B022B40F29C80B6F5004F00F08180CC
:1062300078497A4B89681B68C1F3423160680A4427
:1062400092F84C20D34003EB5003B3FBF0F39BB226
:10625000A3F110020DE0302B97D1B6F5004F4AD0D4
:106260006268530803F50043B3FBF2F39BB2A3F15A
:1062700010024FF6EF718A4287D822680020D3605F
:106280000023C4E91833F8BD624BD3F8903003F40F
:106290004073B3F5007F1BD066D833B3B3F5807F6E
:1062A0007FF473AFB6F5004F2ED0FFF7F9FE6368A9
:1062B00000EB5300B0FBF3F39BB2A3F11002D8E75D
:1062C000544BD3F8903003F44063B3F5006F70D1B2
:1062D000B6F5004F24D06268514B03EB5203B3FB79
:1062E000F2F39BB2A3F11002C3E7B6F5004F34D02E
:1062F000FFF7C4FEDBE762680020530803F5803334
:10630000B3FBF2F39BB274E7FFF7CAFE6168034682
:1063100000204A0802EB4303B3FBF1F39BB268E7AA
:10632000626800203F4B03EB5203B3FBF2F39BB2D6
:106330005FE738490020394B89681D68C1F3423155
:1063400066680A44730892F84C2025FA02F203EBBF
:106350004203B3FBF6F39BB24BE7FFF78FFED5E7A3
:10636000134493F854301EE7B3F5407F3FF475AF04
:106370000BE7284BD3F8903003F03003202BA7D045
:106380003FF669AF002BB0D0102B8BD0FDE6214B30
:10639000D3F8903003F0C003802B99D005D8002BA0
:1063A000A3D0402B3FF47EAFEFE6C02B3FF455AFB8
:1063B000EBE605D8D3B1B3F5806F3FF473AFE4E6F5
:1063C000B3F5406F3FF449AFDFE6124BD3F890309E
:1063D00003F44043B3F5004F3FF47AAF3BD8002BB2
:1063E00083D0B3F5804F3FF45DAFCEE60A4A1BE79A
:1063F000F369FFEF001001400044004000480040F6
:10640000004C004000500040001401400078004063
:10641000007C004000380240C4120608C02C012055
:106420000024F4000048E8010D4BD3F8903003F449
:106430004053B3F5005F3FF44BAF07D8002B3FF458
:1064400054AFB3F5805F3FF42DAF9EE6B3F5405FE8
:106450003FF403AF99E6B3F5404F3FF4FEAE94E648
:106460000038024070B41D4E056803E03468A41A79
:10647000A14226D3AB6913F02003F7D010222023CA
:10648000EA61EB61AB699A0701D50023AB62AB69A6
:10649000DB0703D4AB6943F00103AB616B680022F7
:1064A0000F4C202123406B60436C80F8402043F068
:1064B0000403436480F8411080F84220012070BC3E
:1064C0007047426C202180F840300A43426480F8D3
:1064D000411080F84230012070BC70474C350120DB
:1064E00000E800FE2DE9F041DFF8548004460E4636
:1064F00015460AE09B69DB0602D5FFF7B3FFE0B95A
:10650000D8F800305B1BB34209D823682A463146CD
:1065100020469F69BF07EDD50020BDE8F081636C80
:106520002021002201200B4384F84020636484F87A
:10653000411084F84220BDE8F0810120BDE8F081DF
:106540004C350120F0B484460568049F104E03E0EA
:106550003468E41B9C420AD8AC6931EA04000CBFE1
:10656000012400249442F3D00020F0BC7047DCF8F2
:1065700044302021002201200B438CF84020CCF82D
:1065800044308CF841108CF84220F0BC704700BFBA
:106590004C350120F0B490F841200346002A40D049
:1065A0002420DC68D3E9002183F84100012C106825
:1065B00021F0706120F0010010601161916821F4F8
:1065C00000419160996828D041F40441022C916007
:1065D00002D14FF40061516051680020134C202615
:1065E0009F690C43D3E9041554602943DC69D568DD
:1065F00041EA07211F6A25F400453C43D560D1607C
:106600001460116841F001011160586483F8416021
:10661000186383F84200F0BC704741F40041916078
:10662000DAE702F0FF0180F84010B9E700800002CD
:106630002DE9F8433C4E337D012B6DD0012380467C
:106640000F463375F5F7D4FA054600285FD14FF0B1
:10665000FF333B60D8F80030012B3DD0D8E90193DF
:106660004B444B4553D9314C2DE0022B0CBF4FF41A
:1066700000734FF44073226922F440722261226950
:1066800013432361236923F0F8032361236943EA59
:10669000C90343F002032361236943F48033236178
:1066A000BFF34F8FF5F7A4FA236923F07A03236130
:1066B000002835D1D8F8083009F10109D8F80420AC
:1066C00013444B4523D998F80C30002BD3D0012B21
:1066D000CBD14FF48073CEE7144CD8F80C3022693C
:1066E0001B0222F440729BB22261226942F0040232
:1066F00022612269134343F480332361BFF34F8F38
:10670000F5F776FA2369054623F004032361002395
:1067100028463375BDE8F88302252846BDE8F8838E
:106720000546C7F80090F2E700480120003C02400F
:10673000754B002108222DE9F0411D6882B080468A
:106740000191D0E9166334689A40224204D001686E
:106750000F68780700F18A8001229A40224204D013
:10676000D8F800104969090678D404229A402242D8
:1067700004D0D8F8001009688F0767D410229A4017
:10678000224204D0D8F800100F68380749D42022DC
:106790009A40224217D0D8F800100C68E00612D5B3
:1067A000B26098F83520052A73D00B6813F4802F57
:1067B0000B6800F09080190340F19B80D8F83C30C2
:1067C0000BB140469847D8F854303BB3D8F8543012
:1067D000DA071BD5D8F8002005214C4B88F8351076
:1067E000A3FB0535136823F00103AD0A136002E033
:1067F0001368DB0704D5019B0133AB420193F7D942
:106800000022012388F8342088F83530D8F84C303D
:1068100023B1404602B0BDE8F041184702B0BDE8E0
:10682000F081B2600A6812F4802F0A682AD1D70575
:1068300003D40A6822F008020A60D8F84020002A2F
:10684000A5D040469047D8F85C30A0E7B260D8F8B1
:10685000542042F00402C8F854208FE7B260D8F800
:10686000542042F00202C8F854207EE70F6827F057
:1068700004070F60B260D8F8542042F00102C8F853
:10688000542069E71203D8D5D8F84820002AD8D177
:106890007DE70A68D8F8404022F016020A604A698B
:1068A00022F080024A6154B30A6822F008020A60AA
:1068B0003F220024012102FA03F3D8F85020B360EC
:1068C00088F8344088F83510002AA7D0404602B036
:1068D000BDE8F041104713F480737FF46FAF0A688E
:1068E000012422F010020A6088F8343088F835401C
:1068F00064E7D8F84430002B7FF463AF63E7D8F83F
:106900004820002AD0D1D3E7C02C0120B5814E1BEE
:1069100090F835200346022A03D0802201205A65D0
:10692000704702680521002083F83510136823F0B2
:1069300001031360704700BF70B5324A002590F81C
:106940004130044680F84250283BC2624585426C83
:10695000022B41EA020141642BD80321FBF766FDBB
:106960002822294B80F8412043630563226813687D
:1069700013F4804312D01368A06B23F48043136098
:10698000B0B1224A0023026584F84030FFF7C0FF0F
:1069900070B1A06BBDE87040036D1847116811F429
:1069A000004114D194F84130602B24D084F8401079
:1069B00070BD0721FBF73AFD90F84130602B02D003
:1069C000202380F84130002323636363CEE71168FE
:1069D000E06B21F4004111600028E9D00B4A026508
:1069E00084F84030FFF794FF0028E1D0E06BBDE869
:1069F0007040036D1847202384F8401084F841301C
:106A000070BD00BF0000FFFFFD6A0108B924010846
:106A10000368202270B51E680D46DA61072104461E
:106A2000FBF704FD03683348596841F4004159609D
:106A30005A6802405A609A69910701D500229A6209
:106A40009A69D20703D49A6942F001029A617004EC
:106A50002BD5A26B1AB11268526892B262856A078E
:106A600009D55A6A25F00405636A1A70636A228D93
:106A7000013363624ABB638D9BB21BB1636C43F00D
:106A8000040363640023236384F84230666C636309
:106A900016BBE36A184DAB420DD194F84130202368
:106AA00084F8406084F8413070BD3104D7D5E26B82
:106AB000002AD0D1D3E72046FBF738FD2023E5623A
:106AC00084F8406084F8413070BD638D013A013B29
:106AD00022859BB26385CEE7616C2046FFF72CFFD1
:106AE00094F84130282BDFD129462046BDE870407C
:106AF000FBF7F0BC00E800FE0000FFFFF8B590F8DF
:106B00004030C66A012B00F0848017460123CA0674
:106B100004460D4680F8403020D5FB061ED5438D37
:106B20009BB2002B62D190F84130B6F1007FDBB20E
:106B300002D1282B00F0848094F841301021292BB9
:106B40002368D96102D116F5803F68D1AA0601D524
:106B5000BB0659D4002084F84000F8BD680710D463
:106B60002A072ED53B072CD594F8413003F0280393
:106B7000282B61D0216808200023C86184F84030A8
:106B8000E4E77907ECD5638D9BB27BB1216825F0F2
:106B90000405636A496A1970638D606A218D013B3F
:106BA00001309BB20139606263852185638D9BB2A0
:106BB000002BCBD116F5803FC8D02046FBF7B6FCA2
:106BC000C4E7A807C2D5B907C0D5638D9BB213B37C
:106BD000606A236810F8016B218D9E62638D013914
:106BE0006062013B21859BB26385AFE7036810219A
:106BF000D961436C43F00403436436F08073A5D13C
:106C0000416CFFF799FEA1E729462046FFF700FFF8
:106C1000A0E70220F8BD36F0807397D1CDE79969DF
:106C20008A0701D5002199629969CE07C5D499696F
:106C300041F001019961C0E72046FBF719FC85E7A7
:106C4000FBF748FC82E700BF38B520220368204DDF
:106C50000024DA615A682A401E4D5A600463446376
:106C6000CC06C56205D51022DA61426C42F00402FE
:106C700042649A69910701D500229A629A69D20703
:106C800003D49A6942F001029A610321FBF7CEFB1B
:106C9000436C90F84120602A0CD01A1E18BF0122C4
:106CA00043B990F84130212B08D090F84130222B85
:106CB00004D038BD416CBDE838403DE6202380F863
:106CC000402080F8413090F8423080F8422038BDB2
:106CD00000E800FE0000FFFF38B590F840300446A1
:106CE000C06A012B72D0012384F84030CB0616D540
:106CF000D50614D5D50B930B45EA9232D2072BD586
:106D0000E26B03F001035AB3ED0729D5126852680C
:106D100032BBA26B52B34BB313685B6826E00B0720
:106D200007D4880601D5930612D4002084F84000C9
:106D300038BD1507F5D594F8413003F02803282B0A
:106D400046D0236808220020DA6184F84000EFE78B
:106D50002046FFF75DFEE8E723681022DA61E4E7EA
:106D6000A26B22B31BB313685B6803BB94F841307A
:106D7000282B02D1B0F1007F2ED094F841301022A0
:106D8000292B2368DA61D0D110F5803FCDD09A69E4
:106D9000910701D500229A629A69D20703D49A69B1
:106DA00042F001029A612046FBF7C0FBBDE7236871
:106DB0001022DA61636C43F00403636430F0807383
:106DC000B3D1616C2046FFF7B7FDAEE7022038BDB6
:106DD0002046FBF74DFBA8E72046FBF77BFBA4E72B
:106DE000F8B590F84030012B7BD00123CD06044646
:106DF00080F8403023D5D00621D510222368616B5E
:106E00004548DA61626C814242F00402626466D0F5
:106E1000424A914263D0F4211A680A431A609A697F
:106E2000910701D500229A629A69D20703D49A6920
:106E300042F001029A61002084F84000F8BD0B0680
:106E400031D5570643D523681A6822F040021A60EC
:106E5000628D92B2002A46D05868618DC0F3090055
:106E60008AB2FF2A4BD8628DE56A91B215F5803F50
:106E70002185CDB24BD0E76A2D045A68284E3240A6
:106E800002433A432A435A60628D521A92B2628593
:106E900094F84120222A1A680CBF42F4004242F4BE
:106EA00080421A60C7E74D0611D550060FD5638D95
:106EB0009BB2FBB923685A689101BCD4E26A12F50F
:106EC000803F13D15A6842F480425A60B3E78B0680
:106ED000B1D59206AFD52046FFF7B6FEABE76021ED
:106EE0009AE70220F8BD5B689E0103D42046FBF7B9
:106EF00041FBA0E740212046FFF71EFD9BE7FF2254
:106F00004FF47F054FF0807711462285B5E74FF0AB
:106F100000772D04B1E700BFD96C0108E16D0108CD
:106F2000009C00FC90F84030012B00F09C80012375
:106F30002DE9F041044680F84030C8060D469046E1
:106F40001BD512F0100F18D023681021D961616C85
:106F500041F0040161649969890701D500219962B2
:106F60009969CA0764D5AB0602D518F0200F71D114
:106F7000002084F84000BDE8F0816B0712D4AF0711
:106F800024D518F0020F21D0606A236810F8016B35
:106F9000218D9E62638D01396062013B21859BB228
:106FA0006385E0E718F0040FE9D0216825F00405B7
:106FB000636A496A1970638D606A218D013B0130F3
:106FC0009BB20139606263852185CCE72E0615D41A
:106FD0006906C8D518F0400FC5D0638D9BB2002B51
:106FE00033D1236859688A01BDD4E16A11F5803F25
:106FF00027D1596841F480415960B4E718F0400F37
:10700000B1D0638D9BB2C3B1238DB3B92068416801
:10701000638DC1F309019BB2FF2B26D94368FF277B
:10702000204E27853340204E19430E4346609AE791
:10703000996941F00101996195E723685B689801BE
:1070400003D42046FBF796FA8DE740212046FFF750
:1070500073FC88E720462946FFF7F6FD002084F8F8
:107060004000BDE8F08102207047638DE66A9BB264
:1070700016F5803F23850AD0E76ADBB24668094AE5
:1070800016403E4346EA0343194341606BE74668B6
:10709000DBB2044F3E40314341EA034343F0007307
:1070A000436060E7009C00FC0000FF01F0B4044670
:1070B00090F834000128A66D38D0012594F83500E9
:1070C000A84284F8345005D00023022084F83430DC
:1070D000F0BC704725680227002084F83570A76847
:1070E00060652868402F20F4802028606B601AD0EB
:1070F000A960EA60E16D3F23226C8B40B3602B688E
:1071000043F016032B606B6943F080036B611AB187
:107110002B6843F008032B602B68002043F0010329
:107120002B60F0BC7047AA60E960E3E70220F0BC86
:10713000704700BFF0B490F83530022B34D00368AC
:1071400000221B4D2127D9B21E68103926F00106F6
:10715000A5FB0145174C5F291E6004EB15141A604E
:107160005A6094F868409A60DA601A615F61C46599
:1071700015D8114A1A4000233F218265A1401C46C0
:107180009160436580F8343080F83530C0E90F33C2
:10719000C0E91133C0E913332046F0BC7047A2F5B3
:1071A00080621A400432E6E7DCB22046F0BC704749
:1071B000ABAAAAAAC412060800FCFFFF0246F0B45C
:1071C0004A4C2068002A57D002231168002582F813
:1071D000353082F834500B6823F001030B6003E074
:1071E00023681B1A052B3FD80B68DD07F8D4D2E9BA
:1071F0000130D56803430F68D2E904402B43234391
:10720000146AD2E9066503433948334338402B43B7
:10721000556A2343042D40EA030030D008604B69CF
:1072200023F007031D43CBB2324C4D61103B324873
:10723000A4FB03545F2B314B4FF0010500EB1410FE
:107240004FF0000403EA01034FF03F0190F868009B
:1072500088BF04338140D0652046936599605465AA
:1072600082F83550F0BC7047032320211846516541
:1072700082F83530F0BC70470120F0BC7047D2E98D
:107280000B74936A3C43204308604D6925F0070561
:107290001D4345F00405002FC5D07EB1B6F5005F53
:1072A00012D0022B03D9032BBDD1FB01BBD5012387
:1072B00040211846516582F83530D3E7012B11D0B3
:1072C00033F00203AFD1F0E7032BACD801A050F8A4
:1072D00023F000BFAF720108AB720108AF72010862
:1072E000E5720108B7F1C07F9DD1E0E74C35012080
:1072F0003F8010E0ABAAAAAAC412060800FCFFFF58
:107300000C4B93F84221D20703D5012283F8FB21CD
:10731000704793F8FB2162B9D3F880214AB193F802
:107320003821104493F83921114483F8380183F847
:107330003911704730680120044B93F9000001288F
:1073400002D102221A707047002070473068012075
:10735000114AD2F8FC01A0B1D2F800328BB18842B8
:107360000DD88B4234BF002301239BB15368C2F870
:107370000412994202D0142382F80832DCE7002379
:10738000F3E7A1F59C53083BB3F57A7F2CBF0023AC
:107390000123EAE7704700BF30680120002307B5EA
:1073A0000DF10602ADF806300CF00AFC60B1084B96
:1073B000BDF806201989A3F80A22914202D01422AE
:1073C00083F80C22FFF7B8FF03B05DF804FB00BFA1
:1073D0003068012013B50446262001911EF004F9FF
:1073E000019948B9054BD3F82C312BB1204602B096
:1073F000BDE81040FBF7A4BC02B010BD306801200E
:10740000B1FA81F149204909E4E72DE9F341BE4C85
:107410000D4694F90030013300F06681D4F82C3128
:10742000002B00F0B380022700264FF00108D4F8AB
:107430002C012FF0E3FD002800F0A880D4F82C01E7
:107440002FF0D4FDD4F834315A1C234483F80D02B4
:1074500094F83031C4F83421012B09D0022B15D017
:1074600063B90F280CBF84F83081C4F83431DEE7EB
:10747000A0F17203012B06D9762804D084F830617C
:10748000C4F83461D3E784F83071D0E7102ACED144
:107490009E490023012211F8010F013203440E2AF4
:1074A000DBB2F8D194F81B2284F830619A42C4F818
:1074B0003461BCD194F81C32002BB8D194F80E3250
:1074C000732B59D0762B1BD0722B5FD194F81022DE
:1074D00094F80F3294F9001053EA022356D0C4F8FE
:1074E000FC310029B4F81132C4F800324EDC01231B
:1074F00094F82A222370002A48D184F82A3245E0E1
:1075000094F8102294F80F3253EA02233ED0D4F8B4
:1075100020226360934202D0142284F8082294F857
:10752000121294F81122C4F8203242EA0122B4F86F
:1075300024129142228102D0142184F80C1294F872
:10754000131294F81602617094F81412A4F824220D
:10755000A17094F8151241EA0021A4F82612D4F87B
:10756000041209B9C4F80432B4F80A320BB9A4F809
:107570000A220223237009E094F8142294F81332AB
:1075800043EA02231AB20BB1A4F8282294F900307E
:10759000022B35D00FDCDAB2012A15D9A36D13B155
:1075A000E368002B6CD11F2259495A4802B0BDE84C
:1075B000F04149F0A1B8032BF0D1D4F82C32564A4F
:1075C000EB1A9342EADD13E0D4F82C225349AA1AAD
:1075D0008A42E3DD2BB97220FBF7DEFBC4F82C52A4
:1075E000DCE7D4F830325A1CD907C4F8302203D46F
:1075F0007620FBF7D1FBF1E77320FBF7CDFBEDE73E
:10760000D4F80412D1B194F80832BBB1636899423E
:1076100014D06378DA0703D489B24620FFF7DAFE84
:1076200094F80832013B84F8083205F592250323CB
:1076300005F578752370C4F82C52AFE7B4F80A1238
:10764000238981B194F80C226AB18B420BD0637804
:10765000DB0702D45020FFF7BDFE94F80C32013B4B
:1076600084F80C32E1E70122A4F80A3200232270E8
:10767000626884F80C32C4F8042284F808328DE77A
:10768000274D2A23D4F880710DF1070285F81D32A9
:1076900020230DF10601384685F81E320CF027FB39
:1076A00030B19DF806109DF8076051EA06031ED11F
:1076B000552385F81F32462385F82032202362683F
:1076C000184885F82132002A34D017493EF024FFAB
:1076D000B4F8263215488BB3228915499A420CBF5B
